:020000022000DC
:1060000000000420312F0700FDB60200FD3D030013
:10601000FDB60200FDB60200FDB602000000000061
:10602000000000000000000000000000FDB60200BB
:10603000FDB6020000000000FDB60200FDB6020041
:1060400029BE0200FDB6020039CA0200A1C7020043
:10605000B1C70200FDB60200C1CC0200FDB60200CD
:10606000FDB602005D2C0300452C030035CF020075
:10607000FDB60200FDB60200FDB60200FDB602004C
:1060800065CF020045CF0200FDB60200FDB602005A
:10609000FDB60200FDB6020049620600FDB6020030
:1060A000FDB60200FDB60200FDB60200FDB602001C
:1060B000FDB60200FDB60200000000000000000076
:1060C000FDB60200FDB60200FDB602001950030045
:1060D00055CF0200FDB60200FDB602002DB503004B
:1060E00049CA0200FDB60200FDB602002DC0020042
:0860F00000000000FDB60200F3
:1070000040F8044B40F8045B40F8046B40F8047B04
:1070100040F8048B40F8049B40F804AB40F804BBF4
:1070200040F804CB40F804DB6846704781F000412B
:1070300002E000BF83F0004330B54FEA41044FEA5D
:10704000430594EA050F08BF90EA020F1FBF54EAF8
:10705000000C55EA020C7FEA645C7FEA655C00F094
:10706000E2804FEA5454D4EB5555B8BF6D420CDD65
:107070002C4480EA020281EA030382EA000083EAE8
:10708000010180EA020281EA0303362D88BF30BD88
:1070900011F0004F4FEA01314FF4801C4CEA1131DE
:1070A00002D0404261EB410113F0004F4FEA03333D
:1070B0004CEA133302D0524263EB430394EA050FC8
:1070C00000F0A780A4F10104D5F1200E0DDB02FA37
:1070D0000EFC22FA05F2801841F1000103FA0EF2CB
:1070E000801843FA05F359410EE0A5F120050EF191
:1070F000200E012A03FA0EFC28BF4CF0020C43FAC2
:1071000005F3C01851EBE37101F0004507D54FF0CE
:10711000000EDCF1000C7EEB00006EEB0101B1F51E
:10712000801F1BD3B1F5001F0CD349085FEA300064
:107130004FEA3C0C04F101044FEA445212F5800F6F
:1071400080F09A80BCF1004F08BF5FEA500C50F10C
:10715000000041EB045141EA050130BD5FEA4C0CEF
:10716000404141EB0101013C28BFB1F5801FE9D24C
:1071700091F0000F04BF01460020B1FA81F308BF6F
:107180002033A3F10B03B3F120020CDA0C3208DD3B
:1071900002F1140CC2F10C0201FA0CF021FA02F116
:1071A0000CE002F11402D8BFC2F1200C01FA02F186
:1071B00020FA0CFCDCBF41EA0C019040E41AA2BFAB
:1071C00001EB0451294330BD6FEA04041F3C1CDA73
:1071D0000C340EDC04F11404C4F1200220FA04F093
:1071E00001FA02F340EA030021FA04F345EA03013D
:1071F00030BDC4F10C04C4F1200220FA02F001FAFF
:1072000004F340EA0300294630BD21FA04F0294680
:1072100030BD94F0000F83F4801306BF81F4801119
:107220000134013D4EE77FEA645C18BF7FEA655C8C
:1072300029D094EA050F08BF90EA020F05D054EA5E
:10724000000C04BF1946104630BD91EA030F1EBF63
:107250000021002030BD5FEA545C05D14000494167
:1072600028BF41F0004130BD14F580043CBF01F55A
:10727000801130BD01F0004545F0FE4141F4700140
:107280004FF0000030BD7FEA645C1ABF194610461B
:107290007FEA655C1CBF0B46024650EA013406BF1C
:1072A00052EA033591EA030F41F4002130BD00BFDB
:1072B00090F0000F04BF0021704730B54FF4806498
:1072C00004F132044FF000054FF0000150E700BF19
:1072D00090F0000F04BF0021704730B54FF4806478
:1072E00004F1320410F0004548BF40424FF0000165
:1072F0003EE700BF42004FEAE2014FEA31014FEAA8
:1073000002701FBF12F07F4393F07F4F81F06051F6
:10731000704732F07F4208BF704793F07F4F04BF41
:1073200041F40021704730B54FF4607401F000451E
:1073300021F000411CE700BF50EA010208BF70477E
:1073400030B54FF000050AE050EA010208BF70476F
:1073500030B511F0004502D5404261EB41014FF4D8
:10736000806404F132045FEA915C3FF4D8AE4FF0E0
:1073700003025FEADC0C18BF03325FEADC0C18BFC3
:10738000033202EBDC02C2F1200300FA03FC20FA14
:1073900002F001FA03FE40EA0E0021FA02F1144461
:1073A000BDE600BF4FEA4102B2F1E04324BFB3F5AE
:1073B000001CDCF1FE5C0DD901F0004C4FEAC0026C
:1073C0004CEA5070B2F1004F40EB830008BF20F050
:1073D0000100704711F0804F21D113F13872BCBF0A
:1073E00001F00040704741F480114FEA5252C2F15F
:1073F0001802C2F1200C10FA0CF320FA02F018BFA8
:1074000040F001004FEAC1234FEAD32303FA0CFCFA
:1074100040EA0C0023FA02F34FEA4303CCE77FEA89
:10742000625307D150EA01331EBF4FF0FE4040F4D3
:107430004000704701F0004040F0FE4040F4000082
:10744000704700BF53B94AB9002908BF00281CBFC4
:107450004FF0FF314FF0FF3000F0B8BAADF1080C3B
:107460006DE904CE00F026F8DDF804E0DDE9022342
:1074700004B07047D0B5FFF73DFF0C4B0022064625
:107480000F4600F079F900F0A3FA0446FFF710FF69
:10749000074B002200F070F902460B463046394691
:1074A000FFF7C8FD00F094FA2146D0BD0000F03D82
:1074B0000000F0412DE9F047089D04468C46002B62
:1074C00040F083808A42174647D9B2FA82F242B12D
:1074D000C2F1200024FA00F09140974040EA010CEC
:1074E00094404FEA1748230CBCFBF8F61FFA87FEBE
:1074F00008FB16C143EA014306FB0EF1994209D984
:10750000FB1806F1FF3080F01981994240F2168194
:10751000023E3B445B1AA4B2B3FBF8F008FB103305
:1075200044EA034400FB0EFEA64509D93C1900F1CC
:10753000FF3380F00581A64540F2028102383C44C9
:1075400040EA0640A4EB0E0400261DB1D4400023FF
:10755000C5E900433146BDE8F08702B9FFDEB2FA63
:1075600082F2002A50D1CB1B4FEA174E1FFA87F840
:107570000126B3FBFEFC210C0EFB1C3341EA034148
:1075800008FB0CF38B4207D979180CF1FF3002D2BB
:107590008B4200F2E9808446C91AA3B2B1FBFEF027
:1075A0000EFB101143EA014408FB00F8A04507D97F
:1075B0003C1900F1FF3302D2A04500F2D9801846F1
:1075C000A4EB080440EA0C40BFE78B4209D9002D28
:1075D00000F0B1800026C5E9000130463146BDE823
:1075E000F087B3FA83F6002E4AD18B4202D382424F
:1075F00000F2B880841A61EB030101208C46002D53
:10760000A8D0C5E9004CA5E7C2F1200320FA03F693
:10761000974001FA02F04FEA174ED9403043030C6D
:10762000B1FBFEF61FFA87F80EFB161143EA014381
:1076300006FB08F1994204FA02F409D9FB1806F195
:10764000FF3C80F08D80994240F28A80023E3B44AC
:107650005B1A81B2B3FBFEF00EFB103341EA03412B
:1076600000FB08F38B4207D9791800F1FF3C73D275
:107670008B4271D902383944CB1A40EA064678E782
:10768000C6F1200C03FA06F422FA0CF31C4320FA8C
:107690000CF701FA06F34FEA144E21FA0CF11F43DE
:1076A0003B0CB1FBFEF91FFA84F80EFB191143EAFB
:1076B000014109FB08FA8A4502FA06F200FA06F3CC
:1076C00008D9611809F1FF3048D28A4546D9A9F195
:1076D00002092144A1EB0A01BFB2B1FBFEF00EFB8F
:1076E000101147EA014700FB08F8B84507D9E71928
:1076F00000F1FF312ED2B8452CD90238274440EA98
:107700000940A7EB0807A0FB02894F45C64649463A
:107710001AD317D05DB1B3EB0E0267EB010707FA7E
:107720000CFCF2404CEA0202F740C5E900270026B3
:107730003146BDE8F0872E4628460BE70646E9E6C7
:107740001846FDE64345E5D2B8EB020E69EB0401AD
:107750000138DFE70846D2E760468DE78146B9E7A2
:10776000664675E730464AE7ACF1020C394413E748
:1077700002383C4424E700BF70B54FF0FF0C4CF4D6
:10778000E06C1CEA11541DBF1CEA135594EA0C0F5F
:1077900095EA0C0F00F0DEF82C4481EA030621EA9A
:1077A0004C5123EA4C5350EA013518BF52EA0335D5
:1077B00041F4801143F4801338D0A0FB02CE4FF087
:1077C0000005E1FB02E506F00042E0FB03E54FF0B7
:1077D0000006E1FB03569CF0000F18BF4EF0010EAF
:1077E000A4F1FF04B6F5007F64F5407404D25FEAAB
:1077F0004E0E6D4146EB060642EAC62141EA55515E
:107800004FEAC52040EA5E504FEACE2EB4F1FD0C9F
:1078100088BFBCF5E06F1ED8BEF1004F08BF5FEA1D
:10782000500E50F1000041EB045170BD06F00046CF
:1078300046EA010140EA020081EA0301B4EB5C047C
:10784000C2BFD4EB0C0541EA045170BD41F4801174
:107850004FF0000E013C00F3AB8014F1360FDEBF99
:10786000002001F0004170BDC4F10004203C35DA75
:107870000C341BDC04F11404C4F1200500FA05F3F8
:1078800020FA04F001FA05F240EA020001F0004299
:1078900021F0004110EBD37021FA04F642EB06010F
:1078A0005EEA430E08BF20EAD37070BDC4F10C0439
:1078B000C4F1200500FA04F320FA05F001FA04F2FD
:1078C00040EA020001F0004110EBD37041F10001E9
:1078D0005EEA430E08BF20EAD37070BDC4F12005F4
:1078E00000FA05F24EEA020E20FA04F301FA05F25C
:1078F00043EA020321FA04F001F0004121FA04F204
:1079000020EA020000EBD3705EEA430E08BF20EAD3
:10791000D37070BD94F0000F0FD101F0004640000D
:1079200041EB010111F4801F08BF013CF7D041EA8F
:10793000060195F0000F18BF704703F00046520093
:1079400043EB030313F4801F08BF013DF7D043EA64
:107950000603704794EA0C0F0CEA135518BF95EA1A
:107960000C0F0CD050EA410618BF52EA4306D1D1A1
:1079700081EA030101F000414FF0000070BD50EAC0
:10798000410606BF1046194652EA430619D094EA4A
:107990000C0F02D150EA013613D195EA0C0F05D134
:1079A00052EA03361CBF104619460AD181EA030188
:1079B00001F0004141F0FE4141F470014FF0000040
:1079C00070BD41F0FE4141F4780170BD704700BFC9
:1079D0004A0011D212F5001211D20DD56FF478734E
:1079E000B3EB62520ED44FEAC12343F0004343EAA3
:1079F000505323FA02F070474FF00000704750EAEE
:107A0000013002D14FF0FF3070474FF00000704757
:107A1000024BDA691268DA61704700BFB84501208D
:107A2000C460056146618761C0F81C80C0F8209081
:107A3000C0F824A0C0F828B0C0F82CD080ED0C8B82
:107A400080ED0E9B80ED10ABC0F808E03EF06EBA02
:107A50002DE9F0412A4C00250326D4F8F0700021CE
:107A6000013143189A0803F00303BA5C5B0042FA41
:107A700003F303F00303022BF2D0D4F8FC30090126
:107A80008A0803EB001089B300EB82020368190730
:107A900029D1D4F8FC10994225D8D4F800719F421E
:107AA00021D95B1A48BF0F331B11D4F8F0E04FEA1D
:107AB000930C03F003011EF80C80490048FA01F70B
:107AC00007F00307012F0ED106FA01F141EA080180
:107AD00004EB85083F2D0EF80C109ABF0135C8F84D
:107AE0000C31C4F8087104309042CFD12DB1013D62
:107AF00004EB8503D3F80C01AFE7BDE8F08100BFCC
:107B0000B8450120124BD3F8FC20824217D8D3F895
:107B10000011884213D230B4801A48BF0F300011D0
:107B2000D3F8F040810800F00303655C5B0045FA80
:107B300003F202F00302012A02D030BC7047704702
:107B4000032202FA03F31D43655430BCFFF780BFE4
:107B5000B8450120174AD2F8FC30834219D8D2F830
:107B60000011884215D210B4C01A48BF0F3003115B
:107B7000D2F8F0409A0803F00301A25C49000A41E0
:107B800002F00302012A4FF0000004D05DF8044B1C
:107B900070470020704701301A18910802F0030264
:107BA000615C520041FA02F202F00302022AF2D0B2
:107BB0000001EBE7B8450120030701D1FFF7A2BFA1
:107BC000704700BF61B138B5041F04EB810554F85C
:107BD000040F030701D1FFF795FFAC42F7D138BD81
:107BE000704700BF2DE9F0473B4CD4E93F1200231A
:107BF000C0E90233C0E90433521AC0E900231D462C
:107C000083619C461F4619461A469A4699469E46E7
:107C1000D4F8F06016F80A304FEA490943FA09F33C
:107C200003F00303012B4DD0022B47D0002B3ED095
:107C3000D4F8F4600132B2EB860F4FEA86080FD019
:107C4000D4F8F0604FEA920A02F0030916F80A30FD
:107C50004FEA4906334113F0030301D0012BD7D17A
:107C6000012911D0022902D146690136466186698F
:107C70008E4238BF816190450FD0012B26D04FEA4C
:107C8000920A02F00309C3E70669013606618669B4
:107C90008E4238BF81619045EFD1774500D9C760EA
:107CA0002D014FEA0C13C0E90153BDE8F0870CF138
:107CB000010CC0F808C001371946B9E70135456025
:107CC0000131B5E7013545601946B1E7BE4501D23E
:107CD000C760BE460027D2E7B8450120030701D19F
:107CE000FFF738BF00207047014488420ED241F2AE
:107CF000055310F8012B03EB4313814283EA02037F
:107D0000F7D1D8B2012838BF01207047052070474D
:107D1000074B1B6A5A68904203D21B685A6890420C
:107D2000FBD3821A043253F822301878704700BF10
:107D3000B8450120074B1B6A5A68824203D91B6869
:107D40005A689042FBD3821A043253F82230587892
:107D5000704700BFB8450120074B1B6A5A68904224
:107D600003D21B685A689042FBD3821A043253F83C
:107D700022000230704700BFB8450120084B1B6A43
:107D80005A68824203D91B685A689042FBD3821A10
:107D9000043253F8220043780B600230704700BF72
:107DA000B84501202DE9F04F8946014648448142FB
:107DB00083B043D20B4641F2055613F8012B06EB74
:107DC0004616984286EA0206F7D1F6B2012E38BF6F
:107DD00001261B4BD3F820A0BAF1000F2AD0DAF805
:107DE0000C700AF1100B0BEB8707BB451DD25C46EC
:107DF00001E0A74219D9A04654F8040B0578B54212
:107E0000F7D142784A45F4D102304A4601914FF009
:107E100081FE01990028ECD1DAF80400A8EB0B08E8
:107E200000EBA80003B0BDE8F08FDAF800A0BAF1CB
:107E3000000FD4D1504603B0BDE8F08F0526C8E747
:107E4000B845012043688B422CBF5B1A0023436076
:107E5000704700BF70B546688E4206D90B46114484
:107E60008E420446154601D8436070BD8068721A80
:107E7000014418444FF010FE6268521B626070BDEE
:107E800070B5054608460E464FF066FE044620B122
:107E9000D5E90003314622469847204670BD00BF11
:107EA0002DE9F84F9DF828400B9E14F0DF0F914606
:107EB00005468A46A6EB02023AD0302C0AA9244E87
:107EC0000EBF10270E46012713F0800836D002EBB4
:107ED000D278A2EB68044FEA6808B8F1000F32DDEF
:107EE000C3465F453A46A8BF5A46ABEB020BD5E9FD
:107EF000000331469847BBF1000FF2DCB9F1000FE7
:107F000005D0D5E9000351464A469847C844002C9D
:107F10000BDDA044A7423A46A8BF2246A41AD5E9E1
:107F2000000331469847002CF4DC4046BDE8F88F4A
:107F300013F08008074E4FF01007C8D113F001046A
:107F400004D01446DAE74FF00008D7E79046C4E7BC
:107F5000F84E0800E44E08002DE9F04788B00024F0
:107F60001F469DF84890119B139D8DF80F40804649
:107F700032B1A1421BDB9A074DD52B228DF80F2081
:107F8000C9B930218DF81F100DF11F0613F0400400
:107F90002BD09ABB144608AACDE900954046921B07
:107FA0003146FFF77DFF204408B0BDE8F0872D2261
:107FB00049428DF80F20109808AE0DF1100EA0F177
:107FC0000A0A01E0BC45E1D3B1FBF7F007FB10144E
:107FD000092C8CBF5444303406F8014D76458C464C
:107FE0000146EFD113F04004D3D1002AD3D004A925
:107FF0008E42D0D906F8012C013ECCE70122CDE912
:1080000000920DF10F0140461193FFF749FF013D2A
:10801000119B0446BFE713F004021CBF20228DF819
:108020000F20ADE790F90010037800291EDA024610
:1080300003F07F005B0605D5402320EA03005B08C0
:108040001842FAD1517801F0C003802B10D110B43E
:10805000531C01F03F0413F8011F01F0C002802AF5
:1080600044EA8010F5D05DF8044B7047184670471D
:10807000704700BF034601305B7803F0C003802BDC
:1080800005D110F8013F03F0C003802BF9D07047F1
:10809000014488420CD2421E0139002012F8013FEF
:1080A00003F0C003802B18BF01308A42F6D170471D
:1080B000002070477F289DBF024B185CC0F3400032
:1080C000002070474CCF07007F289DBF024B185CF3
:1080D000C0F3C000002070474CCF07007F289DBF31
:1080E000024B185CC0F38000002070474CCF0700A3
:1080F0007F289DBF024B185CC0F300100020704722
:108100004CCF07007F289DBF024B185CC0F3401086
:10811000002070474CCF07007F2804D8024B1B5C1F
:10812000DB0648BF203070474CCF07007F2804D8BB
:10813000024B1B5C9B0648BF203870474CCF0700A2
:108140000144884237D210B40022E52406E01B0621
:108150002DD50130531E8142DAB222D90378002A8C
:10816000F5D1BF2B11D81A0621D4421C914208D94F
:10817000104612F8013BBF2B07D81B0617D49142BB
:10818000F6D101205DF8044B7047F72B0FD8DB08C0
:1081900003F00603013044FA03F3814203F00302C3
:1081A000DCD8B2FA82F040095DF8044B7047002039
:1081B0005DF8044B70470120704700BFB2EB131FFE
:1081C00020D9F0B41E0901EB4607961B3246012A5E
:1081D000844603F00F013D46044607D055F8023BA4
:1081E000013ACB40012A24F8023BF7D1701E37F840
:1081F000103023FA01F12CF81010002918BF304676
:10820000F0BC7047002070472DE9F041069FD21B5B
:108210009FB39E1EA1F1020E3D46844600243EF807
:10822000023F36F8028F43442344013D2CF8023BC1
:108230004FEA1344F3D101EB470100EB47076AB162
:108240008D1E3E46114635F8023F0139234426F87B
:10825000023B4FEA1344F6D107EB420744B1012336
:1082600027F8023B3F1A47FA03F21046BDE8F081B7
:10827000381A42101046BDE8F081002AF5D03C467D
:108280000746DDE72DE9F041069D521BDDB39F1E39
:10829000A1F1020E2E46844600243EF8023F37F834
:1082A000028F2344A3EB0803013E2CF8023B4FEA64
:1082B0002344F2D101EB450100EB450502B38E1ECC
:1082C0002F46114636F8023F0139234427F8023B76
:1082D0004FEA2344F6D1531E05EB430305EB42025C
:1082E00003E01A4633F8021929B99842F9D9101A4D
:1082F0004010BDE8F0810232101A4010BDE8F08154
:10830000AB1E2A46F1E72C460546D7E700EB4103B2
:1083100002EB4102A1B110B402E00DD1013908D045
:1083200033F8020D32F8024D001B0028F5DA4FF049
:10833000FF305DF8044B704701205DF8044B704737
:108340000846704710B4D0E9013101EB430399426C
:1083500004464FF0000005D233F8022D994242EA5C
:108360000040F9D323785DF8044BDB0748BF404257
:10837000704700BF2DE9F04FB1B39C18D0E9019AC6
:10838000B9F1000F28D0002503EB02084FF0010CD3
:108390002A463AF8026B103246EA054590F800B0DA
:1083A0001BF0010F274604F1FF3EAEB206D0F643A4
:1083B0005CFA86FC1FFA8CF6CCF3072C71B173457E
:1083C00004F8016C08D07446083A072A4FEA1525CC
:1083D000E4DCB9F10109DCD1BDE8F08F07F8016BED
:1083E0004745F9D03C46EFE71C46C7E7D0E90132E4
:1083F00002EB43039A429FED0B0A0DD29FED0A7ADE
:1084000033F8021D07EE901AF8EEE77A9A42E0EE92
:10841000077AB0EE670AF3D30378DB0748BFB1EE03
:10842000400A70470000000000008047D0E9023297
:1084300093423DBF5A1C826018784FF0FF3070475E
:108440000269272A35D0222A33D0A2F162011329EA
:1084500032D8234BCB40DB4313F001032CD14169CD
:10846000272926D0222924D0722A1BD0662A31D16E
:1084700072291FD110B48469272C20D0222C1ED041
:10848000722A0BD0622A09D1722907D18369272B5E
:1084900015D0A3F12203B3FA83F35B0918465DF804
:1084A000044B70476629E5D0622903D18369272BE5
:1084B0000AD101231846704700231846704701234C
:1084C00018465DF8044B7047A3F12203B3FA83F317
:1084D0005B09EFE7622AEDD17229EBD1E6E700BF35
:1084E0001100090010B503690A2B044648D0092B76
:1084F000C36A04BF073323F007030133C362D4E91F
:10850000051394F87020C4E90413D2B1B4F87220B2
:10851000616E8A423AD0501CA16EA4F872008A5C47
:10852000A2610D2B22D0236953B9D4E90701C4E914
:108530000401626A84F870306366A4F87230A26144
:1085400010BDD4E9010398476369A0610D2B0ED0DB
:10855000013010D163695A1C0DD00A2B0BD094F84E
:1085600070300A22A261002BDDD110BDA0690A2360
:10857000984263610DD094F87030002BF5D0D2E7AB
:10858000836A01221344C0E90A32B8E70022A261DB
:10859000C7E7D4E901039847A061D9E770B502693C
:1085A000541C34D004460D46002609E00DB1636B1F
:1085B00083B12046FFF796FF22690126531C09D09C
:1085C0000A2AF3D01046FFF775FD58B9232A0ED0BA
:1085D0005C2A01D0304670BD63690A2BFAD120466F
:1085E000FFF780FF2046FFF77DFF2269E6E7204680
:1085F000FFF778FF2269501C05D1EBE7FFF772FF08
:108600002269511CE6D00A2A2046F7D1D6E7002677
:10861000E0E700BF30B110F0030304D10279392A3A
:1086200003D0184670470020704783680B6013F032
:108630000100F7D19A07F5D11868034BC01AB0FAB8
:1086400080F04009704700BF34450800B0F59F7FB7
:1086500009D010F0010304D043080CBF0120002012
:108660007047184670470120704700BFB0F5AF7FD4
:1086700009D010F0010304D0430814BF01200020EA
:108680007047184670470120704700BF03685BB110
:1086900013F0030F0BD110B41C798C420AD0106078
:1086A0005DF8044B01207047136018467047106056
:1086B0000120704703F10801116058685DF8044B10
:1086C000000A704701B9704770B51D468B0782B02C
:1086D00003D14E68F3B2934204D02B4602B0BDE8FA
:1086E00070401847360A09D00C1D04EB860654F872
:1086F000041F0190A847B4420198F8D102B070BDA0
:10870000024B89689B22FFF7DDBF00BF5161050066
:10871000024B89686A22FFF7D5BF00BFC933040046
:1087200070B582B00DF105060D46344602F07F03A8
:10873000D20904F8013DF9D1311BA84701ADAC4283
:108740000BD00146224612F8013B63F07F03AA4298
:1087500001F8013BF7D1121B10449DF8043003705F
:1087600002B070BD10B4D0E90943026B19448162B4
:108770002344D0185DF8044B704700BF10B444790F
:10878000032C06D80A46816A114481625DF8044BC5
:1087900070475DF8044BFFF7E5BF00BF30B5437984
:1087A000032B83B004460D460AD8836A01338362E3
:1087B00006490570204603B0BDE83040FFF7B0BF62
:1087C00001210192FFF7CEFF019AF1E77D870200B8
:1087D00070B4C568048FAE8B6B8BC58E33442B444D
:1087E0004579042D234404F1010608BFC46B0687B4
:1087F00008BF44F823201A4670BCFFF7CFBF00BF64
:108800002833D9B2FFF7CABF70B54679032E0D469B
:10881000144607D8826A05700332230A82624470C4
:10882000837070BD0321FFF79DFF230A057044701C
:10883000837070BD30B44479012C13460A4609D0C8
:10884000D0E90241013484604D8CAC42C8BF4C84F5
:10885000002181711B3330BCD9B2FFF7D5BF00BFF7
:1088600030B44479012C13460A4609D0D0E90241BC
:10887000013C84604D8CAC42C8BF4C8400218171A6
:10888000243330BCD9B2FFF7BFBF00BF30B4447946
:10889000012C13460A4607D0D0E902414D8CAC4268
:1088A000C8BF4C84002181712A3330BCD9B2FFF794
:1088B000ABBF00BF38B54479032C0D4611D9C1694F
:1088C000836A51F822406FF00202D21A0321144445
:1088D000FFF748FFE3B2C4F30722057043708270CC
:1088E00038BD816A057000220331134681624370EE
:1088F000827038BD38B54479032C0D4611D9846A8D
:10890000C169C4F5FF4351F822407D3303211C4463
:10891000FFF728FFE3B2C4F30722057043708270AB
:1089200038BD816A057000220331134681624370AD
:10893000827038BD38B54179012909D0D0E90214D7
:1089400001318160658CA942C8BF618400218171B9
:108950005BB90F2A09D84379503A032BD4B20AD90C
:108960000121FFF7FFFE047038BD1933D9B2BDE80D
:108970003840FFF713BF836A04700133836238BD48
:1089800038B54179012909D0D0E902140139816053
:10899000658CA942C8BF6184002181715BB90F2A2F
:1089A00009D84379403A032BD4B20AD90121FFF701
:1089B000D9FE047038BD2233D9B2BDE83840FFF784
:1089C000EDBE836A04700133836238BD70B4DDE9A3
:1089D00003541646C4B14279CC1AA4EB4504012ACB
:1089E000A4F1020409D0D0E902120C448460518C35
:1089F0008C42C8BF548400228271711C43EA052254
:108A0000C9B270BCFFF7CABE4279C91A012AA1EBEC
:108A1000450409D0D0E902120C448460518C8C4288
:108A2000C8BF54840022827143EA0522F1B270BCAF
:108A3000FFF7B4BE4379012B09D0D0E902231144DA
:108A400081605A8C9142C8BF59840023837170475A
:108A50004379012B16D030B4D0E90242558CAC4298
:108A600009DC00228271032B03D8C369826A43F8B0
:108A7000212030BC7047548443790022012B82713D
:108A8000F1D1F6E7704700BF38B5012A43790C46AB
:108A900016D0012B27D0D0E90231013B83604D8CE9
:108AA000AB42C8BF4B840023022A837114D143799F
:108AB000032B1AD90121FFF755FE6A23037038BD35
:108AC000012B09D0D0E90231013383604D8CAB42D8
:108AD000C8BF4B84002383716832D1B22246BDE8FF
:108AE0003840FFF791BE022AF6D1836A01338362D0
:108AF0006A23037038BD00BF4379012B0A460FD0AB
:108B0000D0E9023110B4013383604C8CA342C8BF5A
:108B10004B8400235DF8044B83711621FFF774BE6C
:108B20001621FFF771BE00BF4279012A19D010B596
:108B3000D0E90231013383604C8CA342C4BF4B8423
:108B400042790023032A837105D90121FFF70AFE28
:108B50001823037010BD836A0133836218230370E6
:108B600010BD836A0133836218230370704700BF0E
:108B700030B44579012D14464FEA42030A460BD022
:108B8000D0E90251C3F101032B4483604D8CAB4209
:108B9000C8BF4B8400238371002C18BF1F2130BC39
:108BA00008BF1E21FFF730BE4279012A19D010B547
:108BB000D0E90231013383604C8CA342C4BF4B84A3
:108BC00042790023032A837105D90121FFF7CAFDE9
:108BD0003023037010BD836A013383623023037036
:108BE00010BD836A0133836230230370704700BF76
:108BF0004279012A19D010B5D0E9023102338360DD
:108C00004C8CA342C4BF4B8442790023032A837156
:108C100005D90121FFF7A6FD3123037010BD836A3A
:108C2000013383623123037010BD836A0133836291
:108C300031230370704700BF4279012A19D010B563
:108C4000D0E90231013B83604C8CA342C4BF4B840A
:108C500042790023032A837105D90121FFF782FDA0
:108C60003223037010BD836A0133836232230370A1
:108C700010BD836A0133836232230370704700BFE3
:108C80004379012B17D010B5D0E90212548CA142C0
:108C9000C4BF518443790022032B827105D901217D
:108CA000FFF760FD3323037010BD836A01338362D5
:108CB0003323037010BD836A01338362332303704F
:108CC000704700BF022A38B50D46044613D06379B9
:108CD000012B09D0D4E90232023BA360508C8342BD
:108CE000C8BF53840023A3712A4620462621BDE82D
:108CF0003840FFF789BDFFF717FF2046FFF7C0FF99
:108D0000E5E700BFA2B910B44279012A03460C4638
:108D100007D0D0E90212508C8142C8BF5184002292
:108D20009A71224618465DF8044B1D21FFF76CBD71
:108D3000FFF7C8BF8968806A09090022FFF7E2BF10
:108D40004379012B17D010B5D0E90212548CA142FF
:108D5000C4BF518443790022032B827105D90121BC
:108D6000FFF700FD3423037010BD836A0133836273
:108D70003423037010BD836A01338362342303708C
:108D8000704700BF022910B504461DD06279012A40
:108D900013D0D4E90231033BA360488C8342C4BFA3
:108DA0004B8462790023032AA37106D9204601214E
:108DB000FFF7D8FC2723037010BDA36A20460133B8
:108DC000A3622723037010BDFFF7AEFE2046FFF716
:108DD000B7FFDBE7C1B941790129034616D010B5C9
:108DE000D0E90220013A9A60448CA242C4BF428476
:108DF0005979002203299A710ED918460121FFF7EB
:108E0000B1FC2123037010BDFFF7BCBF826A212390
:108E100001328262037070479A6A184601329A6280
:108E20002123037010BD00BF4379012B0A460DD0EA
:108E300010B4D0E902135C8CA142C8BF598400234E
:108E40005DF8044B83713521FFF754BD3521FFF7E1
:108E500051BD00BF4379012B13D030B4D0E90234A7
:108E6000013B8360658CAB42C8BF63840023837180
:108E700019B130BC3621FFF73DBD30BC3721FFF7BB
:108E800039BD11B13621FFF735BD3721FFF732BDAE
:108E90004379012B13D030B4D0E90234013B836015
:108EA000658CAB42C8BF63840023837119B130BCA9
:108EB0003821FFF71FBD30BC3921FFF71BBD11B1B1
:108EC0003821FFF717BD3921FFF714BD134630B421
:108ED0000A46417983B9012909D0D0E90241023417
:108EE00084604D8CAC4200DD4C84002181713D33A7
:108EF00030BCD9B2FFF7DEBC0129F8D0D0E902417D
:108F00004D8CAC42F1DD4C84EFE700BF4279012A81
:108F100019D010B5D0E90231013B83604C8CA342DB
:108F2000C4BF4B8442790023032A837105D90121F0
:108F3000FFF718FC4123037010BD836A013383627D
:108F40004123037010BD836A0133836241230370A0
:108F5000704700BF38B5B1B14379012B2BD0D0E9B0
:108F60000221033282604C8C94421DDA4A84437998
:108F70000022032B82714FF0470410D8836A01331B
:108F80008362047038BD4379012B19D0D0E90242C5
:108F9000558CAC420CDC81714224032BEED90121AB
:108FA000FFF7E0FB047038BD002282714724F4E72C
:108FB00054844379EFE7836A013347248362E0E70F
:108FC000836A013342248362DBE700BF4379012BCC
:108FD0000A460FD0D0E9023110B4013383604C8CC3
:108FE000A342C8BF4B8400235DF8044B8371432127
:108FF000FFF760BC4321FFF75DBC00BF4379012B45
:1090000009D0D0E90232043B8360518C8B42C8BF47
:1090100053840023837170474379012B17D010B517
:10902000D0E90212548CA142C4BF5184437900227A
:10903000032B827105D90121FFF794FB44230370B0
:1090400010BD836A013383624423037010BD836AB9
:109050000133836244230370704700BF4379012BBF
:1090600017D010B5D0E90212548CA142C4BF51846C
:1090700043790022032B827105D90121FFF772FB8E
:109080004523037010BD836A013383624523037057
:1090900010BD836A0133836245230370704700BFAC
:1090A00038B54379012B12D0D0E90242558CAC423D
:1090B000C4BF548443790022032B827107D9A1F1E4
:1090C00030040121FFF74EFBE4B2047038BD836A1F
:1090D000A1F130040133E4B28362047038BD00BFF3
:1090E000302970B504463BD031292DD02939CDB275
:1090F00000266279012A2ED0D4E90231013BA36017
:10910000488C8342C4BF4B8462790023032AA37135
:1091100021D901212046FFF725FB05709EB1637917
:10912000012B20D0D4E90212508C8142C4BF51845B
:1091300063790022032BA27115D920460121FFF784
:1091400011FBD323037070BD6279012A4FF0DE0555
:109150004FF00106D0D1A36A0133A3622046DCE7B9
:10916000DD250126C5E7A36A0133A3622046E8E7AF
:109170001346032B0A4630B4417913D00129C2F1BA
:10918000010408D0D0E902512C4484604D8CAC42DB
:1091900006DC00218171503330BCD9B2FFF7FEBA32
:1091A0004C84F6E70129F6D0D0E902140131816040
:1091B000658CA942C8BF6184EBE700BF4279012AF0
:1091C00019D010B5D0E90231023B83604C8CA34228
:1091D000C4BF4B8442790023032A837105D901213E
:1091E000FFF7C0FA5423037010BD836A0133836212
:1091F0005423037010BD836A0133836254230370C8
:10920000704700BF30B44479012C01EB020309D050
:10921000D0E902542B448360658CAB42C8BF6384A1
:109220000023837141EA022230BC5A21FFF7B6BA0B
:109230002DE9F04F83B080460C9C01948B46174675
:109240009946002C00F09C80137EA2F81E9043F0FB
:109250000803137602681378002B54D0138D002B6B
:1092600037D04FF0000A554603E0138D01359D427B
:109270002CDAD66A16F83530033B012B06EBC5060F
:10928000F3D8388D0028F0D0002401E0844217DAAA
:10929000FB6A13F83420042A03EBC40304F101042D
:1092A000F4D15B6871689942F0D1DBF800007288F4
:1092B0000023FFF73FFB388D84420AF1010AE7DB08
:1092C000D8F80020138D01359D42D2DBBAF1000F92
:1092D0002ED1019BDBF8000053EA090314D1437936
:1092E000012B09D0D0E9023201338360518C8B42CB
:1092F000C8BF5384002383717A69602103B0BDE83D
:10930000F04FFFF765BA08684379012B09D0D0E91F
:109310000232013B8360518C8B42C8BF53840023CF
:1093200083717A69612103B0BDE8F04FFFF750BA4D
:10933000019BDBF8004053EA090362792DD0012A32
:109340006FEA0A0309D0D4E902120B44A360518CDE
:109350008B42C8BF53840023A3717A6963212046DE
:10936000FFF736FA6379032B5FFA8AFA26D8A36AE5
:1093700020460133A36280F800A003B0BDE8F08F5F
:10938000FB8302681378002B7FF468AF019BDBF846
:10939000000053EA0903A2D0B6E7012ACAF101038B
:1093A00009D0D4E902120B44A360518C8B42C8BF90
:1093B00053840023A3717A696221D0E720460121FA
:1093C000FFF7D0F980F800A003B0BDE8F08F00BF30
:1093D0002DE9F0419446044600268779D0F81480A0
:1093E00086711A4682B0154B46610D466146FFF7FD
:1093F00069F9A36813B102B0BDE8F081E38AA28ADB
:1094000003B182B1009204F128012A4604F124003C
:10941000FFF70EFF003F18BF0127A771C4F81480A3
:1094200002B0BDE8F0811946A06AFFF7A1FEA06A6C
:10943000FFF77AFBE38AA28AE4E700BFED6A050042
:1094400000B583B0CDE900230B4664220021FFF76D
:10945000BDFA03B05DF804FB00B583B0CDE900238D
:109460000B4666224FF0FF31FFF7B0FA03B05DF80C
:1094700004FB00BF4279012A18D010B5D0E90231AF
:10948000013B83604C8CA342C4BF4B8442790121D1
:10949000032A817104D9FFF765F95B23037010BDBE
:1094A000836A013383625B23037010BD836A827118
:1094B000013383625B230370704700BF38B5447982
:1094C000012C0B4614D0D0E90221D21A82604D8CB7
:1094D000AA42C4BF4A8444790022032C827107D96E
:1094E0000221DCB2FFF73EF95C234470037038BD03
:1094F000826ADCB202325C2382624470037038BD3F
:1095000010B54379012B1DD0D0E90223521A826095
:109510005C8CA242C4BF5A84C368002282711A7E46
:1095200042F004021A7643795D31032BCCB204D8A1
:10953000836A04700133836210BD0121FFF712F9C1
:10954000047010BDC368EAE74379012B09D0D0E964
:10955000023204338360518C8B42C8BF5384002392
:10956000837170474379012B09D0D0E90232033B64
:109570008360518C8B42C8BF538400238371704732
:109580002DE9F04F10EE104A002C9DF824500446AF
:109590005EDB002D68D19FEDDB7AF0EEC07AF4EE51
:1095A000477AF1EE10FA02F0200E00F3B880B4EE24
:1095B000400AF1EE10FA80F12182002B01F1FF3810
:1095C00056DB42F02005672D4EF0450E00F07E81FF
:1095D00010EE102A002A55D1662D00F0F0805A1D99
:1095E0009045D8BFCB1F652D40F07A814FF02B08F6
:1095F0004FF0000C5E1C00274FF0650A00224FF070
:109600002E09B2EE047A11E03031C9B204F1010B37
:10961000974221705C4616D0F8EEE77A013230EEC0
:10962000670AB24220EE070A80F2D780FDEEC07AC8
:1096300004F1010B17EE901A0029E5DA3021974268
:1096400021705C46E8D1002BE6D004F8019BE3E7EB
:10965000B4EE400AF1EE10FA9BD62D2504F8015B1A
:10966000B1EE400A013996E704F8015B013992E74F
:1096700042F0200510EE102A002A4EF0450E4FF061
:109680000603A9D0B2F17E5F58D29FED9F7A9F4A20
:10969000DFED9F7A9F4FB4EEC70AF1EE10FAACBF30
:1096A0004FF0310A4FF0300A02F1140920264FF032
:1096B000000C01E0F2EC017AB4EEE70AF1EE10FAE8
:1096C00004D5D7ED007A20EE270AB4444A454FEA84
:1096D000660607F10407EDD110EE102AB2F17E5FA5
:1096E0000DD2DFED897AB4EEE70AF1EE10FA80F2DE
:1096F0005181F2EE047A20EE270A0CF1010C662D5E
:1097000000F02481672D00F08D814FF02D088A1F15
:109710009A4240F35481652D3FF46CAF54E18EF0D2
:1097200049028EF04E038EF0460522706370A570DC
:10973000033400232370201ABDE8F08F764ADFED52
:10974000777A774F02F1140920264FF0000C01E0E0
:10975000F2EC017AF4EEC07AF1EE10FA04D8D7ED0B
:10976000007A20EE270AB44491454FEA660607F1D5
:109770000407EDD1FDEEC07A17EE902A092A05DD27
:10978000DFED687A20EE270A0CF1010C662D00F05F
:10979000CD80652D00F0CC80672D18BF4FF02B08D1
:1097A00040F080811A1D904540F326811A46944569
:1097B000C0F25081134600274FF02B0899E05E1C41
:1097C000B0454FF00008DCBFCB1E8E1E4746C44696
:1097D0004FF0660A002E3FF711AF662D6CD0F1EE08
:1097E000047AB4EEE70AF1EE10FA2ADB661E4FF0B7
:1097F000300B32782E2A3146A2F1300906F1FF37BC
:1098000008D0B9F1090F07D8392A78D1B04287F8C2
:1098100001B005D03E46ECE77278302A11D1013113
:109820004A782E2A00F0098101348C4288BF2246F2
:1098300005D912F8016C02F801698A42F9D1312286
:109840000A70672D27D0B8F1000F3FF472AF364A87
:1098500084F800E082FB0C314FEAEC73C3EBA10308
:1098600082FB0321DA17C2EBA10202EB820203EBB7
:109870008301ACEB410CA3EB420330330CF1300C11
:10988000A37084F8018084F803C00434002323709B
:10989000201ABDE8F08F002BD5D014F8012C302A07
:1098A00005D1631E1C4613F8012D302AFAD02E2A4A
:1098B00008BF04F1FF34C6E76645C4DBF1EE047A65
:1098C000B4EEE70AF1EE10FA90DABCE7002B40F0B4
:1098D0009E8010EE103A1A1E4FF001037FF4D2AEB4
:1098E00000263746B046B446AA461A46672D7FF48E
:1098F00074AF002A23DD1E464FF0670A6AE7013283
:1099000032709EE7FFFF7F7FF8FF7F3FC40C0800A7
:109910001FB14F0AD80C0800DC0C0800AEC59D74BE
:10992000C00C0800CDCCCC3D67666666E0454EDCD9
:109930008A1F9A4200DCCB1F4FF02B085AE6012306
:109940001E464FF0670A59E6B7EE000A26461A4649
:1099500006F801AB531C984528DCCA1E2E23BCF127
:10996000010C637004F1020400F0A180164630235C
:1099700001E0002E77D0BCF1010C04F8013B06F1A8
:10998000FF36F6D122EAE273E0464FF0FF374FF0A0
:10999000660A1FE7BCF1000F62D1662DD4D0672D97
:1099A00076D04FF02B08B7EE000AB0E6002AD5D1EA
:1099B00034461346164690464FF0660A0DE7652D6D
:1099C000A1F107033FF416AEAA46002605E70CEB0B
:1099D0000302013290454CDCA8EB0C08B8F1010FF2
:1099E000A8F1020259D013466244561C67464FF054
:1099F00000084FF0660AEDE68A1FD8E64EF04E03E7
:109A00008EF041052370A3706570033491E610EE6B
:109A1000102A002A7FF436AE5A1D90453FF760AFFA
:109A2000CB1F5DE7BCF1040F25DD8A1F9A4237DCAE
:109A300013464FF02D0800275BE7BAF1660F3FF49D
:109A4000F3AE3026B8F12D0F0A704E701AD00CF11B
:109A5000010CEAE60CF10103D21A22EAE273C3E731
:109A6000B7EE000A4BE622EAE273B0464FF0660A10
:109A7000B3E61A46B8E70CF1FF3226461A4406F858
:109A800001AB67E7BCF1010C08BF4FF02B08CCE637
:109A90004FF0FF32B7EE000AEFE700231A46A3E7C4
:109AA0004FF02D0800263746AA461A461EE722EA3E
:109AB000E2731646E0464FF0FF374FF0660A89E63C
:109AC000704700BF064B0340062B07D000F003038E
:109AD000022B01D000687047024870470248704767
:109AE000070080FFDC420800B848080038B58168EC
:109AF000CB07044615D40846FFF7E4FF4369054643
:109B000005209847E168B1EB600F0DDA49002B6A38
:109B1000A06841F0010104229847E3680133E36043
:109B200038BD024B024DEBE7002038BDD1210500C6
:109B300034450800C30701D4FFF7C4BF004870478D
:109B400034450800820710B5014603D1114B026865
:109B50009A4211D0CB0708D40846FFF7B3FF4369F8
:109B600043B1BDE8104005201847BDE810400A4B3E
:109B700005201847184610BD084B0340062B04D09B
:109B80008068400040F0010010BDC008FEF7D2F828
:109B9000F7E700BFC0400800D1210500070080FFA3
:109BA00038B5154B98421AD0144DA842044620D01F
:109BB000134B984213D0C3070CD4FFF783FF4369BC
:109BC0007BB121460420984758B1401BB0FA80F081
:109BD000400938BD430814BF0120002038BD0020D3
:109BE00038BD2046FFF7AEFF18B1013818BF01207D
:109BF00038BD012038BD00BFEC190800F819080075
:109C0000F4190800704700BF10B4054A054C88607D
:109C10000023C1E9004208465DF8044BCB60704761
:109C2000ED9A0200D846080038B510F001040BD1B7
:109C30000546FFF747FFC36A23B128469847B0FAA5
:109C400080F46409204638BD0024204638BD00BF9A
:109C5000062806BF490041F001000020704700BF00
:109C6000042808D0052804D18868400040F001008D
:109C70007047002070478A68024B0348002A08BFDB
:109C800018467047EC190800F81908000023C1E9CC
:109C90000233074A48600A600268064B9A4201D0C4
:109CA000084670474368C3F317238B600846704724
:109CB000F0CE0700E8450800136803B1704770B4A0
:109CC0004668B41C50F8244066B1043C02E00133FD
:109CD0009E4207D054F8045FA942F8D1023350F8ED
:109CE0002330136070BC7047032A0B7906D013B180
:109CF0000649FEF7C5B80649FEF7C2B813B10549D3
:109D0000FEF7BEB80449FEF7BBB800BF607C070091
:109D1000687C0700507C0700587C0700136803B17B
:109D20007047B1F5587F0CD040F287239942F7D1A4
:109D3000836823F0030343F00203A3F1FF4313609E
:109D40007047436823F0030343F00203A3F1FF438A
:109D500013607047044B0B60037A0B7143688B6090
:109D60000023CB60084670470CF3070010B40122B3
:109D7000044C886000230C6008465DF8044B0A71AF
:109D8000CB6070470CF3070004280AD0052806D1E1
:109D90004868C0F31B10400040F0010070470020ED
:109DA00070474A68034B044832F00F0208BF184658
:109DB000704700BFEC190800F819080010B4C46817
:109DC0000023A4461A465DF8044B1946604700BFBD
:109DD00010B582B0C4680191002301AA0121A047F7
:109DE00002B010BD08B50246FFF7A4FE034BC168E0
:109DF000994218BF12690023936008BD95DB0300E8
:109E000010B50446FFF796FE074BC068984218BF8E
:109E10002469A36823B1E3880B60A368136010BDB5
:109E20000B60136010BD00BF95DB030001F1FF4321
:109E300023F00303072805D8DFE800F00D0F040422
:109E4000180423060020704707EE903AF5EEC07A1A
:109E5000F1EE10FA01D40846704783F0004323F076
:109E6000030141F00201A1F1FF40704707EE903A73
:109E700009490A48F5EE407AF1EE10FA18BF084693
:109E8000704707EE903AFDEEE77A17EE903A5900E8
:109E900041F00100704700BFF8190800EC190800F4
:109EA000C30706D5401000280FDB14BF0120002097
:109EB000704783683BB1037913F0010F14BF4FF073
:109EC000FF3001207047184670474FF0FF30704751
:109ED0001D4B984212D01D4B98420CD010F001033C
:109EE0000FD0401007EE900AB8EEE70A81ED000AA5
:109EF000012318467047B7EE000AF7E79FED140AF2
:109F0000F4E710F0030208D110B5124A0468944235
:109F100082B00FD0184602B010BD022AE9D10E4A15
:109F20000240062AE5D000F1FF4020F0030300EED6
:109F3000103ADBE704300191FEF758FA019901234A
:109F400081ED000AE6E700BFEC190800F8190800E7
:109F50000000000034450800070080FF10B4054AE7
:109F6000054C88600023C1E9004208465DF8044BB7
:109F7000CB6070477D9F0200D8460800D0E90212EE
:109F800003468868824205D2C868511C50F82200F6
:109F9000D96070470020704700487047F4190800E6
:109FA00043681847032A02D00249FDF769BF0249F6
:109FB000FDF766BF787C0700707C0700C268002A46
:109FC00005DDD0E901318B4206DB00207047FCD073
:109FD000D0E901318B42F8DD1A445B00426043F066
:109FE0000100704710B4D1E90143CA681B1B134438
:109FF000002ACCBF03F1FF330133042893FBF2F3B3
:10A000000DD0052807D123EAE370400040F001009D
:10A010005DF8044B704700205DF8044B7047044A1C
:10A0200004485DF8044B002BC8BF1046704700BFC2
:10A03000F8190800EC19080030B4D0E90154C268DE
:10A04000034BCA60C1E90154084630BC0B6070473D
:10A050006057080070B4D0E9026374689C4214D958
:10A06000F16803F18042013A01EB820151F8042FBB
:10A070009D003AB1042A05D00133C360F3685859F2
:10A0800070BC704701339C42F0D1002070BC704717
:10A0900010B4054A054C88600023C1E90042084617
:10A0A0005DF8044BCB60704755A00200D84608000D
:10A0B00010F003020FD102680D4B9A4208D010F045
:10A0C000010306D10B4B9A4202D000231846704779
:10A0D00001231846704710F00103FAD1022AF4D187
:10A0E000054B0340063B18BF01231846704700BFCD
:10A0F0000C40080034450800070080FF10B4054AF2
:10A10000054C88600023C1E9004208465DF8044B15
:10A11000CB6070471DA10200D846080010B50F4B58
:10A12000044680680340062B82B010D0D0E902209C
:10A130000192E368934207D2C05C4000013340F0D3
:10A140000100E36002B010BD002002B010BDC008E5
:10A1500001A9FDF713FE019AEBE700BF070080FF9E
:10A16000F0B5204B0B40062B83B0054632D0D1E929
:10A17000023601939BB11C4B9D4206F1FF3711D073
:10A180001A4B9D4203D10DE0019BA3421FD93C46CF
:10A1900017F8010FA8470234A41B0028F4D1144873
:10A1A00003B0F0BD00213C4617F8012F1046FDF723
:10A1B0008BFF034610461BB1A84701460028EED08E
:10A1C000019B0234A41BA342EDD80029E7D0094823
:10A1D00003B0F0BDC80801A9FDF7D0FD019B0646FC
:10A1E000C8E700BF070080FFF18002000581020080
:10A1F000EC190800F819080001460148FFF7B0BF44
:10A20000B580020001460148FFF7AABFC9800200DD
:10A2100001460148FFF7A4BFDD8002000146014866
:10A22000FFF79EBFF180020001460148FFF798BF8B
:10A230000581020070B40023136010F8014B303C1C
:10A2400005E010F8014B303CE5B2092D07D803EBCF
:10A25000830304EB4303884213600646F1D3304680
:10A2600070BC704710B5012A82B00C4608D000239C
:10A270004FF0FF320120C1E900338A6002B010BD07
:10A28000094B0340062B08D0D0E90220206042236E
:10A290000020C4E9012302B010BDC00801A9FDF7E8
:10A2A0006DFD019AF2E700BF070080FF2DE9F0473E
:10A2B0009942DDF820901AD3B9F1010F0C461F46E0
:10A2C0008046924607BFCE1A0024E41A002602E018
:10A2D000B4420CD04C4408EB040528463A4651469B
:10A2E0004DF018FC0028F3D12846BDE8F087002582
:10A2F0002846BDE8F08700BFF0B5884283B0044629
:10A300000D4665D04B4B9C4243D09D4241D0E20765
:10A3100042D4494E04EA0601062947D0A7071BD0BC
:10A32000454B2B40062B34D0AA0703D1434B2A6858
:10A330009A422ED0E3075CD42046FFF7C3FB836923
:10A340003BB32A4621460220984710B33C4C001BE1
:10A35000B0FA80F040091DE0384A20689042DFD111
:10A360002E40062E25D16768E808FDF7D1FC0626A9
:10A3700017B108B1B8420CD106294FD0D4E9023444
:10A380000093062E43D0D5E902210192009B9A4208
:10A3900031D0002003B0F0BDEB07FAD4264E23469F
:10A3A0002C4604EA060106291D46B7D12E40062E8A
:10A3B0003AD0A807EDD1214B2A689A42E9D1062963
:10A3C00020D0062E6768CFD06868002FD4D0D0E7A1
:10A3D00000F00303022B07D01BB91A4B22689A42E4
:10A3E00090D0012003B0F0BD134B0340062B89D160
:10A3F000F7E7154BA5E720464DF08CFBB0FA80F04F
:10A400004009C7E7E008FDF783FC0746DCE701A940
:10A41000E808FDF7B3FC019A0146B7E7E008694692
:10A42000FDF7ACFC0446ACE7601BB0FA80F04009D5
:10A43000B0E700BFF4190800070080FFB848080023
:10A44000F8190800EC410800856B0700054B034034
:10A45000062B03D083680B60C0687047C008FDF707
:10A460008DBC00BF070080FF10B4054A054C886012
:10A470000023C1E9004208465DF8044BCB607047F9
:10A48000A9200400D846080010B582B0044608464A
:10A4900001A9FFF7DBFF042C0CD0052C07D1019993
:10A4A000FDF7F6FD400040F0010002B010BD0020B5
:10A4B00002B010BD019A034B0348002A08BF18469A
:10A4C00002B010BDEC190800F8190800D0E902121A
:10A4D00003464868824205D2901C013251F82000A0
:10A4E000DA6070470020704710B4054A054C886058
:10A4F0000023C1E9004208465DF8044BCB60704779
:10A50000CDA40200D8460800F8B5184A184C194DD9
:10A510000E4607E0C368A34209D1406B20B103682F
:10A52000AB4208D09042F5D100242046F8BD3060FF
:10A5300001242046F8BD476800F1080505EB8707B0
:10A54000BD424FF00004F0D255F8040B3146FFF73E
:10A55000DBFFAF420444E8D955F8040B3146FFF75E
:10A56000D3FFAF420444EFD8DFE700BF60460800E6
:10A570008D5406006C49080070B50C4684B054F840
:10A58000046B019200230393054603A93068FFF78B
:10A59000BBFF0398019B2246691EC468A047306137
:10A5A000014804B070BD00BFF41908002DE9F04166
:10A5B000184C194D0E460AE010F003020CD1036846
:10A5C000A3420CD1406B28B10368AB420AD0B04221
:10A5D000F2D10120BDE8F0810020BDE8F0811046F5
:10A5E000BDE8F081436803F1804808F1FF3800F1CD
:10A5F000080303EB880843450AD21F4657F8040BAB
:10A600003146FFF7D3FF3B460028E3D1B845F5D8E4
:10A610001868DCE7A84908006C490800830703D1E3
:10A62000064B02689A4202D00549FFF7BFBF054BAF
:10A63000C2689A42F8D10120704700BFA8490800BB
:10A640009C37080095DB030030B583B005460191C7
:10A65000FFF770FA0446FFF7E1FF019900280CBFED
:10A660002846204603B0BDE83040FFF79FBF00BF3B
:10A6700070B50C460646FFF75DFA0546FFF796FFF4
:10A6800018B1A54214BF3069304670BD38B50D46CB
:10A6900004491446FFF7ECFF83682B60C36823600E
:10A6A00038BD00BF704508000B4610B50B49044685
:10A6B0001846FFF7DDFF042C08D0052C04D1806874
:10A6C000400040F0010010BD002010BD8268044B26
:10A6D0000448002A08BF184610BD00BF7045080096
:10A6E000EC190800F819080070B50E49FFF7C0FF13
:10A6F0008368012B03EBD37612DD03F18043013B2A
:10A7000076109B000022C168CD5851F8224041F8D4
:10A7100022500132C168B242CC50A3F10403F2DBF3
:10A72000014870BD70450800F419080010B50246D4
:10A73000FFF700FA0346BDE8104010461B6A0422EA
:10A74000184700BF10B50446FFF7F4F9034620464A
:10A750001B6ABDE81040184710B50246FFF7EAF93A
:10A760000346BDE8104010461B6A0022184700BF90
:10A7700010B50A460146FFF7DDF9BDE810408369D0
:10A780002E201847024608B50846FFF7D3F9006B9C
:10A7900018B10388934218BF002008BDF8B50446DD
:10A7A000022C069F0E461846154615D084B9012482
:10A7B000BD422A46314628BF3A464DF0ABF9002843
:10A7C0000CDB21D1AF4221D02CBF01200020F8BDED
:10A7D000032C0DD10424EBE7BA4201D00020F8BDD0
:10A7E000194630464DF096F9B0FA80F04009F8BDB0
:10A7F000BD422A46014628BF3A4630464DF08AF906
:10A800003B462F461D46DAE70120F8BD601E18BF03
:10A810000120F8BD91B1F8B5041F174604EB81057E
:10A82000002654F8040F3946FFF766FD00B10136E3
:10A83000AC42F6D1700040F00100F8BD0120704735
:10A8400000B583B00A4606490192FFF711FFD0E92F
:10A850000210019A03B05DF804EBFFF7DBBF00BF05
:10A86000704508000A46083050F8041CFFF7D2BFB4
:10A870002DE9F04707460D46014640F245309A461D
:10A880001446FFF77FFF9DF82080D0E9019318F070
:10A89000020F4FF0000618BF9946CAF800601CB3BB
:10A8A00008F0010807E0431C10D00644B8F1000F7F
:10A8B00016D1241A07D02946534622463846C8479F
:10A8C00005440028EFD13046BDE8F087DAF80030C3
:10A8D0000B2BF8D1002EF6D00023CAF80030F2E797
:10A8E00006463046BDE8F0872646ECE710B582B054
:10A8F0001446019361B101AB191838B113461044E5
:10A9000011F8012D03F8012B8342F9D102B010BDDB
:10A91000024601A920464DF091F802B010BD00BFDB
:10A92000014B9869704700BFB8450120014B586939
:10A93000704700BFB8450120024B0348002283F84E
:10A940000E227047B8450120F4190800024B034855
:10A95000012283F80E227047B8450120F41908003F
:10A96000044B054A93F80E02044B002814BF10460E
:10A9700018467047B8450120F8190800EC1908007E
:10A9800000B589B001A8FDF72DF90398400040F00B
:10A99000010009B05DF804FB00B589B001A8FDF71E
:10A9A00021F90298400040F0010009B05DF804FB75
:10A9B000034B18699B68C01A400040F001007047C3
:10A9C000B8450120034A0448B2F80C32013BA2F812
:10A9D0000C327047B8450120F4190800034A0448B6
:10A9E000B2F80C320133A2F80C327047B84501209E
:10A9F000F419080010B404460020226812F8013B44
:10AA000003F07F011B0641EAC010F7D422605DF815
:10AA1000044B7047002210F8013B03F07F011B0636
:10AA200041EAC212F7D41046704700BF10F9013B4B
:10AA3000002BFBDB704700BF08B58068FFF7F6FF0F
:10AA4000FFF7F4FF0430FFF7F1FF008808BD00BFF7
:10AA500008B5136803B108BD3029FCD1FFF7ECFF3E
:10AA6000C00040F00600106008BD00BF08B51368C4
:10AA700003B108BD302904D01B2904BF436813600B
:10AA800008BD4068FFF7D8FFC00040F00600106026
:10AA900008BD00BF30B405784C1E35B916E0AA4297
:10AAA00010D110F8015F5B1A7DB1234614F8012F15
:10AAB0000233002AF3D17F2D0ED80B4B5B5D13F0D0
:10AAC0000C0F0CD0002030BC704719440A78B2FA41
:10AAD00082F0400930BC7047012030BC7047B5F1AE
:10AAE0005F0018BF0120EEE74CCF0700002813DD00
:10AAF000002908DD6FF0404393FBF1F18142ACBFC8
:10AB00000020012070474FF0404393FBF0F0884253
:10AB1000D4BF002001207047002908DD4FF04043DA
:10AB200093FBF1F18142D4BF00200120704738B17E
:10AB30006FF0404393FBF0F08142ACBF0020012056
:10AB4000704700BFD0E9023293420DD010B4D0E973
:10AB500000415A1C82608A42E35C24BF002282606A
:10AB60005DF8044B184670474FF0FF30704700BF48
:10AB700030B40346D3E90154C068421C954298BFE3
:10AB80000022944205D01C6821540020DA6030BCB9
:10AB900070474FF0FF30FAE74268D0E902031344F0
:10ABA0001B1AB3FBF2F002FB103070472DE9F041A5
:10ABB00004461046D2B101EB020EE6680EF1FF3EEC
:10ABC0004D1EC1F1010C00E01E46D4E90171731C59
:10ABD000BB4228BF002399420CEB050815F8017F02
:10ABE00006D0216875458F55E360EDD1BDE8F08151
:10ABF0004046FBE712B32DE9F0414C1E0346C1F17C
:10AC0000010C04EB02084FF0000ED3E90256B542E6
:10AC100005F101010CEB04000ED0D3E90067996047
:10AC2000B942755D28BF7146996004F8015F4445DB
:10AC3000EBD11046BDE8F0810246FAE710467047B6
:10AC40002DE9F04F074683B00C469346002A40F0AA
:10AC5000068201F10C053B78D4F800903846002BB1
:10AC60006CD009F10202AA1801924E464FF000087A
:10AC7000292B58D05E2B00F2C081232B40F2998102
:10AC8000A3F124023A2A00F29481DFE812F0A10134
:10AC90009201920192015601920127010C01920149
:10ACA0009201BD00920192019201920192019201E2
:10ACB00092019201920192019201920192019201FC
:10ACC000920192019A0092019201920192019201E5
:10ACD00092019201920192019201920192019201DC
:10ACE00092019201920192019201920192019201CC
:10ACF000920192019201920192019201C6005A00C2
:10AD000092013B00002D00F0A68123685022591CBF
:10AD10002160EA54266863680133384663604378EB
:10AD2000471C002BA4D13846B8F1000F06D02DB136
:10AD30002368013BA3EB080305F8083003B0BDE826
:10AD4000F08F7A78781C002A00F0818142F020018F
:10AD50006429266800F0458122F0040242F02002B6
:10AD6000732A00F03E81002D00F09781721C226052
:10AD70004FF00102AA552268797802F1010CA1F185
:10AD80006107C4F800C02A44172F00F24682DFE8AA
:10AD900017F043026E024402440244026B02440272
:10ADA000440244024402440244024402680244024F
:10ADB0004402440265024402440244026202440224
:10ADC0005F022268B24200F04281002D00F05581FE
:10ADD00005EB060AB01C921B514628444CF05CFE61
:10ADE0002368023323607B783F2B00F01C826123B1
:10ADF000AB5538462368023B9E1B8AF801602668E3
:10AE00006368013363608AE72668002D00F0E981FA
:10AE1000721C02232260AB557DE77B7826685E2B8F
:10AE200000F0BA81781C002D00F0E581721C03232C
:10AE30002260AB55D4E9002301330132C4E9002379
:10AE40007B785D2B08BF00212AD00021002B00F069
:10AE5000FE805C2B00F057812368002D00F08D816F
:10AE60005A1C22600278EA54236842782D2A00F0A6
:10AE7000448102785C2A00F01381002D00F080816B
:10AE80005A1C22600278EA54024653785D2B01F185
:10AE9000010102F10100D9D1002D3FF440AFC9B248
:10AEA000AB1959703BE72368B34200F0D0807A7841
:10AEB0003F2A00F08E81002D00F0A7816222EA5423
:10AEC00038462368C3F1FE022B4416445E702368A3
:10AED00062689E1C0132C4E9006220E72268B24227
:10AEE00000F0B580002D00F0D08005EB060AB01C04
:10AEF000921B514628444CF0CFFD23680233602258
:10AF00002360EA542268F1B2C2F1FE032A440B44E2
:10AF100053702368023323607B783F2B00F06781F6
:10AF20006123AB5538462368023B5B1A8AF801302F
:10AF30002668636802336360F1E67B7826683F2BFE
:10AF400000F03F81A36803F1010AC4F808A0002DB6
:10AF500000F04A81721C7E232260AB5522684FEAC2
:10AF60004A03511C2160AB546368013363600123C1
:10AF7000781C5A4621460093FFF762FE002866D0EF
:10AF80000278292A63D1009B002B3FF4C8AE2368C6
:10AF9000002D00F04C81591C7E222160EA54236868
:10AFA0004FEA4A0A0AF1010A5A1C226005F803A076
:10AFB00026E72668002D00F01181731C23604FF0F6
:10AFC0000103AB5523685A1C22603A78EA54A2E682
:10AFD000002D40D023685122591C2160EA54266874
:10AFE00099E6002D59D0721C05232260AB552368C9
:10AFF0005A1C22607A78EA5402E77C2BD9D1B8F146
:10B00000000F2ED07DB32368013BA3EB080305F8A6
:10B0100008302268019805EB09063146A2EB0902C7
:10B020004CF03AFD2368EA186021033323609170E5
:10B03000D4F80080612308F10102226005F809308C
:10B040002368023BA3EB09037370266810E000201D
:10B0500003B0BDE8F08F2668013626605BE6002568
:10B06000F9E5002DD5D123681E1D266003F10308E4
:10B07000636802333846636051E6961C26607B782D
:10B080003F2B00F0E3803846BAE6161D26607B7839
:10B090003F2B00F0C48038464BE7B31C2360AFE67B
:10B0A000421C002D75D0407803F1010CA0F161071E
:10B0B000C4F800C02B44172F0ED8DFE807F00CAA05
:10B0C0000D0D0D1B0D0D0D0D0D0D0D180D0D0D158F
:10B0D0000D0D0D120D0F07201870D6E65C201870AC
:10B0E000D3E60B201870D0E60D201870CDE60A20AC
:10B0F0001870CAE60C201870C7E682785D2A3FF403
:10B10000B8AE0230B6E6471C002D3DD02368427829
:10B1100003F1010CA2F16100C4F800C02B44172810
:10B120000ED8DFE800F00C740D0D0D250D0D0D0D82
:10B130000D0D0D200D0D0D1B0D0D0D160D11072202
:10B140001A702368384690E65C221A7023683846E5
:10B150008BE60B221A702368384686E60D221A7099
:10B160002368384681E60A221A70236838467CE64E
:10B170000C221A702368384677E60133236074E6A0
:10B1800001332360024680E623680133384623609A
:10B190006BE60133236078E6002D4BD0721C04234C
:10B1A0002260AB55D4E9002301330132C4E9002306
:10B1B000BB785D2B07F1020008BF00217FF445AE8C
:10B1C0006DE6BB783A2B7FF4BDAE002302379A467A
:10B1D000CEE635B36122EA54781C72E6B31C2360D4
:10B1E00099E5731C236096E5B31C2360BCE66223DB
:10B1F000AB55781C97E66368B21C0133C4E90023A1
:10B200007B785D2B7FF421AE89E5384660E6082225
:10B2100096E70820187038E607211170F0E5781CD1
:10B2200087E6781C54E66223AB55781CE2E50233CE
:10B230002360E5E56368B21C0133C4E90023BB78F1
:10B240005D2B07F102007FF400AE68E5781CD7E5BE
:10B2500019461170D4E50B211170D1E50D21117043
:10B26000CEE50A211170CBE50C211170C8E508214B
:10B270001170C5E52DE9F84303782F2B06460F46DC
:10B2800029D0DFF88480D8F8D8502DB13E60D8F8A6
:10B29000D8502846BDE8F883002BFAD0D8F8DC5007
:10B2A0004FF0000965B9F1E7296801314CF07AFCEB
:10B2B000321918B9335D2F2B1ED0FBB1ED68B5B133
:10B2C0006C68013C30462246EED1A6EB09063E6092
:10B2D0002846BDE8F88345780136002DD9D0DFF83F
:10B2E0002880D8F8DC502DB14FF00109E8E7B9F11A
:10B2F000000FCBD00125CCE73A60CAE7014B3B6099
:10B30000C7E700BF807C0700B845012030B5C3887F
:10B310008288934285B0044611D3172A16D9014674
:10B32000012551F8080B009503AB1822FFF7A0FA8E
:10B33000039B80B2A0804BB940B12A4601E05A1C61
:10B3400092B22344E280187A05B030BD4FF0FF304E
:10B3500005B030BD38B50446D0E90005954228BF98
:10B3600015462A464CF06AFBD4E900322B44521BA6
:10B37000C4E9003238BD00BFBFF34F8F0549064B0B
:10B38000CA6802F4E0621343CB60BFF34F8F00BF83
:10B39000FDE700BF00ED00E00400FA0541DF704763
:10B3A00012DF704708B50748074BD3F80415D0E9FA
:10B3B00002234909521843F10003C0E90223FFF7B1
:10B3C000DBFF00BFC8480120004002407F292DE973
:10B3D000F04104462CDDA1F180053B2D0CD98B11E9
:10B3E00001F03F0163F03F0361F07F0103704170A2
:10B3F00002263046BDE8F081FDB91A4F20214FF0FA
:10B4000009082046FFF7E2FF0135002645452F4495
:10B4100004440644EDD2204617F8011BFFF7D6FF7F
:10B420000135454504440644F5D33046BDE8F08176
:10B43000017001263046BDE8F0810B4B19445A5D7E
:10B4400011F8813C4FEA450808F1020803EB450377
:10B450009044434503D2034F1D46F95CD1E70026D3
:10B46000C7E700BFECA50800A8A508002DE9F04F2C
:10B4700090F80090457883B009F101038846019364
:10B48000B9F1000F34D01F4F83464FF0000A072454
:10B4900001264FF0000C604663466146490015F0F6
:10B4A000800F03F1010306F1010218BF41F0010111
:10B4B000DBB25CB9D6B207241BF8065008B1814252
:10B4C00009D3FA5C02EB40009444E7E76D00013CCD
:10B4D000EDB2E4B2F2E761440B4B091A08EB0A0043
:10B4E000595CFFF773FF50441FFA80FACA45D0DB5E
:10B4F000019B43440022404603F8012C03B0BDE801
:10B50000F08F00BFC80F080060A008002DE9F843C5
:10B51000DFF8A890254E264C264FDFF8A480322273
:10B520000021054648464CF0CFFA4FF0FF32224941
:10B53000C9F80220C9F80620C9F80A20C9F80E2067
:10B54000C9F81220C9F81620C9F81A20C9F81E2017
:10B550000022C1E90022C1E9022233780A61914642
:10B56000C4B14B4518D8A9EB0303DBB2032B1AD89F
:10B570001BB2C3EBC30307EB83035B682846984702
:10B58000337809F101095FFA89F9DA1C4A45E7DAEB
:10B59000BDE8F8834B46E9E7D8F80030C9EBC902AB
:10B5A00003EB8203E9E700235B68FFDEAC060120C2
:10B5B0000000000000BE0700600F0120FC3B0120DE
:10B5C000A80601200248402200214CF07DBA00BFAD
:10B5D0009C3401200248402200214CF075BA00BF83
:10B5E0009C3401200120704708B50B7803F06003FC
:10B5F000202B09D10A4B8A881878904204D14A78C6
:10B60000202A03D0012008BD002008BD054A002AD9
:10B61000F8D0991D0020AFF30080012008BD00BFC5
:10B62000B0060120000000004DDF70474EDF70477C
:10B630004FDF704750DF704708B1002070470B4B59
:10B64000D3F8DC000028F9D00346C0680028FBD1FD
:10B650009B68002BF2D09A69002AEFD0988800F0FE
:10B660003000203818BF0120704700BFB8450120C6
:10B6700002482C2200214CF027BA00BF38200120BC
:10B6800002482C2200214CF01FBA00BF38200120B4
:10B69000807A400040F00100704700BFC07A40004F
:10B6A00040F00100704700BFF0B41746E9B9013B14
:10B6B00017F8010B9BB20F4A002415462E7A8642DA
:10B6C00005F1140504D00134042CF7D1F0BC704707
:10B6D00004EB840402EB8404227C9A42F6D3E068F3
:10B6E00039461A46F0BC4CF0A9B90229E3D0F0BCA7
:10B6F000704700BFE403012000207047FEE700BF51
:10B7000061DF70474BDF704710B40A4CD4F8D43077
:10B7100063B1D43402E01C461B683BB19A68824294
:10B72000F9D15A688A42F6D11B6823605DF8044B50
:10B73000704700BFB8450120B1DF7047B2DF7047E6
:10B7400070B4144C144E05460020F0B14378FF2B22
:10B7500018D0C388033323F0030308331844A042EE
:10B7600010D84378002BF0D09942EED1FF2907D0B2
:10B77000037803F00103AB42E7D143889342E4D15D
:10B7800070BC7047002070BC7047737802489942C3
:10B79000DBD1EBE7FB1F0B0004A00A0042884378D3
:10B7A000007843EA022340EA032070470B0A017045
:10B7B00043700B0C090E8370C1707047036A023925
:10B7C000023B8B4283BFC389406B01FB0300002017
:10B7D0007047836A02680433D289490AB1FBF2F1E7
:10B7E000186830B1814202D3091A0833F8E7586863
:10B7F0000844704700F10B010022D30143EA5203D1
:10B8000010F8012B52FA83F38842DAB2F5D11046D0
:10B810007047CA7E8B7E032843EA022305D1487D08
:10B820000A7D42EA002243EA024318467047C2F307
:10B8300007238A76CB760378032B03D1120C0A7583
:10B84000120A4A757047000010B40B490023C72242
:10B8500003E0802B0CD031F8022F90429CB203F110
:10B860000103F6D104F1800080B25DF8044B70470B
:10B8700000205DF8044B704700BD070070B4264AF5
:10B88000264BB0F5805F41F67D512CBF13466121F8
:10B8900004330DE081420ED833F8022CD4B265187F
:10B8A000A8424FEA122208DB04337AB133F8041CB1
:10B8B0001E460029EED170BC7047082AFBD8DFE88D
:10B8C00002F00E12181B1E2124270A0036F814104D
:10B8D00006EB4403DCE7A0F5E35080B2EBE7411A46
:10B8E00033F81100E7E7411A01F00103C01A80B2F2
:10B8F000E1E7103880B2DEE7203880B2DBE730388D
:10B9000080B2D8E71A3880B2D5E7083080B2D2E7E3
:10B91000503880B2CFE700BF1CF0070028EE0700C8
:10B92000584BA0F59E00A0F5D05083FB00230344A4
:10B93000C217F0B4544CC2EB234304FB130000289D
:10B9400004DA00F5A83000F5C070013B4F4A504FB3
:10B95000504EA2FB00546409A2FB045252099D1CE4
:10B96000C2EB0212A4EB820287FB05C7C4EB0414EE
:10B97000A6FB00C6A0EB84042F44E817C0EBA70089
:10B98000C0EBC000281A48BF0730F60A002B4A71E6
:10B990008C710E71C87143DB00253F483F4A404C13
:10B9A000A0FB0360C00902FB003384FB03241C449A
:10B9B000DA17C2EB2422042A59D06FF4B67404FBC0
:10B9C00002F492B205EB8000024497B207F5FA65E3
:10B9D0002344ADB21E2B0D804CDD324E1E240020C0
:10B9E0001F2201E016F9014F9B1A9C4200F1010051
:10B9F0002246F7DDC0B2821CD2B20B2A16D9093812
:10BA0000C0B2294A8870441E013332F81400DBB2F8
:10BA100007F2D172CB700A800344F0BC0B817047EF
:10BA200003F50E43AD334FF69C75B6E70330C0B255
:10BA30001D4A8870441E013332F81420DBB2CB70EB
:10BA40001344AA070AD1194A194802FB05F2B0EBC0
:10BA5000B20F03D20133F0BC0B817047134A154873
:10BA600002FB05F5B0EB351FD7D30133F3E7124CDA
:10BA70000322A7E70133DBB20322CB708A703B338A
:10BA8000DFE700BF07452EC2805101008988888802
:10BA900093244992C5B3A29173B06D164BFAFFFF80
:10BAA000B1F98CB3D9F00700E4F00700295C8FC22C
:10BAB000285C8F020AD7A300B9FBFFFFF0B5214C29
:10BAC000059D4E1EC5EB051534F8166002294FF48E
:10BAD0006164324404FB03F3069E4FEA850509D9ED
:10BAE000840725D11849194C01FB00F1B4EBB10FC3
:10BAF0001ED20132DFF868C0154C6FF4C8614118DE
:10BB000004FB0066ACFB0171124CA0F26D77C90911
:10BB1000A0F2CD7E01EB9E003444ACFB0771A0EB9C
:10BB200051101C440C4B10442C4403FB0040F0BD4E
:10BB300005490A4C01FB00F1B4EB311FDAD30132A5
:10BB4000D8E700BFE4F00700295C8FC2285C8F02B1
:10BB50008033E10180569C50805101000AD7A30038
:10BB60001F85EB51002910B414680FDBA14228BFD8
:10BB700021460368002BBCBF1B1903609942ACBF70
:10BB8000C91A00215DF8044B116070472144F0E7A9
:10BB900001291DBF16224FF0FF301A6000207047A8
:10BBA00000487047F419080029DF704728DF704704
:10BBB00010B582B000238DF80730EFF310830D4CE1
:10BBC00023B100232370207802B010BD0DF10700CF
:10BBD000FFF7E6FB9DF80730002BF2D02378012B0E
:10BBE000F1D1FFF7DBFB2378012BFAD0207802B0EC
:10BBF00010BD00BF7C480120074B10B501241C700C
:10BC0000FFF7D2FF08B1002010BDFFF7D1FF0238C7
:10BC100018BF012010BD00BF7C480120F0B500F125
:10BC2000080683B00D4614464FF0FF3702E0A4B279
:10BC300004350436042C2246294628BF042201A8D4
:10BC400001974BF0FBFE012201A93046FFF7D4FF1C
:10BC5000042CA4F10404EAD803B0F0BD00283FD0BE
:10BC6000F0B4364D00232A46904202F1080213D068
:10BC700001330C2BF8D1324B04681A68944257D028
:10BC80004368304F23F003033A6823449A4228D094
:10BC90000023F0BC03607047294F04683A6894425F
:10BCA000426839D122F00302A1180B2B3960EFD082
:10BCB000254E05EBC303002408E0DA68083322F0C0
:10BCC00003029E4211444FF0010404D09A68002AF6
:10BCD000F3D0002CDCD039600023F0BC0360704747
:10BCE00070473C600B22002608E04968531C21F095
:10BCF0000301A4EB01044FF0010608D055F83230DF
:10BD000005EBC201013A002BEFD0002EC0D03C6001
:10BD10000023F0BC036070470A4F22F00302396829
:10BD200022449142B4D13C605A1E002BDBD1AFE7D4
:10BD3000426822F0030222441A60A9E7043D012070
:10BD4000B4410120D84101205C3D012010B5084CD0
:10BD5000206858B1FFF782FF064B93F8501000227D
:10BD600062F3C30183F8501022605A6210BD00BF15
:10BD700098480120080301202DE9F041DFF874C044
:10BD8000DFF87480DCF80070D8F800E0AEEB070351
:10BD9000834210DB82070ED10029154D0BBF01260F
:10BDA0004FF0FF3600230B2355F833209C1932B196
:10BDB000E3B20B2BF8D900221046BDE8F08105EB69
:10BDC000C30261B920F0030145F833700F44CCF889
:10BDD000007005EBC30358601046BDE8F08120F009
:10BDE0000301AEEB010145F83310C8F80010F0E78D
:10BDF000043D0120D8410120B4410120054B064AF1
:10BE00001B681068834203D0C01A0021FFF7B4BF3B
:10BE100000207047D8410120B441012042DF704723
:10BE200043DF704744DF704710B54FF0804386B062
:10BE3000D3F80443620705D5D3F8082103F58473CA
:10BE4000002A4ED1A30603D52A4B1A68002A3FD1F7
:10BE5000600603D5284B1A68002A2FD1210602D587
:10BE6000264B1A680ABBE20502D5254B1A6892B91F
:10BE7000A3050ED5234B1A685AB100221A601A681E
:10BE8000214B0592059A1B68022006B0BDE81040C0
:10BE9000184706B010BD00221A601B4A1B680493A5
:10BEA00001201368049A9847E2E700201860164AB8
:10BEB0001B6803931368039A9847D4E700221A601B
:10BEC000124A1B68029301201368029A9847C5E73B
:10BED000002018600D4A1B6801931368019A984767
:10BEE000B6E700221A600A4A1B6800931368009A9A
:10BEF0009847A7E714010040180100401C010040CA
:10BF00002001004024010040AC450120A84501204B
:10BF1000A445012090F82030FF2B0FD0827F6AB912
:10BF2000C27FA2B11F2B8ABF0F494FF0A04103F07F
:10BF30001F03012202FA03F3C1F80C350022034665
:10BF40004277027253F8082B4168184610471F2B9E
:10BF50008ABF05494FF0A04103F01F03012202FAF6
:10BF600003F3C1F80835E9E700030050F0B50379A1
:10BF7000284C03EBC30104EB8106357F002D41D033
:10BF80008900DA00615800293DD00168DFF894E0AB
:10BF9000DFF894C041F307356D092035C1F3043152
:10BFA000012707FA01F14EF825100168C1F808C30E
:10BFB000707F48B14F61D1F804010028FBD0D01840
:10BFC00004EB800000254577D01804EB800090F842
:10BFD0002100FF280BD01F2886BF00F01F000E4E47
:10BFE0004FF0A04600F5E070022546F820500B48BF
:10BFF00000258142C1F8005507D0134404EB8304A7
:10C0000000232377F0BD0168DEE7054901200860C1
:10C01000F3E700BF0C4401200003005000F0024091
:10C0200004F0024000E100E052010800084BD3F8A0
:10C03000182102B97047002282B0C3F81821D3F842
:10C0400018310193019B034802B0FFF763BF00BFA3
:10C0500000F0024030440120F0B505793E4E044620
:10C0600005EB450006EB800C83B09CF80830002BF4
:10C070006FD180006F0032504A68CCF8042062799A
:10C0800082B11A469C469B00206803F5A0730132DA
:10C0900040F803C0C35860790193D3B29842DDF8E9
:10C0A00004E0F0D82268CB7842F3073000284FEA4A
:10C0B000123246DB00F1604000F561405B01DBB20B
:10C0C00080F800332268254842F3C43323F06043EC
:10C0D00023F0030303F1604303F561434FF0010CC8
:10C0E000C2F304320CFA02F2C3F880211A60D4F8C9
:10C0F00000E04B78DEF8042503F0030322F003028E
:10C100001343CEF80435D4F800E08B78DEF8082528
:10C1100003F0030322F003021343CEF8083524682A
:10C120000B78D4F810253D4406EB850622F00F026B
:10C1300003F00F03134386F808C0C4F8103503B0AA
:10C14000F0BD074802F00F025B011044DBB203763A
:10C15000B8E7044803B0F0BD544401200000AD0B23
:10C16000FCEC00E00500AD0B0379184A03EB430338
:10C1700002EB83031B7A43B3036843F30731490996
:10C1800030B420310124124DC3F3043304FA03F315
:10C1900045F8213003680021D3F80052C3F800129B
:10C1A00003684FF0FF35C3F8085303681C61037937
:10C1B00003EB430302EB83031C72037903EB43039A
:10C1C00002EB8302117230BC704770475444012067
:10C1D00000E100E00F4B984218D003F108029042B2
:10C1E00016D003F11002904205D01833984208BFD0
:10C1F000032201D070470222074910B40023074CE4
:10C200008B54A3545DF8044BFFF7AEBF0022F3E755
:10C210000122F1E74C02012024480120204801209E
:10C220000A7B0346032A11D8DFE802F0121E24021B
:10C230008868194A904228D0886840F202229042C9
:10C2400004D14969D3F84C25914206D101207047A9
:10C250000969D3F84C259142F8D000200622C3F892
:10C260000005C3F8002570470969D3F83C259142C1
:10C27000F3D1EBE7D3F84C2508699042EDD1496939
:10C28000D3F83C259142E8D1E0E7D3F84C25086982
:10C290009042E2D1D0E700BF000204002DE9F04156
:10C2A0001646002280F82E20F26802F06042B2F1B9
:10C2B000005F88B035D19846924BC1F8083390F8AA
:10C2C0002F3005460C4603F0FF0E002B40F0CC80CB
:10C2D000012380F82F30B446BCE80F0005F10C07AD
:10C2E0000FC7DCF800303B6085F830E07378C4F8A5
:10C2F0008835C4F804E1D4F804310193019BC4F8F3
:10C3000024E1D4F824310093009BC4F850E5C4F82C
:10C3100040E53378032B00F2EF80DFE803F045714E
:10C320008507794E304608B0BDE8F081336903F0E7
:10C330006043B3F1005FF4D14FF48073C4F800326E
:10C34000F3687268C4F844350023C4F84825C4F87B
:10C350005031D4F850210492049AC4F86031D4F8D2
:10C3600060210392039AC4F84831D4F8483102930B
:10C370000123029A2362A360D4F85031002BFBD032
:10C380000023C4F85031D4F850310593B2683169B4
:10C390005E4B0598C4F84415C4F84825AB60337863
:10C3A0004FF4827108221CE07368F268C4F84425D7
:10C3B000C4F84835B8F1000F00F08B804FF480735B
:10C3C000C4F80032514AAA600023C4F84831D4F8B6
:10C3D00048310693069B4FF4A471012323623378FE
:10C3E0000822032B4A4E01D00123A3502B68002BB7
:10C3F00042D0AB68C4F80433304608B0BDE8F081E1
:10C400007368F268C4F834254FF48051C4F83835A5
:10C4100040F202220123C4F80012AA60236233789A
:10C420004FF482710022DCE77368F268C4F8442597
:10C43000C4F84835336903F06042B2F1005F7FF41D
:10C4400070AFB068C4F834354FF4845140F2022222
:10C450000123C4F83805C4F80012AA6023623378B7
:10C460004FF482710822BCE72A4E8368C1F8043376
:10C47000304608B0BDE8F0810120214402E0D4F844
:10C480002421DAB90B68002BF9D0D4F8C434C4F8ED
:10C49000C434002285F82F202BB31F481F49204E9B
:10C4A000204A13F0010F18BF064613F0020F18BF01
:10C4B0000E4613F0040F18BF164633E7C4F82431B4
:10C4C000D4F824310793079B20624FF48271606196
:10C4D000D3E74FF4007240F20223C4F800224FF475
:10C4E0008271AB6079E729462046FFF799FE0C4B35
:10C4F000002808BF1E4615E70B4E4FF48271082234
:10C5000072E700BF02029C010A00AD0B00020400AA
:10C510000000AD0B0B00AD0B0000AE0B0100AE0B2D
:10C520000100AD0B0200AE0B0400AD0BF0B5D0F86E
:10C5300024318DB004460D4653B10023C0F8243198
:10C54000D0F824310193019BD0F80431002B74D032
:10C55000D4F80431002B3AD00023C4F8043105F19B
:10C560000C070FCF07AE0FC6D4F8041195F82E3084
:10C570003A6802913260029A002B7FD00023C4F8FF
:10C580006031D4F860210492049AC4F85C31D4F884
:10C590005C2195F830300392039A002B3ED095F839
:10C5A0002E30002B3AD1D4F8C434C4F8C4349A07DE
:10C5B0002DD501238DF8183095F830300BB985F85A
:10C5C0002F30D5E9003106A898470DB0F0BDC4F86A
:10C5D0004831D4F848212B7B0592059A002B3BD19A
:10C5E00005F10C070FCF07AE0FC695F830303A684B
:10C5F0003260002BD7D1274AC4F80032AB60C4F8B0
:10C600000823D4F8C434C4F8C4349A07D1D413F03E
:10C61000050F0BD002238DF81830CDE700231D4AFB
:10C62000C4F80032AB60C4F80823BCE795F82E309C
:10C630006BB304238DF81830BEE78B68C0F808335D
:10C6400002238B608B68C0F80433012303624361CB
:10C6500081F82E300DB0F0BD0E4B4FF4007140F25A
:10C660000222C4F80012AA60C4F80833AB68C4F808
:10C6700004330123A36023620DB0F0BD2946204698
:10C68000FFF7CEFD80F0010085F82E0076E78DF8EB
:10C69000183091E702029C01F0B403792D4934224D
:10C6A00002FB03F28C1894F82D40002C4ED08A58CF
:10C6B000002A4DD00468284E44F307325209203234
:10C6C000C4F30434012505FA04F446F82240047941
:10C6D0000268224F342505FB0414002605FB0315D0
:10C6E000A660C2F8087395F83270D2F800524FF085
:10C6F000010C25F4BC55C2F8005284F82DC0C2F8D4
:10C700000065EFB90268D2F808251F2A86BF02F03B
:10C710001F02134C4FF0A04402F5E072022544F8CA
:10C7200022500268D2F80C251F2A86BF02F01F0291
:10C730000B484FF0A04002F5E072022440F822407E
:10C74000342202FB0313002283F82D20F0BC704733
:10C750001C46BDE76C44012000E100E002029C01A0
:10C760000003005010B40C4C027903680B493420CC
:10C7700000FB024200209060C3F80813D3F80012B7
:10C78000012421F4BC51C3F8001282F82D40C3F8F3
:10C7900000055DF8044B70476C44012002029C01C7
:10C7A00001490248FFF7C2BE6C440120003000403E
:10C7B00002494FF04020FFF7B9BE00BFA04401205E
:10C7C00070B5D0F824318AB004460D46002B6AD0EB
:10C7D0000023C0F82431D0F824210192019AD0F826
:10C7E0008024C0F88024D0F83C05C9680992C5E9C6
:10C7F0000633022208900791D5E9001306A88DF8A8
:10C8000018209847D4F844314BB10023C4F8443180
:10C81000D4F84411AA6903910399002A34D1D4F8B9
:10C82000203153B10023C4F82031D4F820210492E0
:10C8300001220499E2606A69CAB9D4F85831A3B1F7
:10C840000023C4F85831D4F858210592059A6A6932
:10C850005AB1D4F84C15AA6808918DF818306B615C
:10C860000792D5E9001306A898470AB070BDD4F81E
:10C870004C15AA688DF8183008916B610792D5E9BC
:10C88000001306A89847D8E7C5E90633D4F83C3525
:10C89000EA68089301238DF818300792D5E9001350
:10C8A00006A89847BBE7D0F81021002AAAD0C0F804
:10C8B0001031D0F810210292029A8A69D0F83C1502
:10C8C0008A429FD1E96979B1D0F80012EE680892E6
:10C8D00021F02001C0F80012E86929690796C5E92E
:10C8E00006030122E96087E7E868A9610123CDE931
:10C8F00007028DF8183006A8D5E90013984781E79C
:10C90000F0B50179484C01EBC10304EB830383B01C
:10C9100093F82020002A00F084805B68CF0083B168
:10C920000368424AC3F808230268414E42F30733C2
:10C930005B092033C2F30432012505FA02F246F8FE
:10C9400023200268D2F8003223F02003C2F800321C
:10C9500002680123536002680025C2F85851D2F8DA
:10C96000585102680195019DD3600268D2F8583190
:10C97000002BFBD00023C2F8003503684FF0FF3EC8
:10C98000D3F80CC5D3F81465D3F80825D3F810559F
:10C99000C3F80CE5C3F814E50368F445C3F808E5EB
:10C9A000C3F810E50CD0BCF11F0F86BF0CF01F0CB4
:10C9B000204B4FF0A0430CF5E07C022043F82C0004
:10C9C000731C0BD01F2E86BF06F01F06194B4FF0AD
:10C9D000A04306F5E076022043F82600681C0BD041
:10C9E0001F2D86BF05F01F05124B4FF0A04305F524
:10C9F000E075022043F82500531C0BD01F2A86BF88
:10CA000002F01F020B4B4FF0A04302F5E072022030
:10CA100043F82200394404EB8104002384F82030D9
:10CA2000636003B0F0BD00BFD44401201003420096
:10CA300000E100E00003005001490248FFF7C0BEDA
:10CA4000D44401200020004001490248FFF7B8BE4D
:10CA5000F844012000800240F0B4464F3B1893F99F
:10CA60002430002B03DB444AF0BC1046704791F899
:10CA700002C0CCF3400CBCF1000F0CBF0823002314
:10CA800007EB8304A4F104040CBF0926082602E086
:10CA900001339E424ED954F8045F0135F8D13C1859
:10CAA00047F8232084F82430BCF1000F02D1FA1893
:10CAB00082F84C008A7854071CD4D6074BD51F281F
:10CAC00087BF2E4A00F01F0404464FF0A04202EB3D
:10CAD0008402D2F8004724F00204C2F80047284D2F
:10CAE000C40800F0070C2E5D012202FA0CF232435A
:10CAF0002A558A78950721D59B0003F1804303F5D9
:10CB0000C0430C78D3F810551E4A25F44F3525F450
:10CB10004075C3F810552404010201F47C5104F45B
:10CB20004030D3F8104501432143C3F81015104697
:10CB3000F0BC7047144AF0BC10467047083B1F44D5
:10CB4000097897F854300F4A43EA811387F8543034
:10CB50001046F0BC70471F284A7887BF074D00F089
:10CB60001F0404464FF0A04504F5E074920045F818
:10CB70002420B4E71C4501200B00AD0B000300503E
:10CB8000714501200000AD0B0200AD0B174B0344B3
:10CB900093F92430072B0FDD1F288ABF144B4FF069
:10CBA000A04300F01F0003EB8000D0F8003723F40F
:10CBB0004033C0F800377047DAB2072A14D810B4EF
:10CBC0009A0002F1804202F5C0420A4CD2F81005E8
:10CBD000012120F0010001FA03F3C2F81005C4F8A6
:10CBE00008335DF8044B7047704700BF1C450120B7
:10CBF000000300500060004070B50446FFF7C6FF18
:10CC00002C48031993F92420D3B2072B3ED82A4984
:10CC100002F5A272002541F8225000F15502E10808
:10CC200004F00706555CF540ED0702EBD40224D56D
:10CC30001F2C8BBF04F01F052546204B4FF0A0434F
:10CC400005F5E075022143F8251001231178B34062
:10CC500021EA03010319117093F824304FF0FF32D9
:10CC6000072B40F8232003D90344FF2283F84C20EC
:10CC70002044FF2380F8243070BD4FF0FF3240F88D
:10CC800023202044FF2380F8243070BD00F155029A
:10CC9000E10804F00706515CF140C90702EBD40239
:10CCA000C6D44FF0FF3240F823200344FF2283F81C
:10CCB0004C20DDE71C4501200060004000030050CF
:10CCC0002DE9F04F002289B0684B694C6948CDE9E5
:10CCD0000222164615460122196841B1D4F8041300
:10CCE000114204D01D601968009100991643043365
:10CCF00083424FEA4202EFD15F4B1A68002A75D097
:10CD000000221A601B6801934FF0A042019BD2F8E9
:10CD100010255A4B0292D3F81035039316F0FF0FEB
:10CD200040F088804FF0FF3306ADCDE90433002298
:10CD3000534C524F6A6006924FF0010894F95430F8
:10CD4000DAB203F03F00013371D008AB03EBD00E31
:10CD500002F0070C1EF8103C23FA0CF3DB074FEA35
:10CD6000D00964D52318910993F9243054F823305D
:10CD7000002B70D0032970D01F288BBFB9464FF00D
:10CD8000A04902F01F02024609EB82021EF818ECCD
:10CD9000D2F800672EFA0CFC1CF0010FC6F3014913
:10CDA0004BD1B9F1030F42D103294BD14FF4003CD1
:10CDB000D2F8001721F4403141EA0C01C2F8001703
:10CDC0000BB1032198474FF0A043029AD3F8100506
:10CDD000D7F81035824202D1039A9A4227D0DDE972
:10CDE0000612CDE90203CDE90412A7E716F0FF0F02
:10CDF0001AD0234F01250024A30003F180432E42C3
:10CE000003F5C0434FEA45050BD0D3F8100557F89A
:10CE10002420D3F81015C0F30520C1F3014102B15D
:10CE200090470134082CE7D1002EFFF67BAF09B004
:10CE3000BDE8F08F46F00046DBE7B9F1020FF6D10E
:10CE4000032905D0002BF2D009B0BDE8F04F1847F8
:10CE50004FF4403CACE70329E9D115F809A008FAE2
:10CE60000CFB4AEA0B0A05F809A085E700610040BF
:10CE700000600040206100407C61004000030050E1
:10CE80001C4501202DE9F04F0024DFF8A4B085B047
:10CE900006468A46174600F5A078A1464FF480352D
:10CEA000D6F804332B4210D058F82430E0B263B1E6
:10CEB000C6F84853C6F8085348F8249058F8243068
:10CEC00001935BF82A30019A98470134A7424FEA50
:10CED0004505E5D1D6F80433DA0702D5D6F8003196
:10CEE000C3B9D6F804339B0711D5D6F8043173B112
:10CEF0000023C6F80431D6F804210D4B0392039A9F
:10CF000053F82A30052005B0BDE8F04F184705B0AA
:10CF1000BDE8F08F0023C6F80031054BD6F800219C
:10CF2000029253F82A30029A04209847D9E700BFAA
:10CF300098450120024803220021FFF7A3BF00BF4C
:10CF400000B00040024804220121FFF79BBF00BF50
:10CF500000100140024804220221FFF793BF00BFE6
:10CF60000040024010B5074C236882B03BB1064B2D
:10CF70005B6898470023236023680193019B02B0FC
:10CF800010BD00BF00010140844501206CDF7047E7
:10CF90006DDF704770DF704772DF704773DF704777
:10CFA00074DF704775DF704778DF70477ADF70474E
:10CFB0007BDF70477CDF70477DDF70478ADF70471B
:10CFC0008BDF70478CDF70478FDF704790DF7047D3
:10CFD000A5DF704760DF704769DF704767DF704724
:10CFE00010DF704711DF70470388102B06D01B2B12
:10CFF00002D10120887070470020704783880B8021
:10D0000001208870704700BF31291DD8102918D918
:10D010001139202914D8DFE801F01E21131313134E
:10D0200013131313131313131313241113131313C1
:10D03000131313131313131313131B00222303705F
:10D04000704721B9017070474129FBD07047704784
:10D05000312303707047112303707047122303704C
:10D060007047212303707047A3DF7047ABDF704721
:10D07000ADDF7047AEDF70474368014613B1024829
:10D08000FEF742BB704700BF5198030076DF704740
:10D090007EDF70477FDF704786DF70479BDF70471A
:10D0A0009DDF70479EDF7047B5DF7047406828B14D
:10D0B00000884FF6FF73C01A18BF0120704700BFE9
:10D0C000406840B1406830B183791BB1C06810B18D
:10D0D000FFF7ECBF0120704718B143680BB1188807
:10D0E00070474FF6FF707047A4DF704770B5044675
:10D0F000408C94F8263086B080B233B394F8243054
:10D1000094F825208DF8082006330022656854F82D
:10D110002310CDF809208DF80D20AA8A238C0491C4
:10D1200002A9ADF80A20ADF80E30FFF79DFF50B907
:10D1300094F824302084013303F00103012284F8A1
:10D14000243084F8272006B070BD94F8242061684C
:10D15000268C898A94F82550ADF80810063202A969
:10D1600054F8222005920DF10602ADF80C30ADF80E
:10D1700006608DF80A500492FFF77CFFD7E700BFE6
:10D18000A8DF7047AADF704762DF704764DF70472F
:10D19000A1DF7047ACDF70470288362A01D000203B
:10D1A000704738B50C4621B18188A2899142034667
:10D1B00001D0012038BDC288E281C589D4E90002CE
:10D1C000954228BF154603F110012A464AF036FC65
:10D1D0000120A560207438BD0120704710207047E1
:10D1E00030B54368264C1A791B68342505FB02428A
:10D1F0000624C3F800450225C3F888150024012140
:10D20000C3F8444582F82D50C3F8484585B01962EB
:10D21000996002E0D3F824211AB9D3F85021002AEA
:10D22000F8D00022C3F85021D3F8502101920122F6
:10D2300001995A61D3F80421002AFBD00024C3F8D5
:10D240000441D3F8041102910299D3F8241179B161
:10D25000C3F82441D3F8241103910399D3F8C414DB
:10D26000C3F8C4144068FFF77DFA204605B030BD0E
:10D270004068FFF777FA0124204605B030BD00BFB3
:10D280006C440120F0B44468174DA668D4F800C07F
:10D29000B14228BF3146A94223D2144D144F002475
:10D2A00000E0B5680134A94207EBC406F9D3716800
:10D2B000CCF8241552B14268002B136814BF062223
:10D2C0000422C3F854250120F0BC70474268002BAB
:10D2D00013680CBF00220222C3F854250120F0BCC1
:10D2E00070474FF0A051E3E70048E8010024F40044
:10D2F000C4D8070010B443681B791F2B86BF03F006
:10D300001F03104A4FF0A04203F5E07300240129E7
:10D3100042F8234013D0022914BF22460422436856
:10D320001B791F2B86BF03F01F0306494FF0A04156
:10D3300003F5E07341F823205DF8044B70470C229D
:10D34000EDE700BF0003005030B443681B7940F2A2
:10D35000037440F20335012A0CBF22462A461F2BD4
:10D3600088BF03F01F0303F5E0738CBF124C4FF02E
:10D37000A04444F8232043681B7971B91F2B86BF52
:10D380000D4903F01F034FF0A041012202FA03F3FD
:10D39000C1F80C35002030BC70471F2B86BF0649F2
:10D3A00003F01F034FF0A041012202FA03F3C1F87A
:10D3B0000835002030BC70470003005043681B79DB
:10D3C0001F2B86BF03F01F03044A4FF0A04203F552
:10D3D000E07352F8230000F0010070470003005092
:10D3E00043681B7961B91F2B86BF0C4903F01F03EB
:10D3F0004FF0A041012202FA03F3C1F80C35704747
:10D400001F2B86BF054903F01F034FF0A0410122E7
:10D4100002FA03F3C1F80835704700BF000300505B
:10D4200043681B791F2B86BF03F01F03084A4FF088
:10D43000A04203F5E07152F82110C90754BFD2F899
:10D440001005D2F80405D84000F00100704700BF75
:10D450000003005008B510300021FFF7C1FF012084
:10D4600008BD00BF70B5A1F10101049DB1FA81F1C1
:10D470000646490908301C46FFF7B2FFD6E90D21E0
:10D4800065B160190138631EC2F80C1513F8015F0D
:10D49000746883422570C2F80815F5D170BD00BFCD
:10D4A00010300121FFF79CBFFF2816D0430970B44C
:10D4B0000A4E0B4D56F8234055F8231000F01F007C
:10D4C000012202FA00F024EA000421EA000046F8F2
:10D4D000234045F8230070BC70477047244001206A
:10D4E000FC4701204368ABB110B51B791F2B86BFE9
:10D4F00003F01F0308494FF0A04103F5E073022237
:10D5000041F82320436804461879FFF7CDFF002334
:10D51000636010BD704700BF0003005010B50446A3
:10D520004068FEF723FD607AFFF7BEFFA07AFFF7A1
:10D53000BBFFE07ABDE81040FFF7B6BF437AFF2B90
:10D5400001D0FFF7EBBF7047FF280FD010B441099F
:10D55000074A00F01F0052F82140012303FA00F0AF
:10D56000204342F821005DF8044B7047704700BF2C
:10D57000FC47012010B50D4B42689A42044605D085
:10D5800010339A4208BF012301D010BD0023084A7E
:10D59000607A0121D154FFF7D7FFA07AFFF7D4FFBB
:10D5A000E07ABDE81040FFF7CFBF00BF9002012036
:10D5B000F84701200379FF2B0FD010B45809074911
:10D5C00003F01F0351F82040012202FA03F3234322
:10D5D00041F820305DF8044B70477047FC4701204C
:10D5E0000379FF2B16D05A0970B40B4E0B4D56F829
:10D5F000224055F8220003F01F03012101FA03F332
:10D6000024EA030420EA030346F8224045F82230C6
:10D6100070BC7047704700BF24400120FC470120C8
:10D6200010B403790649580903F01F0251F820404D
:10D6300001239340234341F820305DF8044B7047A9
:10D640002440012038B505460C460846FFF7E8FFA0
:10D650006C6023791F2B86BF03F01F03044A4FF031
:10D66000A04203F5E073002042F8230038BD00BF5C
:10D67000000300504FF01023D3F80C3213F0010FC9
:10D68000037903D0A3F10902012A0DD9074A5909E8
:10D6900003F01F0352F82110012202FA03F30B4298
:10D6A0000CBF104600207047002070472440012026
:10D6B0004CDF7047024B800143F00103184700BF65
:10D6C000F0F1070008B1FFF7F5BF704730DF704792
:10D6D00031DF7047B0F5A07F03D1024A13680133F0
:10D6E00013607047284801204268AAB110B40B4962
:10D6F00054680B78127AC4F86025013BDBB2002233
:10D700000B70426013B15DF8044B7047044B5DF839
:10D71000044B1868FEF75EBD704700BF5D480120EE
:10D72000A0480120184B53F8203030B40022174D88
:10D73000C3F800250221C3F80425C3F810154FF4DF
:10D74000FA41C3F8142505EBC004C3F80C25C3F84F
:10D7500008150421C3F82045C3F824154FF40041EF
:10D76000C3F8282525F83010C3F82C256180C3F8AC
:10D770004025A180C3F84425E180C3F84825C3F8BB
:10D780004C2530BC704700BF0C57080038480120BA
:10D790002DE9F04F83B093469DF830209BB18A4627
:10D7A0006449984681460027012547F6FB73B1FB83
:10D7B000F5F4B4FBF8F4261F9E424FEA450506D95E
:10D7C0000137082FF3D1022003B0BDE8F08F5A498A
:10D7D0005A48D1F8003513F0010300F10C060ED0C1
:10D7E0001AB9D1F80855AC427FD0864200F0938038
:10D7F00050F8041BD1F8003513F00103F0D11D4699
:10D8000099F80900C9F8041063F3060089F80900C3
:10D810009AF8043089F8083050460192FFF700FF6B
:10D8200099F8091099F80830019AC9F80C8062F348
:10D83000C7111F2B89F8091069D84FF0A04103F5D3
:10D84000E073032241F82320D9F804300022C3F802
:10D850000025E5B9D9F80430374A934264D002F57F
:10D86000A042934264D002F5805293425ED0344885
:10D87000834214BFFF200320FFF754FFD9F8043080
:10D880000022C3F80C75C3F80425C3F8084599F8BD
:10D890000930D9F804209AF804002A4903F07F03DC
:10D8A00003F5AC73012442F82300D9F80430C3F81F
:10D8B0000045D9F80430A9F80AB0D3F82005D3F808
:10D8C000083599F8092003FB0BFBA1FB0B3B1E4914
:10D8D00002F07F0341EADB3B20F813B0D9F80430B3
:10D8E00000209C6003B0BDE8F08FD1F80C55AF422A
:10D8F0007FF47BAF94460CF5AC7551F8255001359B
:10D900000ED00CF1010CBCF1040FF4D16DE70F49FE
:10D9100003F01F0393E70023C9F80430042053E702
:10D92000DDB20CF07F036BE72846A5E70220A3E7F2
:10D930000120A1E70024F40000C0014010570800B6
:10D9400000D00240018000800080FFFF00030050F3
:10D95000436863B310B5037A1F2B86BF03F01F0320
:10D96000134A4FF0A04203F5E073022142F823105E
:10D97000427A416802F07F02044602F5AC7200234D
:10D980004FF0FF30636041F8220003F5AC720133C1
:10D9900051F82220013204D1042BF6D10023C1F822
:10D9A0000035207AFFF780FDFF23237210BD7047FA
:10D9B00000030050254B53F82030002B45D030B4E5
:10D9C00019795D791F298ABF214A4FF0A04201F0E1
:10D9D0001F01D2F810251F2D22FA01F28ABF1C491F
:10D9E0004FF0A04105F01F05D1F810059979E840E6
:10D9F00002F0010200F00100540042402244511A9A
:10DA000001F00301012916D0032919D093F9071059
:10DA10009A71032906DD9A68002101329A60D97152
:10DA200030BC70470331FBDA9A680021013A9A60F2
:10DA3000D97130BC7047D979013149B2D971E7E762
:10DA4000D979013949B2D971E2E77047FC34012034
:10DA50000003005010B504460079FF281AD00E4B81
:10DA60006179002243F8202043F82120FFF78EF847
:10DA70006079FFF78BF82079FFF7BEF86079FFF740
:10DA8000BBF82079FFF710FD6079FFF70DFD4FF629
:10DA9000FF73A38010BD00BFFC34012008B5FDF763
:10DAA00081FC00BFB0F5A07F00D0704710B5074BD8
:10DAB000074C1B681A680120002350600B72204637
:10DAC000FCF790F9034B5C6610BD00BFA448012031
:10DAD0002C020120B8450120034AC068034B0028EE
:10DAE00014BF104618467047F8190800EC190800D2
:10DAF000024B8068002808BF18467047F4190800D8
:10DB000008B5FFF7B9FA014808BD00BFF4190800CD
:10DB100008B5FFF7CBFA034A034B002814BF1046A1
:10DB2000184608BDF8190800EC19080043683BB115
:10DB300093F85A200348044B022A08BF184670473E
:10DB400000487047EC190800F8190800024B80687B
:10DB5000002808BF18467047F4190800406870474D
:10DB600008B543681BB101460248FDF7CDFD0248E8
:10DB700008BD00BFE53B0300F4190800034AC07963
:10DB8000034B002814BF104618467047F8190800C8
:10DB9000EC190800024B8068002808BF184670473F
:10DBA000F4190800C30782B045D5401007EE900A6B
:10DBB000F8EEE77A9FED407AF4EEC77AF1EE10FACC
:10DBC0000EDD9FED3E7A27EE877ABCEEC77A17EE20
:10DBD000103A1B0207EE103AB8EE477A77EEC77A92
:10DBE0009FED377AF4EEC77AF1EE10FA47D4DFED05
:10DBF000356AF4EEE67AF1EE10FA23D477EEE67A9F
:10DC0000B0EE087A67EE877A9FED2B7A37EE677A67
:10DC1000FCEEE77ACDED007AFCEEC77A9DF8003095
:10DC2000CDED017A9DF8040040EA0340400040F049
:10DC3000010002B0704700F1FF4020F0030307EE3F
:10DC4000903AB7E777EEC77AB0EE087A67EE877A50
:10DC50009FED197A37EE677AFCEEE77ACDED017A1F
:10DC6000FCEEC77A9DF80400CDED007A9DF80030F7
:10DC700040EA0320400040F0010002B07047B0EEDF
:10DC8000087A67EE877A9FED0C7A37EE677AFCEEBA
:10DC9000E77ACDED017AFCEEC77A9DF80400CDED70
:10DCA000007A9DF80030000240EA0340400040F056
:10DCB000010002B0704700BF00007F430000803BBE
:10DCC0000000AA4200002A4308B5FFF70BFC0148F8
:10DCD00008BD00BFF419080008B50868FFF702FC8A
:10DCE000004808BDF419080038B5084B0C681B68DB
:10DCF0000025C3F800552079FFF7D6FB6079257120
:10DD0000FFF7D2FB6571024838BD00BF4802012011
:10DD1000F419080008B5FFF711FC014808BD00BF61
:10DD2000F419080008B50868FFF708FC004808BDAA
:10DD3000F4190800064BD3F8C43093F8250093F883
:10DD400024204000D2B240F0010083F82520704723
:10DD5000B845012070B4184D184E002405E0013478
:10DD60001A2C06EBC4050ED06D68A842F7D1002529
:10DD70000D604FF4D7701149106051F83420D2086B
:10DD80001A6070BC70470E4D0E4E002405E0013441
:10DD9000302C06EBC405F4D06D68A842F7D14FF4DF
:10DDA0003A750D6040F229300649106051F8342070
:10DDB000D20870BC1A607047244F080070E6070054
:10DDC000144F0800AC12080000487047844E080049
:10DDD00008B50868FFF788FC004808BDF41908007A
:10DDE00008B5FFF781FC014808BD00BFF419080021
:10DDF00008B50868FFF7ACFD004808BDF419080035
:10DE000008B5FFF7A5FD014808BD00BFF4190800DB
:10DE10001020704701207047FA2070470B46910789
:10DE200010B402D50269120608D5083007C883E885
:10DE30000700002420465DF8044B7047012420466B
:10DE40005DF8044B704700BF08B50868FFF702FE95
:10DE5000004808BDF419080008B5FFF7FBFD0148AC
:10DE600008BD00BFF4190800024BC3F8C000024807
:10DE7000704700BFB8450120F41908000B46910710
:10DE800010B402D5826A120608D5203007C883E88C
:10DE90000700002420465DF8044B7047012420460B
:10DEA0005DF8044B704700BF024B034800221A7014
:10DEB000704700BF683D0120F4190800062801D012
:10DEC0000020704710B50E4B0C4689680B40062B9E
:10DED00082B010D0486830B123795840400040F0FB
:10DEE000010002B010BD084601A9FCF7AFFA019984
:10DEF000F9F7FAFEF0E7C808F9F70AFFEBE700BF09
:10DF0000070080FF2DE9F04F83B092469DF8302046
:10DF1000019300921BB307468B464FF000091AF895
:10DF2000096009F10109BBF1000F12D000240AEBCE
:10DF3000090807E0AE4202D849F0ECFDA8B12C4434
:10DF40005C4506D23D5D0134324641463819002D0C
:10DF5000F0D1009B63B1019BB1449945DFD3009B95
:10DF600083F0010003B0BDE8F08F009B002BF2D0DE
:10DF7000009803B0BDE8F08F80687047C0687047B4
:10DF8000034A0079034B002814BF10461846704717
:10DF9000F8190800EC190800034A4079034B0028DF
:10DFA00014BF104618467047F8190800EC1908000D
:10DFB000F0B4876882B0042F9DF818409DF81C606B
:10DFC0003DD0456A01FB07F1002D54D00D44477B3D
:10DFD000EA55877BEB55C77BEC558568076A042DAE
:10DFE000394435D007EE902A90ED067A427BF8EE60
:10DFF000E77A67EE877A07EE103AFCEEE77AB8EE3A
:10E00000C77A17EE903A8B54D0ED066A827B27EEE2
:10E01000267A07EE904ABCEEC77AF8EEE77A17EE5A
:10E02000103A8B5490ED067AC27B67EE877AFCEE4D
:10E03000E77A17EE903A8B5402B0F0BC7047877CB9
:10E04000E7B9456A890005B3077C0D44EE55BEE784
:10E05000877C6FB907EE906A90ED067AF8EEE77A62
:10E0600067EE877AFCEEE77ACDED017A9DF80460E1
:10E07000057C4E55B6E7056A2944B3E7456AF608BC
:10E0800046F0E0068900002DDED1056A2944002F04
:10E09000EED1DFE72DE9F04FD1F80031A3F1100206
:10E0A000102A87B000F2D8800123934003F0013397
:10E0B00023F08073002B14BF8C464FF0000C031D1F
:10E0C00005931E460027C3190CEB07041A7814F8B1
:10E0D000015B6A4003F8012B9E42F7D10437102FF1
:10E0E00006F10406EFD10123009300F1140303931A
:10E0F000DFF86CB1DDF814A0CDF810C000F110030A
:10E10000019302910246002312F823101BF801101C
:10E1100002F823100133042BF6D101325245F2D11B
:10E120004378447B43738379417A82784472847B59
:10E130008373C37A4579867A90F80FE041718272D1
:10E14000C178C279C373029BC272457086708471B4
:10E15000C17180F803E093F80431009A934262D0D1
:10E1600003461A7893F803C09F78597882EA050429
:10E17000E50986EA0E064FEA450E7544664005EB52
:10E18000C50582EA0C0985EA440572404FEAD914B4
:10E1900055401D70650087EA0C082C4481EA070E83
:10E1A00086EA0C0C774004EBC4044E404FEAD811C9
:10E1B0004FEADE1284EA49094C002144540022440B
:10E1C00002EBC20201EBC10182EA4E0E81EA480174
:10E1D000019A89EA0C0C4F408EEA060683F803C0C8
:10E1E0009F705E7004339A4204D05D789E7893F8F5
:10E1F00003E0B6E7009BDDE903C71D015446231F7A
:10E2000079191A7811F8016B724003F8012B9C42BE
:10E21000F7D10434A44505F10405F0D1009B013386
:10E22000DBB200936EE7009BDDF810C0059C039EF7
:10E230001901231F0CEB01001A7810F8015B6A40EA
:10E2400003F8012B9C42F7D10434A64201F10401EA
:10E25000EFD107B0BDE8F08F4FF0000C2FE700BF03
:10E26000BC6108002DE9F04FD1F800318BB0A3F16B
:10E270001002102A079000F24C810123934003F012
:10E28000013323F08073002B14BF0B46002301934E
:10E29000079B91F80461019F1C1D143308943601FB
:10E2A00009939C46231FB8191A7810F8015B6A403D
:10E2B00003F8012B9C42F7D10434A44506F104066F
:10E2C000F0D191F80431013BDBB29B000593079B31
:10E2D00010330693079F78787C7B79797A7ABB78BC
:10E2E0007871F878BE7A97F806C07C707972BC7B3A
:10E2F000F97B7A73BB72FA7AFB79F8730898FA7132
:10E30000BE7087F80EC0BC71F972FB703A460023EC
:10E3100012F82310804C615C02F823100133042BA7
:10E32000F6D101329042F2D1059B0898019E099FD7
:10E330009D00031F71191A7811F8014B624003F810
:10E34000012B9842F7D10430874205F10405F0D142
:10E35000059B002B00F0DA80079B9E469EF800107C
:10E360009EF801209EF802009EF80390CF09D30981
:10E370007C00C60927445D0074002B4407EBC707E7
:10E380004FEAD91587EA4107264403EBC303C7F3D5
:10E39000C01483EA42034FEA450C06EBC60686EA40
:10E3A000400665444FEA4408C3F3C01C44444FEAA6
:10E3B0004C0AC6F3C018D4444FEA480AFFB2D0440E
:10E3C00004EBC40484EA4704DBB2F6B20CEBCC0CD9
:10E3D00005EBC50508EBC80885EA4905C4F3C01A72
:10E3E00088EA460804948CEA4304C5F3C01BCDF8C0
:10E3F0000C80029482EA00084A40029C4FEA4B0CCF
:10E40000414089EA08085040DC4487EA080878401F
:10E41000039FEDB24FEA4A0B89EA010182EA090241
:10E420000CEBCC0CC4F3C019C7F3C0179DF8104017
:10E43000DA4459409DF808B072408CEA450C83EAF2
:10E4400008084FEA490371406A4068407E00CCF3F7
:10E45000C01599440AEBCA0A9DF80C305FFA8CFC8F
:10E460003E448AEA440A84EA080862408BEA0101D1
:10E470008BEA000009EBC9096F005FFA8AFA83EAA8
:10E4800008085A408CEA01018CEA000006EBC60637
:10E4900089EA4B093D445FFA89F98AEA08088AEA61
:10E4A000020286EA43068AEA010105EBC5058AEA0B
:10E4B000000AF6B289EA080889EA020289EA01013B
:10E4C00085EA4C0C89EA0A095FFA8CFC86EA08089E
:10E4D0007240714086EA09068CEA08088CEA01015C
:10E4E0008CEA0202069B8EF800808CEA060C8EF8FD
:10E4F00001108EF802208EF803C00EF1040E734551
:10E500007FF42CAF059B043B0593E3E60BB0BDE81D
:10E51000F08F00230193BBE6005B0800182A2DE969
:10E52000F047C0F8002155D0202A7AD0102A72D0A6
:10E5300000239E46A0F804311C463D49DFF8F480D4
:10E540000EEB840229E011F80CA018F8077011F8FE
:10E5500006C04E5D11F809508AEA0709E31A013432
:10E560001EF823700EEB830389EA070982F80090F6
:10E570005F788CEA070C82F801C09F787E40967025
:10E58000DB785D40D57090F804310133B4EB830F34
:10E5900002F104023DD290F80531B4FBF3F703FB1E
:10E5A000174A12F8049C12F803CC12F8026C12F805
:10E5B000015CBAF1000FC6D0D0F80071202FCDD188
:10E5C000BAF1040FCAD111F8099011F80CC08E5D90
:10E5D0004D5DC3E740F20C63A0F804318646024665
:10E5E00000250B7813704B7853708B789370CB7831
:10E5F000D37090F8053101359D4201F1040102F11B
:10E6000004021C46EDD390F804210132B3EB820FD3
:10E6100093D3BDE8F08740F20A43A0F80431864660
:10E62000DDE740F60E03A0F804318646D7E700BFC9
:10E63000BC610800D4BC07002DE9F04100F10408DA
:10E640000E46174600214FF4847204461D4640468C
:10E6500049F03AFA3A46314640467DB1FFF75EFF4F
:10E6600029686A68AB68E868C4F80001C4F8F41067
:10E67000C4F8F820C4F8FC30BDE8F081BDE8F041F2
:10E68000FFF74CBFDAB32DE9F0414C1E84B00646CB
:10E69000A518102100F1F0074FF0000810290FD045
:10E6A0000A46013104AB1A4414F8013F12F8102C49
:10E6B000AC4283EA02032370F0D104B0BDE8F081DC
:10E6C00038687968BA68FB68EC46ACE80F003146F8
:10E6D0006846FFF7DFFC06F580710F2211F8013D57
:10E6E000FF2B06D03244013382F8F03001210022A2
:10E6F000D8E7013A531C81F80080EFD1F6E7704764
:10E700000023436000487047F4190800006970470F
:10E71000007B7047807B7047704700BF70B4039CDC
:10E720008568256071B1857B017B4668B2FBF5F495
:10E7300005FB1422D0B2CA0800FB02621A60002056
:10E7400070BC704742681A60002070BC704700BF00
:10E7500010B401241470427B1A70019B82681A6005
:10E76000029B01B1847B1C705DF8044B704700BFB5
:10E770000B68024800225A60DA607047F4190800FA
:10E78000806A7047807E704790F82400704700BF11
:10E7900030B400241470827EDDE90254082A94BF4C
:10E7A000002201221A704FF400732B6021B190F8FF
:10E7B0002430237030BC70470123237030BC704775
:10E7C0000023C0E901330148704700BFF419080075
:10E7D00040697047C07C7047007C704710B40024CB
:10E7E0001470827C1A70019BC2681A60029B21B16E
:10E7F000C27C1A705DF8044B704701221A705DF8F4
:10E80000044B7047008B07EE900AFBEEE87A17EE98
:10E81000900A20F0030040F00200A0F1FF40704792
:10E82000406B704790F83D00704700BF30B4002542
:10E83000012415701C70029A036B1360039B09B1CD
:10E8400090F83D401C7030BC704700BF10B500F11F
:10E850000C0420460121FEF74DFDFEF7E1FD0122EB
:10E860000346114620461C46FEF76EFD204610BDAD
:10E870008388994219DA002917DBC3889A4214DA8F
:10E88000002A12DB70B48489837B02FB04F2DC086B
:10E890000DD08368012C03EB820219D0022C19D011
:10E8A000042C1AD0002070BC704700207047C47B35
:10E8B0000569866841FA04F422442940048C56F81C
:10E8C000220001FB0333C3F12003D8402040EAE7D4
:10E8D000505CE8E732F81100E5E752F82100E2E782
:10E8E000020C10B4C3B20D4C02EBC201363302EB82
:10E8F0004102C0F30720A4FB0313B621A4FB02C20C
:10E90000DB0901FB00F103EBD210A4FB012300EBB8
:10E91000D310C0B25DF8044B704700BF8180808087
:10E92000C2B210B4040C9442C0F30723214638BF8E
:10E930001146994238BF19469442204628BF1046D6
:10E94000984294BF081AC81A10F0FF0007D0C9B245
:10E950008C4207D08B4226D08A421BD000205DF823
:10E96000044B70479B1A144A03EB8303DB0093FBB1
:10E97000F0F382FB03121A44D817C0EBE210C0EB8D
:10E980000010A3EB00100028B8BFF030C0B25DF853
:10E99000044B7047E31A03EB800303EB8303DB00B4
:10E9A00093FBF0F0EFE7131B03EB400303EB830350
:10E9B000DB0093FBF0F0E6E789888888034A00795A
:10E9C000034B002814BF104618467047F81908007A
:10E9D000EC1908002DE9F04F0479106883B09B46CC
:10E9E000002C47D10C78102C00F0C2804A79002A04
:10E9F00000F0D480050C5FFA80FC964EC0F3072728
:10EA000005EBC5084FF0B60E654505EB48080CF15F
:10EA100036020EFB07FEA6FB0232A6FB0838A6FB59
:10EA20000E3E2E4628BF6646654538BF6546D2096C
:10EA3000BE4228BF3E4602EBD812BD422CBFC6EBF9
:10EA40000505C6EB070502EBDE12C4F10804D2B2DD
:10EA5000EDB242FA04F4102DCBF8004000F2CB8066
:10EA60000A790AB9CBF8002001228BF8042003B000
:10EA7000BDE8F08FB2F80C805689DFF8E8E1764BFC
:10EA8000DFED765A9FED766A0C7808F12105C5EB2B
:10EA90000545354406F12102C8EB0848464485EA9D
:10EAA000553790444EF64D4986EA563A88EA58382A
:10EAB00007FB07F509FB05E50AFB0AF608FB08F268
:10EAC00007FB053509FB06E609FB02E20AFB0636F1
:10EAD00008FB023225F0004306EE903A26F0004390
:10EAE00007EE103A22F0004307EE903AF8EEE66A9D
:10EAF000B8EEC77AF8EEE77A66EEA56A27EE257AD1
:10EB000067EEA57A66EE866A27EE067A67EE867A63
:10EB1000102C4FEA104CC0F30727FCEEE66ABCEE5F
:10EB2000C77AFCEEE77AC0B27BD016EE906A17EE99
:10EB3000105A17EE903AFF2222411640154013401A
:10EB400050FA86F65CFA85F557FA83F0FF2E28BF57
:10EB5000FF26FF2D2A4628BFFF22FF2828BFFF20BF
:10EB6000000240EA0240102C40EA06007FF43EAF6B
:10EB7000C40CC0F3C40242EAC422C0F38520097A5F
:10EB800042EA401080B209B140BA80B20122CBF80B
:10EB900000008BF8042003B0BDE8F08F0A7922B39F
:10EBA000082C22D82B4D010CC2B201EBC106363223
:10EBB00001EB4601A5FB0232C0F30720B626A5FBF8
:10EBC0000131D20906FB00F002EBD112A5FB0030A7
:10EBD00002EBD012D2B2C4F1080442FA04F40122CA
:10EBE000CBF800408BF8042002E000228BF80420D0
:10EBF00003B0BDE8F08F0191FFF792FE01998A788A
:10EC0000101A80B200F10A0292B2142A03D900B29B
:10EC100010F1DB0F15DA0A79C2B90122CBF8002016
:10EC2000E6E716EE903A03F0070617EE103A03F007
:10EC3000070517EE903A03F0030206446544D01925
:10EC400084E7DB28E7DC0A79002AD1D10022CBF85F
:10EC50000020CDE7818080800DDD0852000000306B
:10EC600000007F431F073101436800221A7270477A
:10EC7000C088400040F00100704700BF808840001D
:10EC800040F00100704700BF042808D0052804D1D7
:10EC90008868400040F0010070470020704701483C
:10ECA000704700BFF819080070B490F95030002B7D
:10ECB000836AB8BFB0F912609A7BA8BFB0F9106040
:10ECC000DAB15A8893F90510B0F90C5001FB05210F
:10ECD00009B2A0F8461093F905205C88AB1912FB25
:10ECE00003F323441BB2994270BCD2BFA0F84A3050
:10ECF000A0F84A10A0F8463070471A8893F904101B
:10ED0000B0F90C4001FB042109B2A0F8441093F9BA
:10ED100004201D88A31912FB03F32B441BB2994254
:10ED200070BCD2BFA0F84830A0F84810A0F844301A
:10ED3000704700BF70B490F95030002B836AB8BFA1
:10ED4000B0F910609A7BA8BFB0F91260DAB11A88E6
:10ED500093F90410B0F90E5001FB052109B2A0F897
:10ED6000441093F904201C88AB1912FB03F32344CD
:10ED70001BB2994270BCD2BFA0F84830A0F848102E
:10ED8000A0F8443070475A8893F90510B0F90E4046
:10ED900001FB042109B2A0F8461093F905205D8813
:10EDA000A31912FB03F32B441BB2994270BCD2BFD0
:10EDB000A0F84A30A0F84A10A0F84630704700BFCB
:10EDC000B1F90030B0F900209A42C8BF0380B1F910
:10EDD0000230B0F902209A42C8BF4380B1F9043032
:10EDE000B0F904209A42B8BF8380B1F90630B0F977
:10EDF00006209A42B8BFC380704700BF30B4B0F954
:10EE000000301380B1F90040A342BCBF14802346F8
:10EE1000B0F904409480B1F90450AC42C4BF2C4610
:10EE200095809C4218DDB0F902305380B1F9024060
:10EE3000A342B8BF5480B0F90600D080B1F90610E3
:10EE4000B8BF23468842C4BF0846D1809842D4BF89
:10EE50000020012030BC7047002030BC704700BF4C
:10EE600083880188C28840885B1A101A9BB280B2DE
:10EE700000FB03F0704700BF274B83FB01235A18A8
:10EE8000CB17C3EB22234FF4B47202FB13130022FF
:10EE9000012170B4A0F84430B0F84240066CB0F8DC
:10EEA00040504262028680F8322080F82A1093B1E6
:10EEB000B42B18D0B3F5877F80F8321020D040F201
:10EEC000FF1304874587848480F8301070BC426348
:10EED000C2630385704740F20112C0E90E634363C9
:10EEE00070BC0285704740F201114FF6FF738663D4
:10EEF0008584C484426370BCC26301860385704705
:10EF00004FF6017304874587C58480F8311070BCC3
:10EF10004263C26303857047B7600BB683690068BC
:10EF2000184700BF036A0068184700BF2DE9F04189
:10EF30002DED028B90F89A30012284B0044680F8BF
:10EF40009920B0EE408A1BB9F7EE007A37EEC08AFE
:10EF5000A36E494A93423ED0484A934260D0B4F8E7
:10EF60008C30B3F5807F07D1002084F8990004B07D
:10EF7000BDEC028BBDE8F08104F108052846FFF7DF
:10EF8000CDFF0028F0D094F89760DFED3D7AB4F81B
:10EF90008C308DF80C3068EE277A002E51D0FCEEC4
:10EFA000E77A022217EE903A00928DF80D30666AE9
:10EFB000A06803AB01220021B0472846FFF7B2FF4B
:10EFC000002384F89930012084ED228A04B0BDEC3E
:10EFD000028BBDE8F081DFED2B7AE26E94F87110C0
:10EFE000294D68EE277A01F07F01FCEEE77A17EEF3
:10EFF000903A9BB2A4F87230D2F82005D2F80825D6
:10F0000002FB03F3214AA5FB035342EAD33320F862
:10F010001130E26E01210023916084F89930D2E72B
:10F02000DFED1B7AB4EEE78AF1EE10FACCBF0121D6
:10F03000002104F16800FEF7D3F9002384F8993029
:10F04000C1E7FCEEE77A4FF0010817EE903ACDF8F1
:10F050000080A0688DF80B30424603AB3146676AEA
:10F06000B847CDF800803246A068666A41460DF187
:10F070000B03B047A1E700BFD056080048F40700D3
:10F0800000007F4300FF7F47018000800080FFFF7A
:10F09000A4707D3F2DE9F04F2DED028B91B0044619
:10F0A0001F9894F84A704588B0F800B0B0F804A0F2
:10F0B000C0880690BDF870000A909DF87400049016
:10F0C000072F9DF880000395CDE908239DF878501F
:10F0D00005900E460FD894F850200823B3FBF7F3A1
:10F0E000002A00F0088194F84B2003FB02F3BBFBDD
:10F0F000F3FBBAFBF3FA002D40F00C81049B002BCC
:10F1000040F0C280A36920689847049D8DF838605C
:10F110000127009700220EAB11462068E66908EE31
:10F12000103AB04700223B46B8464FF00209174656
:10F13000B4F84610FF2900F2BC8094F8541010A8CF
:10F14000821818444B1E5344594402F8081C0B9271
:10F150000790CA4600F8083C059B3BB10BF00F0B2B
:10F160006BF04F0B4FF0010A8DF838B0CDF800A0CE
:10F170002068E66918EE103A2A464146B047236AED
:10F1800020689847099BB3F5807F1CD08DF83730F5
:10F190004FF0010BA36920689847CDF800B02068B4
:10F1A000E6690DF137032A460021B047CAF3470349
:10F1B00000932068E66918EE103A59462A46B0478F
:10F1C000236A20689847A36920689847049A089B97
:10F1D0008DF838303AB9012300932068E66918EEBB
:10F1E000103A1146B047B4F84830FF2B00F29B802C
:10F1F00094F8563006995A1E0A4403990B440B9909
:10F2000001F8083C079B03F8082C059B63B1039A9F
:10F21000C2F3031343F0100302F00F024FF0020990
:10F220008DF839308DF83820CDF800902068E769E6
:10F2300018EE103A41462A46B847236A2068984794
:10F240000A9BB3F5807F1AD08DF837300127A36968
:10F250002068984700972A462068E6690DF1370331
:10F260000021B047C9F347030093206818EE103A15
:10F270002A463946E569A847236A2068984711B0AD
:10F28000BDEC028BBDE8F08FA369206898470EA9FA
:10F2900008EE101AB4F846108DF838600122FF29E4
:10F2A000A846174615464FF003094FF002037FF6B4
:10F2B00044AFB4F8541010AE164410AAD3188B44BF
:10F2C000CBF30722079306F8082C079A0B961FFA30
:10F2D0008BFB481E02F808BC10AA0AEB00034A4444
:10F2E000C3F3072102F8081C10AA3A4407F1040AE4
:10F2F00002F8053C30E794F84B2003FB02F3039A35
:10F30000B2FBF3F20392069AB2FBF3F30693002DDD
:10F310003FF4F4AEA36920689847049B8DF83860E9
:10F320000BBB0125F4E610A901EB0900B4F8563037
:10F3300003995A1E0B440699C3F3072C9EB211443D
:10F340000B9B03960A4610A903F808CC3944079B87
:10F35000C2F3072C03F8086C07F1040900F808CC85
:10F3600001F8052C51E701220EA908EE101A1546E6
:10F3700017464FF0030902234FF00008D8E600BFFC
:10F3800070B504463430FFF739FD18B3154694F8CC
:10F390004A20072A1ED894F84B6094F8501008238E
:10F3A000B3FBF2F313FB06F3DBB2A1B1B5F90040F6
:10F3B00094FBF3F203FB12420AB1A21A2A80B5F9B8
:10F3C000042092FBF3F403FB14241CB113441B1B15
:10F3D000AB80084670BDB5F9021091FBF3F203FB58
:10F3E00012120AB18A1A6A80B5F9062092FBF3F16B
:10F3F00003FB11210029EDD013445B1AEB8070BD93
:10F40000F8B5C468068A2644B44214D20F460025D3
:10F4100001E0B0420FD22046F8F704FE0246204633
:10F42000F8F728FEBA42EBB2044605F10105F0D127
:10F430005F33D8B2F8BDFF20F8BD00BF4068704709
:10F44000B0F88600704700BF90F8B330044A90F8D7
:10F45000B400A2FB03235B0803FA00F0704700BF6F
:10F46000ABAAAAAA064A002352F83310884203D056
:10F4700001330C2BF8D1704702EBC300FCF7EEBB55
:10F48000043D012008B5436823B1002343600830E0
:10F49000FEF728F8004808BDF4190800C08D704731
:10F4A000808D704702207047808D0730C010023079
:10F4B000704700BF10B500F10C0304468068984205
:10F4C0000CD0E069FEF78CF8206AFFF7CBFF2046EE
:10F4D0003822BDE81040002148F0F6BAFEF72EF8B9
:10F4E000EFE700BF034B02689A4200D07047FFF776
:10F4F000E1BF00BF18650800154B2DE9F041054636
:10F5000043F001080A27002442F20F76002201216D
:10F510002868FDF719FF4FF42070C04728680021C4
:10F52000FDF7E8FE03E0B4420DD80134A4B2286828
:10F53000FDF776FF0028F6D1013FBFB2002FE5D1DD
:10F540002046BDE8F08142F210742046BDE8F0810B
:10F55000D0F1070010B50C68606818B1FDF7C2FF64
:10F5600000236360004810BDF41908000029B8BFEB
:10F570004942002AB8BF5242B0F9040009B212B29F
:10F580008B18834210DD88420CDB90420ADB02FBC1
:10F5900002F200FB00F001FB01218142CCBF002000
:10F5A0000120704700207047012070478388DB43AB
:10F5B0000B808388DB434B80838801338B80838877
:10F5C0000133CB80704700BF4FF080236FF0802263
:10F5D000C1E90023836893B32DE9F041184F00245B
:10F5E00047F6FF76B8462546B64607E0B1F900E093
:10F5F000B1F90260B1F90480B1F9067043681A5993
:10F6000003EB040C9645DCF80430A4BF02F1FF3C88
:10F61000A1F800C09E42A4BF03F1FF364E80904582
:10F62000DCBF01328A809F42DCBF0133CB8083681C
:10F630000235AB4204F10804D8D8BDE8F081704728
:10F640000080FFFF03468068002844D02DE9F04782
:10F6500000F10108D3F804C0B8F1010F8E46DCE9CF
:10F66000001739D902244FF0000908E0974203DD62
:10F67000002B01DA09F101090234444525D8B4FB15
:10F68000F0F5631CB3FBF0FA00FB1A3A00FB1545DA
:10F690003B465CF82A700E465CF82510AEEB060A75
:10F6A000FD1A05FB0AF59342A1EB0606A2EB030344
:10F6B00006FB1353DADD9742DEDC002B04F1020473
:10F6C000C8BF09F1FF394445D9D9B9F1000018BFC5
:10F6D0000120BDE8F08770470020FAE7002908DB29
:10F6E0008388994205DCC3889A4202DCD043C00F6C
:10F6F00070470020704700BF4FF0FF330B608388D6
:10F700008B80C388CB8070472DE9F041044684B0DC
:10F71000D0E9010301A99847A569AB7B002B4AD02A
:10F72000BDF90420B4F91460BDF9061095F9040080
:10F7300095F90530B4F916C0B5F800E0B5F80280C7
:10F74000324413FB02F387B2614411FB07E14344E7
:10F750001BB209B2ADF80630ADF80410BDF90A00CD
:10F760002A88BDF908E0604410FB072000B2ADF81C
:10F77000080095F905206D88764412FB06F22A44AC
:10F7800012B28142C4BFADF80400ADF80810934234
:10F79000ADF80A20C8BFADF80A304FF0010301A947
:10F7A000237704F12000C8BFADF80620FFF708FB5F
:10F7B00004B0BDE8F081BDF90620B4F91660BDF9CA
:10F7C000041095F9040095F90530B4F914C0B5F8A2
:10F7D00000E0B5F80280324413FB02F387B26144C3
:10F7E00011FB07E143441BB209B2ADF80630ADF896
:10F7F0000410BDF908002A88BDF90AE0B3E700BF8C
:10F80000B0F91400400040F001007047B0F9160054
:10F81000400040F0010070470069704710EE102A68
:10F82000914922F000438B424FEAD27027D9B3F1BD
:10F83000FF4F23D8002840F0AF80DFED8C7AB4EE84
:10F84000E70AF1EE10FA00F3A280DFED896A60EEBC
:10F85000266AF6EE007A77EEA67A9FED867ADFEDDD
:10F86000866AFDEEE77A17EE903AF8EEE77AA7EEB1
:10F87000C70A67EEA67AB0EE407A3BE070477F4950
:10F880008B422AD8B3F14C5FC0F08980B6EE006A93
:10F8900020EE066A9FED7A7ADFED7A5A60EE066A0C
:10F8A000F7EE007AE6EE875AB0EE087AE6EEA57A31
:10F8B000F1EE085AA6EE677AB0EE656AA0EE476AE6
:10F8C00077EEC77A87EE867A27EE267AF0EE667AAA
:10F8D000D0EE077A30EE670A70476B4A934200F227
:10F8E00081809FED647A002875D1DFED637A30EE78
:10F8F000477A012337EE670AF6EE003A60EE234AB4
:10F90000DFED5F5A9FED5F6A60EE246AB7EE004A52
:10F91000A6EEA56AB0EE445AA6EE265AF0EE085AB4
:10F92000B0EE456AE4EEC65AB1EE085AA0EE655A4A
:10F9300037EE407A36EE656A77EE677A86EE057ABC
:10F9400027EE267A002BC1D037EE677A5A1CD7EE05
:10F95000007A77EEE67A54D0012B2CD003F17F02A7
:10F96000382B4FEAC25253D8C3F17F01162B4FEA0E
:10F97000C1515CDC30EE677A07EE901A74EE677A5C
:10F9800077EE277A07EE102A27EE870A7047DFED19
:10F990003F7A20EE270A7047BFEE000A704712F048
:10F9A000FF4F7FF46BAF60EE007A82B0CDED017A4D
:10F9B000019B02B07047BDEE007AB4EEC70AF1EECB
:10F9C00010FA41D570EE233AB8EE000A77EEE37AEA
:10F9D00027EE800A7047DFED2E7A30EE077A4FF07F
:10F9E000FF3387E7DFED227A0028BEEE007AB6EE1D
:10F9F000006A60EE276A0CBFF0EE467AF0EE477AB6
:10FA000029E770EE677ABEEE000AA7EEA30A7047F8
:10FA100070EE677A802B77EE847A1ED007EE102A7C
:10FA200027EE270AF7EE007A30EE670A704707EEF6
:10FA3000101A77EE877A07EE102A70EE677A77EE63
:10FA4000847A27EE870A704770EE677AB0EE007A04
:10FA5000A7EE874AB0EE440A704777EEA77A9FED8B
:10FA60000B0A27EE800ADDE743B895418071B14269
:10FA70003BAAB83F8071313FD1F717371872B13EBA
:10FA80001030CF3A688808BD9115853F0000007F8F
:10FA9000D1F717B782B08DED010A0199A1F50003E6
:10FAA000B3F1FF4F0ED34B005AD0002960DBDFEDDE
:10FAB000367A9DED017A67EE277A6FF0180017EE1F
:10FAC000901A06E0B1F1FF4F46D2B1F17E5F58D0F7
:10FAD00000202E4B2E4ADFED2F2ADFED2F6A9FEDFF
:10FAE0002F3ADFED2F4A9FED2F0ADFED2F3A0B441F
:10FAF000C3F316010A4407EE902AB7EE007A37EEF8
:10FB0000C77AF0EE007A77EE277ADB0DC7EE275A38
:10FB10007F3B0344B6EE006A25EEA54A27EE066A4F
:10FB200024EE045A07EE903AE5EE226AE5EE034A27
:10FB300066EE846AF8EEE77AE4EE856A27EE800ADC
:10FB4000E6EE076AA6EEA50AA6EE470A30EE070A19
:10FB5000A7EEA30A02B070479DED010A02B07047FC
:10FB600060EE007ABFEE007A87EE270A02B0704797
:10FB7000DDED017A37EEE77ADFED0C7A87EE270AC2
:10FB8000E8E79FED0A0AE5E70000004C0DFB4A009C
:10FB9000F304353FEEE9913EAAAA2A3F269E783E1D
:10FBA00013CECC3ED1F717378071313F00000000F3
:10FBB00008B5FFF76FFFDFED027A80EE270A08BD78
:10FBC0008E5D134008B5FFF765FFDFED027A80EE2A
:10FBD000270A08BD1872313F10EE103AC3F3C7521E
:10FBE0007F3A162A2ADC002A10EE101A82B014DBA3
:10FBF000154840FA02F21A420DD0DFED147A70EE89
:10FC0000277A0029CDED007AA8BF8918009B21EA48
:10FC1000020300EE103A02B07047DFED0C7A70EE8E
:10FC2000277A002BCDED017A019A08DB5A00B7EE56
:10FC3000000A08BF00EE103A02B0704770479FED0F
:10FC4000040A02B0704700BFFFFF7F000000807B06
:10FC50000000008010EE103AC3F3C7527F3A162A14
:10FC600026DC002A10EE101A82B014DB154840FA88
:10FC700002F21A420DD0DFED147A70EE277A0029D5
:10FC8000CDED007AB8BF8918009B21EA020300EE8F
:10FC9000103A02B07047DFED0C7A70EE277A002B35
:10FCA000CDED017A019A04DB9FED080A02B070479E
:10FCB00070475A00BFEE000A08BF00EE103A02B0CB
:10FCC000704700BFFFFF7F000000807B0000000046
:10FCD00010EE103A23F00042B2F1FF4F32D282B35D
:10FCE000002B3DDB13F0FF4F70B44FEAE3502CD0F4
:10FCF000C3F3160343F40003C207A0F17F0658BF05
:10FD00005B00002476105B00254619214FF08072BD
:10FD1000A818984202DC1B1A8518144401394FEACE
:10FD200043034FEA5202F3D113B1013424F001042A
:10FD3000641004F17C5404EBC65300EE103A70BC1E
:10FD400070477047A0EE000A704713F400020CD110
:10FD50005B001C02114602F10102F9D5401AC7E707
:10FD600070EE407A87EEA70A70474FF0FF31F5E753
:10FD700010EE103A23F00043B3F1485F04DAFDEED1
:10FD8000C07A17EE903A5BB360EE007A9FED155A99
:10FD9000DFED155A9FED156ADFED156A9FED157AB7
:10FDA000E7EE855A20EE275AA5EEA76AE6EE276A07
:10FDB000A6EEA77A30B9DFED106AE7EE876AA6EE05
:10FDC000850A704727EE457AF6EE006AA0EEA67A1D
:10FDD000DFED0A6AD7EE270AE5EE260A30EE600A62
:10FDE000704700BFD3C92E2F342FD7B21BEF383640
:10FDF000010D50B98988083CABAA2ABEABAA2A3E9D
:10FE000010EE103A23F00043B3F1485F2CDAFDEE18
:10FE1000C07A17EE903A002B60D020EE007ADFED2A
:10FE2000314A9FED315ADFED315A9FED316ADFEDF6
:10FE3000317ADFED316AA7EE245AE7EE055AA7EED4
:10FE4000256AE7EE067AE7EE276A67EE266A60EE35
:10FE5000C00AF6EE007AE7EE260AB7EE000AD7EE01
:10FE6000270A30EE600A704720EE007ADFED1D4A67
:10FE70009FED1D5ADFED1D5A9FED1D6ADFED1D7AC6
:10FE8000DFED1D6A1D4AA7EE245A9342E5EE075A9C
:10FE9000A5EE876AE6EE077AE7EE876A66EE876A7E
:10FEA000D5DD174A934214DC03F17F4307EE903A05
:10FEB000B7EE006A36EE676A60EEC00AF6EE005AE8
:10FEC000E7EE260AD7EE257A77EEE00A36EE600AEC
:10FED0007047B6EE076AF5EE027AEDE7B7EE000A74
:10FEE000704700BF4ED747ADF6740F317CF293B424
:10FEF000010DD037610BB6BAABAA2A3D9999993E4C
:10FF00000000483F10EE103A23F00042B2F1465F85
:10FF100012DAFDEEC07A17EE901A11BB431C1343A0
:10FF200000F0AC80012800F0B280BFEE007AC7EE8E
:10FF3000007AB0EE670A704756498A4211DBDFED5E
:10FF4000567A9FED567A002BBCBFF1EE600AB1EEF7
:10FF5000400A37EEC00A77EE607ADFED510A37EEDD
:10FF6000800A20EE007A9FED4F1ADFED4F2A9FEDB9
:10FF70004F2ADFED4F3A9FED4F3ADFED4F4A9FEDAD
:10FF80004F4ADFED4F5A9FED4F5A9FED4F6ADFED1D
:10FF90004F6ADFED4F1A3F4967EE077A2DED028B6E
:10FFA0009FED4C8AE7EE812A8A42A7EE882AE2EE8C
:10FFB000A73AA2EE273AE3EEA74AA3EE274AE4EED9
:10FFC000A75AA4EE275AA5EEA76AE5EE276AF0EE37
:10FFD000467AE7EE876A20EE076AF0EE667AF0EE80
:10FFE000606AE7EE866AE6EE870AE6EE210A70EEC0
:10FFF000207A21DA01281AD0BFEE007AC7EE276AEC
:020000023000CC
:10000000354B17EE902A1A4006EE102A16EE902A6B
:10001000134007EE903AB7EE007AA6EE277A36EE56
:10002000400A70EEC00AA0EEA77AE7EE267ABDEC91
:10003000028BB0EE670A704707EE100AF8EEC76A47
:1000400067EEA75A37EEA67A9B1785EE876A03F00C
:100050000203C3F10103BDEC028BB0EE007A76EE31
:10006000600A07EE903A30EE600AF8EEE77AE0EECA
:10007000476A67EEA67AB0EE670A7047B0EEC00A2C
:10008000B7EE007AC7EE007AB0EE670A7047F0EE7E
:10009000407A4EE740A12C3FDA0F493F68212233D6
:1000A000000000008453D9377AC0953845F4A3384E
:1000B000B9378139C8261A3A48DEBE3A16696B3B11
:1000C0001F37113CA427B33CD10D5D3D8988083E04
:1000D000ABAAAA3E5FAE9BB700F0FFFF10EE102A5E
:1000E00022F00043B3F17E5F07D30FD070EE407A69
:1000F0009FED307A87EE270A7047B3F17C5F27D2F5
:10010000A3F50003B3F1645F09D270479FED2A7A2B
:10011000DFED2A7AE0EE077AB0EE670A704760EE0C
:10012000007A9FED277A9FED276ADFED276ADFEDE2
:10013000275AA7EE876AB7EE007AE7EE866AA7EE3F
:10014000A57A67EEA67AC7EE876AA0EE260A704700
:10015000F0EEC07AF7EE006A76EEE77AB6EE000AC5
:1001600067EE807ADFED164A9FED165A9FED176A0B
:10017000DFED155A9FED160A9FED0F7AA7EEA45AF0
:10018000002AE7EE866AE7EE855AB0EE666AF1EE7F
:10019000E76A67EEA57AF0EE005A87EE865AE6EE39
:1001A000856AA6EEA50A37EE400AB8BFB1EE400A4E
:1001B000704700BF00000000DA0FC93F0000800355
:1001C0006BD30DBCBA132FBD75AA2A3EAEE534BF62
:1001D0006821A2B310EE102A22F00043B3F17E5F33
:1001E00009D346D1DFED4C7A9FED4C0A002AA8BF17
:1001F000B0EE670A7047B3F17C5F05D2B3F14A5F96
:100200003ED89FED470A7047002A5CDBB7EE007AC4
:1002100037EE400AF6EE007A20EE270ADFED415A6B
:10022000DFED417A9FED416A9FED415AF1EEC06AE0
:10023000E0EE275A16EE903A23F47F6323F00F0383
:1002400007EE903AA0EE256AA0EE057AB0EE405A8D
:10025000A7EEE75A20EE060A76EEA75A80EE076A66
:1002600085EE250AA6EE860A37EE800A30EE000AF1
:10027000704770EE407A9FED287A87EE270A704724
:1002800020EE007A9FED286A9FED265ADFED275A6F
:10029000DFED274ADFED276ADFED217AA7EE065A68
:1002A000B7EE006AE7EE055AA7EE246A27EE257A34
:1002B000C7EE065AB0EE667AA0EE657A30EE470ACF
:1002C00037EEC00A7047F7EE006A30EE260AF6EE07
:1002D000007A20EE270ADFED144A9FED127ADFED57
:1002E000135A9FED135A9FED146ADFED0D7AA0EEBD
:1002F000247AE0EE056AE0EE075AB1EEC07A20EE0D
:10030000250AC0EE265AA7EE256A37EE060A37EE12
:10031000C00A30EE000A704700000000DA0F4940C2
:10032000DA0FC93FBA132FBD6BD30DBC75AA2A3E95
:10033000AEE534BF6821A2336821A2B310EE102AC3
:1003400022F00043B3F1994F4FEAD2710DD3B4EECE
:10035000400AF1EE10FA62D6DFED4B7A9FED4B0AC0
:10036000002908BFB0EE670A7047494883421DD88C
:10037000B3F1665F50D360EE006ADFED464ADFED11
:10038000465A9FED465A9FED466A9FED467A66EEC5
:10039000A67AE7EEA45AA7EE856AA7EEA57A67EEDD
:1003A000867AE6EE877AA7EEC00A70473E4A934205
:1003B000B0EEC00A34D93D4A934254D8F7EE087AD9
:1003C000B7EE006AA0EE276A70EE677A9FED387A82
:1003D0009FED380AC7EE866A66EEA65ADFED2D3A23
:1003E000DFED2D4A9FED2D4A9FED2D5A9FED2D6A91
:1003F00065EEA57AE7EEA34AA7EE845AA7EEA46AB3
:1004000067EE857AE5EE867A97EEA67A77EE667ADB
:1004100030EE670AB9B9704712F0FF4F2CD0704721
:10042000A2F5D002934211D8F0EE007ABFEE006A36
:10043000A0EE276A70EE277A9FED1F7A9FED1F0AC4
:10044000C6EE276AC8E7B1EE400A7047F7EE007AB9
:1004500030EE676A70EE277A9FED197A9FED190AE0
:10046000C6EE276AB8E7FFEE007AC7EE806A9FED16
:10047000167A9FED050AAFE760EE007A82B0CDED07
:10048000017A019B02B07047DA0FC93FDA0FC9BF8A
:10049000FFFFDF3E25AC7C3D0DF5113E4712DABD76
:1004A00098CA4CBEA9AAAA3EFFFF973FFFFF1B4078
:1004B000B40F14335E987B3F6937AC313863ED3E3F
:1004C00068212233DA0F493F6821A23370B510EE5C
:1004D000106A26F000450123B5F1FF4F2DED028B88
:1004E000B0EE402A036024DAC5B1B5F1E45F0446FA
:1004F0000FDA002EBEBF4FF0FF33B1EE400A0360AB
:10050000FFF7C8FAB1EE402ABDEC028BB0EE420A0A
:1005100070BD002E14DAB5F1964F69DBDFEDD87AA5
:10052000B7EE007A87EE272ABDEC028BB0EE420AC6
:1005300070BDBDEC028B20EE002AB0EE420A70BD09
:10054000B5F17E5F51D0B5F1804F4ED0DFEDCC1AC2
:10055000730073D4CB4B9D4240F33282CA4B9D4211
:1005600040F3D881B0EE007A37EE427A9FEDC40AAC
:10057000DFEDC60ADFEDC62A9FEDC61A9FEDC63A2B
:10058000DFEDC63A9FEDC64ADFEDC64A9FEDC65A7B
:10059000DFEDC65A9FEDC66A9FEDC62ADFEDC66A3B
:1005A00067EE077AE7EEA02AA7EE813AE2EEA73AD5
:1005B000A3EE274AE3EEA74AA4EE275AE4EEA75A91
:1005C000A5EE276AA5EEA72AE6EE276A22EE072AFD
:1005D000B6EE006AA6EEA72AA7EE462A32EE002A59
:1005E000002E91DA31EEC22A8EE79FEDA52A8BE725
:1005F000B5F17A5FC0F2F281B1EE407AB0EE470A0F
:10060000FFF728FBB4EE407AF1EE10FA40F0F180EB
:10061000DFEDAA7A77EEC27A17EE903A03F0010383
:1006200007EE903AF8EEE77A9B00062B00F2338251
:10063000DFE803F06194945D5DA3A300B5F1824F00
:1006400080F2EA80BDEEC27A9FED9D0ADFED9D8AC1
:10065000DFED9D0A9FED9D1A9FED9D8A9FED9D3ACE
:10066000DFED9D2A9FED9D4ADFED9D3A9FED9D5A5E
:10067000DFED9D4ADFED9D6ADFED9D5AF8EEC77A0A
:1006800017EE103A72EE677AB0EE407AA7EEA87ACB
:10069000033BB0EE602AA7EE271AA7EE882AA1EE48
:1006A000273AE2EE272AA3EE274AE2EEA73AA4EE83
:1006B000275AE3EEA74AE5EE276AE4EEA75AB7EE1B
:1006C000006AB0EE667AF0EE466AE5EEA76A27EEBB
:1006D000277AB6EE006A87EE262AA7EE862A042B32
:1006E0003FF67EAFDFE803F06B587D6E8000B7EE1B
:1006F000007A77EE677A9FED7F0ADFED610A27EED9
:10070000800A0020FFF734FBF1EE401AF5EE401AA4
:10071000F1EE10FA3FF402AF62EE217A9FED750A16
:10072000F0EEE77A80EE270AFFF7B4F9F5EEC01A8B
:10073000F1EE10FA4CBF4FF0FF330123B5F17E5FAD
:100740002360F0EE401A00F05E81B5F1804FB1EE0B
:10075000422A7FF4FDAE9FED4A2A43E7B6EE007AC7
:1007600077EE677A9FED630ADFED450A27EE800A90
:10077000FFF746FBF1EE401AC8E7B7EE087A77EECE
:10078000C77A9FED5C0ADFED3E0A27EE800AFFF78D
:1007900037FBF0EE401AB9E7B7EE007AB0EE080A80
:1007A00037EE800A20EE070AB0EE007A77EE877AFD
:1007B00027EE800AFFF76EF932EE002A10E7B7EE57
:1007C000000AF1E7B7EE000AB1EE047A37EE877A55
:1007D00027EE000AB1EE007A37EE877A27EE007A2C
:1007E000DCE7B7EE000AF5E7B1EE080A37EE800A5B
:1007F000EAE7F6EE007A27EE277AB0EE470AFFF72F
:1008000029FA37EE400A70EE007AB0EE677ABEEE53
:10081000CF7A17EE103A08E7B5F1B94FB0EE420AB9
:1008200080F2E880FFF736F9B7EE003A83EE026A0D
:10083000DFED312ADFED313A9FED314ADFED314A0C
:100840009FED315ADFED315A9FED317A66EE067A2F
:10085000F6EE006AE7EEA23A72EE666AA3EEA74AE7
:1008600030EE430AE4EE274AA4EEA75AE5EE275AF3
:10087000A5EE867AB0EE472AA6EE802AB0E600BF43
:10088000000000006666663F17A6DD3FA283D337EF
:1008900067976739752C3C384584E238A1549C3AF7
:1008A00034B6053A7E02F23BC66E3D3B01F0893D0F
:1008B0001599A83C3F239E3D661AA53E0000004BBB
:1008C000B435F13A67FF0538D6EE4B3AE440DA3CEE
:1008D000BDD7F536E6DC153E54BF983C7ACCA63E33
:1008E0006E0F303E5A245C3EC5D0383F3F239EBD3C
:1008F0003B2DB23FDB0F4940E8C4D5BAD23D5B3A4D
:100900005C061CBAFD0C503A610B36BBABAAAA3D83
:100910001D7FD63E624B9D4278DD9FED627A9FED52
:10092000620A32EE477A27EE071A9FED608ADFED02
:10093000602ADFED600A9FED605ADFED605A9FED9F
:10094000606A9FED603ADFED603ADFED606ADFEDEF
:10095000604A9FED602A9FED604A61EE077AE7EEFC
:10096000882AA7EEA05AE2EEA75AA5EE276AA5EEBE
:10097000A73AE6EE273AE3EE276AE3EEA74AA7EEA8
:10098000824A9FED565ADFED565A9FED562A9FED4B
:10099000566ADFED562AE4EE876AA4EE275AB0EED7
:1009A000667AF0EE656AE5EE276AA7EE672AA6EE9C
:1009B000A76A91EE062A32EE622A32EE002A0FE68C
:1009C000B0EE420AFFF766F8494B9D42B1EE400A8D
:1009D00059DDB7EE007A37EE427AC9E59FED450A58
:1009E000DFED310A22EE000A0020FFF7C1F9F0EE38
:1009F000401A8BE6FFF74EF8F7EE007A30EE670A02
:100A000020EE022AECE5B0EE402A7DE5F7EE007A12
:100A100032EE672A9FED240ADFED372ADFED373A01
:100A20009FED373A9FED374ADFED374A9FED375A52
:100A3000DFED375A9FED376ADFED376A9FED377A82
:100A4000DFED377AE2EE223AA2EE034AE3EE824A83
:100A5000A4EE025AE4EE825AA5EE026AE5EE826A3C
:100A6000A6EE027AE6EE827AF7EE006AE7EE026A16
:100A700067EE827ABEEE006A87EEA67AA2EE067A6A
:100A800037EE002AACE5274B9D42C5DD9FED267A67
:100A900032EE477A47E7B0EE007A77EEC77A2AE679
:100AA0001FA69D3FC316BB3F0000000027F9A3B956
:100AB00067F8663AF7E9AF3985300DBAFE7771BB52
:100AC0009916143B3D37933CFEFC28BC3C2117BED5
:100AD000155A843D6B7BA53976F4B7BA07E7C73B57
:100AE000474D06BD521CE6315EB9F73ECDCDF83D0F
:100AF0001F4A3B3FDB0F49405E3C5B3C78756A3EDA
:100B0000DBD5523BAF72D53DB24B7A3FDFEF443F6E
:100B1000E73ABA3F2D390840F400223FBE2E1D406F
:100B20003F239EBD07336D3E0C5BEC3E00B583B0AA
:100B300001A8FFF7CBFC03B05DF804FB42290AD003
:100B400062291CD048290CD0682911D000EB820002
:100B500090ED000A7047835C00EE103AB8EE400A50
:100B6000704730F8123000EE103AB8EE400A704785
:100B700030F9123000EE103AB8EEC00A70478356D2
:100B800000EE103AB8EEC00A704700BF83070FD1DD
:100B90000068094B98420DD0084B98420AD0084B88
:100BA000984207D0074BC01AB0FA80F0400970474E
:100BB0000020704701207047E47408006C49080069
:100BC000704508005047080010B4054A054C88607D
:100BD0000023C1E9004208465DF8044BCB60704732
:100BE0000DD40500D846080008B50069F9F71CF8CF
:100BF00080F00100C0B208BDF0B4D0E9013401F0CA
:100C00001F01C1F11F0203FA01F5D340621A002A45
:100C100045604FEA5303826002DB1846F0BC704720
:100C2000C668032EA1EB04011FDC00244460002EE3
:100C30003FD0056805EB060C0135056015F8017C11
:100C40003C43240265454460F6D1C6F10305ED003E
:100C5000AC4002F1200524FA05F504FA01F12B431A
:100C6000002402EBC602C4601EE005682F466C1C1F
:100C7000046017F8024B0760240644606F7844EA6A
:100C80000744EF1CC0E90074AF7844EA07242F1D25
:100C9000C0E90074ED7820322C43043E24FA02F5BA
:100CA000C66004FA01F12B43C0E901121846F0BCFA
:100CB00070473146D4E700BF002800F0D5800368B4
:100CC000002B00F0D1800A78FF2A40F0CD804A78CE
:100CD000F0B402F0E004E02C40F0C380D60812F03B
:100CE000180F1ABFF64306F0010602261E704A7856
:100CF000C2F34102C2F104025A604C78E44304F0AA
:100D000001049C608F783F09DF608C78C4F3810414
:100D10001C618D78C5F340055D618D7805F0010596
:100D20009D61CD78AD091D7791F803C0CCF3011C0E
:100D3000C3F820C091F803C0CCF3C00CC3F824C0A2
:100D400091F803C0CCF3800CC3F828C091F803C01D
:100D5000032C0CF0030CC3F82CC000F08280042A92
:100D60007FD00F2F7DD0DE2707FB06F7404A4A26AB
:100D700016FB04741444012D5C6305D00022032D7E
:100D80001A6201D1012200E00222C0F8BC271A78C1
:100D90001D69384C384E02EB42022A4454F8222096
:100DA000C0F8C0271A78002A0CBF02250125C0F818
:100DB000C4571A785C6802EB4202013C224436F9BF
:100DC000122092FBF5F2C0F8C8275A68C0F8D02765
:100DD0001C7880F8D447DD68002D35D05A68274E3E
:100DE00004EB4404013AC4EB0414C2EB02122244A3
:100DF0002A44234D36F91220C2EB421402EB84023E
:100E0000D200C0F8B8271F781A691C7F07EB470685
:100E1000C6EB0616C2EB02123244033CDE6818BF72
:100E20000124324404EB4704164E35F9122036F9FA
:100E300014409D68141B221F05B1A21F5C69002C81
:100E400018BF0132C0F8CC279A681AB91A63042077
:100E5000F0BC70478A8852BA92B21A630620F0BC7E
:100E600070474FF0FF30F3E74FF0FF30704700BF9F
:100E700058D3080020D3080044D30800ACA80800C9
:100E800000D60800F4D508002DE9F04F8BB0CDE96D
:100E90000412149C0893052C00F33C83C4F1060B48
:100EA000031F00F17C0153F8042F42FA0BF2994220
:100EB0001A60F8D10168C36FC74ACC1AD0E90F563F
:100EC0000B4482FB0414A91BAA196400C34D85FBC3
:100ED000016103EB020E49019B1AC0F800E0C04E0D
:100EE00086FB03235B006518621AC0E90F3586FB99
:100EF00002324768836F856B466CBA4C5100C167FC
:100F0000FA1A3B4484FB0212AC1BA9195200B64DDD
:100F100085FB04645D18069545605B1AE400B34DDB
:100F200085FB031311195B00121B8363416485FB6E
:100F300002328368476F456B866CAD4C5200826706
:100F4000D91BDA1984FB0131AC1BAB194900A94D3F
:100F500085FB046405F1D765D61805F58F45D31ACE
:100F6000E40007968660343585FB03235A000E198A
:100F70000B1B4263866485FB0323C768016F056B07
:100F8000C46C9D4E5B007A1A4367394486FB02327B
:100F90009A4E2B1B52002C4486FB03530F199B00C7
:100FA000091B0097C760964C84FB0151D518490076
:100FB000D31A0163C56484FB03230769C16EC56A44
:100FC000046D904E5B007A1A0367394486FB023247
:100FD0002B1B52002C448C4D85FB036301EB040852
:100FE0009B00091BC0F81080884C84FB0151D51868
:100FF0004900D31AC162056584FB03234769816EEA
:10100000856A446D824E5B007A1AC366394486FB5A
:1010100002322B1B52002C447E4D85FB036301EBF7
:10102000040C5B00091BC0F814C07B4C84FB01510D
:10103000D5188900D31A8162456584FB032386692C
:10104000426E476A846D754D9B00B11A83661644E3
:1010500085FB0131724A3B1B49003C4482FB035330
:1010600006EB04095B00341BC0F818906D4D85FB3E
:101070000424A400CE18CA1A4462866585FB023295
:10108000C569036E076AC66D674C9200E91A42662D
:101090002B4484FB0121654ABC1B4900BD1982FB1E
:1010A00004645A1964005B1BC261614D85FB0363D4
:1010B0000E191B01091B0362C66585FB01315D4CDE
:1010C0000194A4F13754A4F53214A4F5E87425462C
:1010D000594B5A4C5A4F5B4ECDF824B009019346F8
:1010E000DFF86CA101667246AE46009D029603973A
:1010F000264600F120011C46DDE906370690A2EBEA
:101100000B005A4484FB00B0A5EB080440004544A2
:1011100086FB0484561BE40015448EFB0626021948
:10112000A0EB040B760000928EFB0B2BA3EB0902C5
:1011300002984FEA4B0B4B4480FB0242A7EB0C0496
:1011400001985200674480FB04C4A3EB070803988E
:1011500064003B4480FB0878A2EB040E4FEA880849
:10116000144480FB0E2E384FA5EB030C4FEA8E0E75
:10117000384687FB0C2CA6EB080780FB07271D448D
:101180004644009B06EB47064FEA4C027F0041E9CC
:10119000066741E908521B1B80FB0323ABEB0E05DE
:1011A0005B00F34480FB05250BEB450B03EB0B06C3
:1011B000009A03EB450341E90336244B14440AF13A
:1011C000180A5C446D00534541F8104C41F8045C2A
:1011D00001F1200158D03DE051C21340FB2285515E
:1011E00072464F40BD45B340CF200B6D103CE142ED
:1011F0006D2DFA419057D9412134F943968DFC5E0B
:10120000630ECB52C41BCC46971AD84A2E40E264D8
:10121000F09C9D4AB31D7D7CA924E2431137AE4F5B
:1012200026CF6F6BC1923C6EA71E6056EBF64C5FEB
:10123000044E9E51BF6B327346FB404142670352DE
:1012400045BA9E5388DEF84C9A79825A60F10700BD
:1012500000F10700DAE91AE30293DAF8703001933B
:10126000DAF874300393DAE9184651E9055851F871
:10127000202C51F804BC51F81C3C51F8089C51F842
:10128000187C51F80CCC3AE7DDE905300899DDF817
:1012900024B05B1A03F0070303F580639A0000296A
:1012A00000F02C81049E05990468B51889002C6211
:1012B00046F8234001F588510027049E44687318BE
:1012C000A2F57C621C627450466F416E446C3144DE
:1012D0000C44C3F82041C3F80041466B446A3444CF
:1012E000C3F82042C3F80042446D2144C3F82013E0
:1012F000C3F800134469416FC66EC3F82044C3F8B5
:101300000044446D0E443444C3F82045C3F80045FE
:10131000C46A416B2144C3F82016C3F80016C16C9F
:101320003144C3F82017C3F80017C16EC66FC468F4
:10133000C3F82048C3F80048C46C0E443444C3F8D2
:101340002049C3F80049C46BC16A2144C3F8201A7C
:10135000C3F8001AC16D3144C3F8201BC3F8001B49
:10136000C169C46FC3F8201CC3F8001CC16D2144BF
:10137000C3F8201DC3F8001D04991744C26BC3F8BD
:10138000202EC3F8204FC3F8004FC3F8002ECC190D
:1013900042682262CA51466E826F416C32441144E7
:1013A000C4F82011C4F80011466A816B3144C4F8B6
:1013B0002012C4F80012816D0A44C4F82023C4F836
:1013C00000238269C4F82024C4F80024866F826E4A
:1013D000816D32441144C4F82015C4F80015866BA1
:1013E000816A3144C4F82016C4F80016816C0A449E
:1013F000C4F82027C4F800278268C4F82028C4F85D
:101400000028866E026F816C32441144C4F82019A2
:10141000C4F80019866A016B3144C4F8201AC4F874
:10142000001A016D0A44C4F8202BC4F8002B02698D
:10143000C4F8202CC4F8002C066F026E016D3244F3
:101440001144C4F8201DC4F8001D016A066B314424
:10145000C4F8201EC4F8001E016C0A44C4F8202FF2
:10146000C4F8002FBBF1000F45D02A68CBF11F0054
:101470004FF0004642FA00F126FA0BF6B1EBE27F9C
:101480004FEAE27706F1FF3618BF86EA070202FA52
:101490000BF203F120012A622A6003F5815351F80F
:1014A000202C42FA00F5B5EBE27F4FEAE27718BF55
:1014B00086EA070202FA0BF20A6041F8202C01F5D5
:1014C00080718B42EBD104F1200204F5815452F873
:1014D000203C43FA00F1B1EBE37F4FEAE37518BF1C
:1014E00086EA050303FA0BF3136042F8203C02F589
:1014F00080729442EBD10BB0BDE8F08F049E059949
:10150000046802F58853F51889002C624FF4885757
:10151000F450D2E64FF0000BCCE400BF2DE9F04FC1
:10152000684D694E4FEAA30803F0030489B005EB48
:10153000841E454656F8243000931C2DDEE90243F4
:10154000A8BF1C25DEF80470CDF804E0033525EAB9
:10155000E575B8F11F0FC34644FA05F6A8BF4FF072
:101560001F0B2F412B410024DE46CDE9066300EB23
:10157000820205970494C3460EE008AD05EB86068B
:1015800056F8105C002B44EA0504B8BF6D42904247
:1015900041F8045B00F0928050F8043B23F00045D2
:1015A00025F0030523F00046002DE6D023F000458A
:1015B00025F00F055DB9019DBBF1000F55F82650D0
:1015C000BABFCEF10006B54045FA0EF5DAE723F0D2
:1015D000004525F03F0575B93C4D103E55F8266095
:1015E000009D86FB05752F46AEF10305002D5ADBE5
:1015F00047FA05F5C6E77504B5F1006FBABF750582
:101600004FF0040C4FF0000CB5F1005FBCBFAD0013
:101610000CF1020C2E4E2F4FDFF8E080B5F1804F19
:10162000BCBF6D000CF1010CB5422B4ED8BF3E463D
:1016300002962A4E2A4FC8BFB14606F1F95606F562
:10164000CE2606F29B16C8BFB246264EDCBF4646E3
:10165000B9460396244F254ED8BFBA46244FD8BF6B
:1016600037462E4687FB0686039F3E442F4686FB61
:101670000787BA442E468AFB0676B14489FB056586
:101680001C4E029F56F82C602F4487FB0656009D87
:10169000F60086FB0575184E56F82C602F46AEEB0B
:1016A0000605002DA4DA6E426FF0004545FA06FCEF
:1016B000BC45FFF667AF07FA06F563E7204609B0B9
:1016C000BDE8F08F04530800F451080044520800AC
:1016D0009979825A591858FFB477F5FEF0CEC2278F
:1016E0008D496C23A4F633D31BAA5759A9BDA02951
:1016F00063218510245208000452080028482EB0A7
:10170000022A2DE9F0411ED03C4B02EBC20603EB4E
:10171000061606F1480C01F144078C3600F1240E40
:1017200050F8043B56F804495CF8045B1A4685FB04
:10173000028241F8042B84FB0323864547F80439D1
:10174000EED1BDE8F08182682D4B83FB02422D4D26
:10175000846985FB046422440A604268DFF8B4C0EF
:101760008CFB0242284EC46986FB047422444A6002
:10177000026883FB0242046A85FB046422448A6097
:101780000268224E86FB0242214C056A84FB0575E5
:101790002A44CA6042684FF0604585FB0272C769FF
:1017A00085FB07E73A440A61826884FB0272876915
:1017B00086FB07E73A444A61426983FB02728A6109
:1017C00002698CFB0272CA61C26883FB02720A6200
:1017D000C36886FB03234B62036985FB03238B628B
:1017E000426984FB02320023C1E91033C1E90E33A0
:1017F000C1E90C33CA62BDE8F08100BF60CC0800CB
:10180000D8E3CEB8281C3107CD3C410D9A615FC9A1
:10181000669EA0F633C3BEB22DE9F04F044683B0F6
:10182000BBBB12F0010031D0D4F88027D4F880631C
:10183000D4F88072D4F88054D4F880050192D4F89A
:101840008021D4F880167642C2F1000CC7F1000E58
:10185000019AC4F880636F42D4F88068C4F880C1EC
:1018600045421846D4F88030C4F880E249425242DA
:1018700076425B42C4F88074C4F88055C4F8801680
:10188000C4F88027C4F88068C4F8803003B0BDE88D
:10189000F08F4FF0004C12F001002CFA03FC4AD0FC
:1018A00000200CF1FF3C8646C3F11F0704F18006BF
:1018B00004F5106856F8805C45FA07F94FEAE57AB6
:1018C000B9EBE57F18BF8AEA0C059D40724646F8E1
:1018D000805C85EAE572A2EBE572D4F880506D4237
:1018E00045FA07FA4FEAE57BBAEBE57F18BF8CEAC9
:1018F0000B059D40F146C4F8805085EAE579A9EBD7
:10190000E5790D6842EA090245FA07F9B9EBE57F86
:1019100040EA02004FEAE57218BF8CEA020504F5BE
:1019200080749D40A04541F8045B06F58076C1D1E6
:1019300003B0BDE8F08F0CF1FF3CC3F11F0704F1C9
:10194000800604F51068864656F8805C45FA07F96B
:101950004FEAE57AB9EBE57F18BF8AEA0C059D40AE
:10196000724646F8805C85EAE572A2EBE572D4F82F
:10197000805045FA07FA4FEAE57BBAEBE57F18BFDE
:101980008CEA0B059D40F146C4F8805085EAE57964
:10199000A9EBE5790D6842EA090245FA07F9B9EBC6
:1019A000E57F40EA02004FEAE57218BF8CEA0205C3
:1019B00004F580749D40A04541F8045B06F58076EF
:1019C000C2D103B0BDE8F08F70B4D0F8C827D0F80A
:1019D000C447D0F8BC3702FB04F203FB02F3002B30
:1019E00011DD00240239264621F8026FD0F8C457D1
:1019F000D0F8C827D0F8BC3702FB05F2013403FB4E
:101A000002F39C42F0DB70BC704700BF30B490F82A
:101A10006B20002AFBD102F0FF030268012454600E
:101A20001464816B056CD2F840250D6090F860203D
:101A3000B2B1224D0269D25C1F2A86BF02F01F029A
:101A400029464FF0A04104FA02F2C1F80C2590F8A3
:101A500060200133DBB202EB4202B3EB420FE9DB61
:101A6000B0F85C301BB3154D0022012190F85F30B7
:101A70001F2B86BF03F01F032C464FF0A04401FA32
:101A800003F3C4F8083500BF00BF90F85F301F2B88
:101A900086BF03F01F032C464FF0A04401FA03F366
:101AA000C4F80C35B0F85C3001329A42DED3826A59
:101AB000036B1360C26A136030BC704700030050B0
:101AC00090F8641090F863304A1E013BDBB2D2B24A
:101AD00080F86830012980F8692088BF90F8693063
:101AE00090F8612088BF03F1FF33F0B488BFDBB208
:101AF0004FF0000498BF012380F86A3080F86B40F3
:101B00008465002A3CD001213C4F23460E4640F21A
:101B1000033512E01F2B86BF03F01F033A464FF038
:101B2000A04206FA03F3C2F8083590F861200134A8
:101B3000E3B249009A42C9B222D9826C02EB031285
:101B40001B01127B1F2A86BF02F01F02BC464FF00A
:101B5000A04C02F5E0724CF8225090F86A200A423C
:101B6000826C13441B7BD5D11F2B86BF03F01F0350
:101B70003A464FF0A04206FA03F3C2F80C35D4E718
:101B800003681F4A934208BF4FF480751DD01D4A59
:101B9000934218D002F58052934228D002F5803249
:101BA000934227D002F58052934208BF4FF0006560
:101BB0000BD001224FF47A715A60DA60C3F84015F5
:101BC0001A60F0BC70474FF40075012100220E4CE2
:101BD0005960C3F80425D9604FF48031C3F8082553
:101BE000C3F81025C3F8041325600368E1E74FF438
:101BF0008065EAE74FF08065E7E700BF000300502B
:101C0000008000400090004000E100E090F8653066
:101C100033B1012380F86B3090F86B30002BFBD18F
:101C2000704700BF2DE9F04F8DB003460446069083
:101C300090F8640093F86530049202FB00F2656945
:101C4000666A52003BB1234694F86740DB6CC4F1EE
:101C5000010403FB0466049F069BFC1DE41093F83B
:101C60006330C7EBC40756FA87F6E400062B0196EB
:101C7000059400F08280C3F10504E4B24FF4006CD7
:101C80000CFA04F640274FF0010E099607FA04F605
:101C90000EFA04F40A960B94002868D0023A049CC9
:101CA0008A1803928A1E04F1FF38029262001FFA1A
:101CB00088F80892002201EB48080792002B47D0D1
:101CC000DDE90A674FF0000A0998D346049A4AB33F
:101CD000019BDDE9024C03F1FF3E34F8022F3CF892
:101CE000021F12EA000318BF2B7832421CBF95F87E
:101CF000019043EA09033A421CBFAA781343014208
:101D00001CBFEA78134331421CBF2A79134339427E
:101D10001CBF6A79134344450EF8013FDDD1069B91
:101D200093F863307600BBF1000F23D1052B21D946
:101D300001274FF40060019A05990AF1010A5FFA40
:101D40008AFB0A445B450192C0D8069A92F8640067
:101D5000029C079A089901322646039C0792D2B248
:101D60000E440C449042884402960394A6D80DB0C9
:101D7000BDE8F08F40007F00DDE720241026CDE98C
:101D80000A464FF40044099486E700BF2DE9F04F5E
:101D900090F85E308FB0012B009200F0B581022BDD
:101DA00083468A4600F0E18090F8642090F8651040
:101DB0004669456A009800FB02F20AEB42080029D6
:101DC00040F0C380DBF84C2000999BF86330CC1DB9
:101DD000E410C1EBC407062BFFB24FEAC40900F0C0
:101DE000A681C3F10503DBB24FF4006C4020012152
:101DF0000CFA03F4984001FA03F30794089009934E
:101E00000021284645F060FE009C9BF863309BF85B
:101E100064209BF86010204605EB870500FB03F06B
:101E2000019502FB00F5002900F08C80601E80B255
:101E3000274640004FEA89040D90780006F1180902
:101E40000A940B906C000020D6460C94CA4604906D
:101E5000CDF808B0C146002A69D000273D46002BC6
:101E60005BD00D9A06957244DDE908C10026059203
:101E7000079AB04637460098002837D0019BA9F151
:101E80000205AEF10204181F0395039B34F802BF4C
:101E900033F8026F03931BEA020318BF5AF8183C89
:101EA0001BEA0C0F1CBF5AF8145C2B431BEA010FF2
:101EB0001CBF5AF8105C2B4316421CBF5AF80C5C2E
:101EC0002B4316EA0C0F1CBF5AF8085C2B430E423A
:101ED0001CBF5AF8046C334350F8046F334303605B
:101EE000059B9C42D1D1029B93F863304FEA4C0C86
:101EF000B8F1000F36D1052B34D901214FF400621F
:101F000001980A9C01375FFA87F820444345019005
:101F1000B1D8029A069D92F864200B980135E9B277
:101F20008A42864481449AD8029991F860100498B4
:101F30000C9C01300490C0B28142A644A1440AF135
:101F4000180A88D80FB0BDE8F08F9BF86710DBF84F
:101F50004C20B2FBF3F3C1F1010101FB03F305EBEC
:101F6000830531E752004900CAE790F864300099D0
:101F700090F865204669476A01FB03F30AEB4308C2
:101F8000002A40F0C680C26C00999BF86330CC1DDB
:101F9000E410C1EBC405062BEDB24FEAC40900F012
:101FA000CE80C3F10503DBB24FF4006C4020012169
:101FB0000CFA03F4984001FA03F30794089009938C
:101FC0000021384645F080FD009C9BF863309BF86B
:101FD00064209BF86010204607EB450500FB03F0EA
:101FE000019502FB00F50029ACD0601E80B22746A7
:101FF00040004FEA49040D9078000A940B906C0061
:102000000020CDE902B00C94C34606F10C09D0467D
:102010004FF0000A002A69D0002B5BD00D9ACDF852
:1020200014A04244DDE908014FF0000E0492079A23
:102030007546009C002C36D0019B0695A8F102073E
:10204000ABF1020A9E1E37F8024F3AF802CF14EAAB
:10205000020318BF39F80C3C04421CBF39F80A5C73
:102060002B430C421CBF39F8084C23431CEA020FD7
:102070001CBF39F8064C23431CEA000F1CBF39F87B
:10208000044C23431CEA010F1CBF39F8024C2343C4
:1020900036F8024F23433380049BBB42D3D1029BCB
:1020A000069D93F863304000002D3DD1052B3BD9B0
:1020B00001214FF40062019C0A9E0EF1010E5FFAAD
:1020C0008EF534449D420194B3D3029ADDF814A0F6
:1020D00092F864200B980AF1010A5FFA8AF18A42A9
:1020E0008044834498D8029991F8601003980C9C1E
:1020F00001300390C0B28142A044A34409F10C090D
:1021000086D80FB0BDE8F08F0FB0BDE8F04FFFF7F5
:1021100089BDC26C90F867305108C3F1010303FB1D
:1021200001F307EB43072FE752004900C3E72023E1
:102130001021CDE908314FF40043079360E62023D6
:102140001020CDE908304FF40043079338E700BF73
:1021500030B5044690F8B73083B00D4621B963B965
:1021600084F8B75003B030BD002BF9D1836B002B3E
:10217000F6D01430FFF74AFCF2E714300190FFF775
:102180009FFC0198B4F88620A168FFF7FFFD019835
:10219000FFF73CFD84F8B75003B030BD08B5B5EE8D
:1021A000C00AF1EE10FA94BF01210021FFF7D0FF21
:1021B000012008BD2DE9F04F4FF0007300270E6895
:1021C000CC6D85B082463D461A46C6FB07256FF0AA
:1021D000730CC4FB0C25D1F8DC60D1F880003C46C0
:1021E000C0FB0734C6FB0C344FF455764868C0FB7F
:1021F0000625886DA7F22C77C0FB0725D1F884004F
:10220000C0FB0634D1F8D800C0FB073441F6D47EB9
:102210008868C0FB0E25964F486DC0FB0725D1F896
:102220008800C0FB0E34D1F8D400C0FB073446F25E
:10223000B868C868C0FB08258E4F086DC0FB07252D
:10224000D1F88C00C0FB0834D1F8D000C0FB0734B3
:10225000DFF830920869C0FB0925874FC86CC0FBC6
:102260000725D1F89000C0FB0934D1F8CC00C0FBA1
:1022700007348F6C4869C0FB082545F2840CC7FB06
:102280000C25D1F8C870D1F89400C0FB0834C7FB06
:102290000C344F6C8869C0FB0E2540F22C7CC7FBC8
:1022A0000C25D1F8C470D1F89800C0FB0E34C7FBE0
:1022B0000C340F6CC869C0FB06254FF0740CC7FBCB
:1022C0000C25D1F8C070D1F89C00C0FB0634C7FBC8
:1022D0000C340C26142705FA06FC45FA07F522FAF9
:1022E00007F242EA0C025615B6EBE27F1BBFD51788
:1022F00085F4FF42921182F07F02AAF80020142593
:1023000022460C2402FA04F642FA05F223FA05F3F7
:1023100043EA06035C15B4EBE37F4FEAE37216BFB2
:1023200082F4FF439B1183F07F0301F58054AAF8E8
:1023300002304FF00077002625683A4633464FF4C6
:10234000D074C5FB042301F584552D68C5FB0476C4
:1023500041F204040D5941F67C04C5FB042341F20B
:1023600084054D59C5FB047641F208040D5949F224
:10237000FC74C5FB042341F288054D59C5FB047666
:1023800041F20C0514464A593C4DC2FB054341F24B
:102390008C0C3A4651F80C70C7FB052641F210052B
:1023A0004F59374DC7FB054341F29007CF59C7FB43
:1023B000052641F214054F596FF0B305C7FB0543DD
:1023C00041F29407CF59C7FB052641F218054F5932
:1023D0004FF41275C7FB054341F29807CF59C7FB6D
:1023E000052641F21C054F596FF01305C7FB054345
:1023F00041F29C07CF59C7FB05260C25142703FA89
:1024000005FC43FA07F324FA07F444EA0C046515C3
:10241000B5EBE47F4FEAE47316BF83F4FF44A411E5
:1024200084F07F04AAF84040134634460C22142559
:1024300004FA02F644FA05F423FA05F343EA060324
:102440005C15DA17B4EBE37F16BF82F4FF439B11F0
:1024500083F07F03AAF842300AF10803CDE9013A7C
:102460006FF00303DFF820B04FF0680E984611E0DC
:102470007CAFFFFF3CB6FDFFC44902004CE80300FF
:102480002464FFFF78940400E0CE0800DBE9108E9E
:102490000BF1400BD1F80001D1F85C314FF0007422
:1024A0004FF0000CC0FB084C4FF000720026C0FB40
:1024B0000E26CEF10009C3FB094CC3FB08264FF0E2
:1024C0000070D1F880A103920027CAFB08074FF0E3
:1024D00000730025CAFB0E35D1F8DC21C2FB0907C9
:1024E000C2FB0835DBE902AED1F80491D1F858817E
:1024F000C9FB0A4C039AC9FB0E26CEF10009C8FBA2
:10250000094CC8FB0A260392D1F8D881D1F884215E
:10251000C2FB0A07C2FB0E35C8FB0907C8FB0A3518
:10252000DBE904AED1F80891D1F85481C9FB0A4C1B
:10253000039AC9FB0E26CEF10009C8FB094CC8FB63
:102540000A260392D1F8D481D1F88821C2FB0A0768
:10255000C2FB0E35C8FB0907C8FB0A35DBE906AE2E
:10256000D1F80C91D1F85081C9FB0A4C039AC9FBF0
:102570000E26CEF10009C8FB094CC8FB0A260392BF
:10258000D1F8D081D1F88C21C2FB0A07C2FB0E35ED
:10259000C8FB0907C8FB0A35DBE908AED1F8109182
:1025A000D1F84C81C9FB0A4C039AC9FB0E26CEF127
:1025B0000009C8FB094CC8FB0A260392D1F8CC815C
:1025C000D1F89021C2FB0A07C2FB0E35C8FB0907F0
:1025D000C8FB0A35DBE90AAED1F81491D1F848817D
:1025E000C9FB0A4C039AC9FB0E26CEF10009C8FBB1
:1025F000094CC8FB0A260392D1F8C881D1F894216E
:10260000C2FB0A07C2FB0E35C8FB0907C8FB0A3527
:10261000DBE90CAED1F81891D1F84481C9FB0A4C22
:10262000039AC9FB0E26CEF10009C8FB094CC8FB72
:102630000A260392D1F8C481D1F89821C2FB0A0777
:10264000C2FB0E35C8FB0907C8FB0A35DBE90EAE35
:10265000D1F81C91D1F84081C9FB0A4C039AC9FBFF
:102660000E26CEF10009C8FB094CC8FB0A260392CE
:10267000D1F8C081D1F89C21C2FB0A07C2FB0E35FC
:10268000C8FB0907C8FB0A350C224FF014080CFAE6
:1026900002FE4CFA08FC24FA08F444EA0E044FEA5D
:1026A000645E4FEAE47CBEEBE47F18BF8CF4FF4429
:1026B000019A0CBFA41184F07F0422F8044C4FF05F
:1026C000140C0C2207FA02F447FA0CF720FA0CF06B
:1026D00040EA04004715C417B7EBE07F18BF84F445
:1026E000FF40019A0CBF801180F07F0022F8020C9D
:1026F0000C24039A142706FA04F046FA07F622FA85
:1027000007F242EA00025415D017B4EBE27F18BF7B
:1027100080F4FF4202980CBF921182F07F02A0F871
:102720007C2014240C2005FA00F245FA04F523FA63
:1027300004F343EA02035815DA17B0EBE37F18BF3E
:1027400082F4FF43029A0CBF9B1183F07F03A2F82F
:102750007E30019B04330193131F0293044B9B456E
:1027600001F580717FF492AE05B0BDE8F08F00BF37
:1027700060D208000120704730B43B4B0021032099
:102780000124C3F8F00584B0C3F8F4150A460846DE
:10279000C3F80045130103F1804303F5E043013220
:1027A000082AC3F81405C3F81005F3D12E4B2F4A9D
:1027B000092001214FF400350DF10204C3F818552A
:1027C000C3F81405C3F81005C3F82C46C3F8301637
:1027D00019601368002BFCD0002313601368244A8F
:1027E00003930121234B039811601A68002AFCD03F
:1027F00000221A601B68204A029301211F4B029895
:1028000011601A68002AFCD000221A601968164B61
:1028100001910199C3F80025BDF9023093421BDBF9
:1028200007EE903A9FED166ADFED166AB8EEE77A8A
:10283000C7EE067A67EEA67AF4EE677AF1EE10FA42
:102840000DD617EE903A23F0030040F00200A0F1FD
:10285000FF4004B030BC7047DFED0B7AF1E70B4866
:1028600004B030BC704700BF0070004000710040F1
:102870000470004004710040087000401471004072
:10288000FFA66A463333534000000000F4190800E5
:10289000074B4FF6FF7103F52A721888884203F13F
:1028A000880303D19342F8D1024870470248704729
:1028B000703D0120EC190800F819080070B42E4D85
:1028C0002A1883B092F9241007291EDD294491F8B3
:1028D0004C309B09032B3DD0012B0CBF4FF4003132
:1028E0004FF440311F2886BF244A00F01F004FF0EC
:1028F000A04202EB8000D0F8003723F440330B43B2
:10290000C0F8003703B070BC7047CBB2072BF9D8C2
:10291000880000F1804000F5C0409B00D0F81045D1
:1029200003F1804303F5C24344F001040026C0F8DC
:1029300010451E6092F924001A6855F82030019263
:10294000019A002BDED00E4A012303FA01F1C2F8EE
:102950000413D7E71F288ABF084B4FF0A04300F0AD
:102960001F01D3F8103598BF0146CB4003F0010397
:1029700002331904B6E700BF1C45012000030050D4
:102980000060004001F06043B3F1005F5FD1F0B43C
:102990000279494C02EBC20504EB850582B06D68F3
:1029A000D30025B106684FF40477C6F808731344C2
:1029B00004EB83039A694ABB0125C3E90652D96037
:1029C0000368C3F81021D3F8106103680196019ED3
:1029D000C3F84421D3F8442103680092009AC3F855
:1029E0003415C3F8385503681D60057905EBC50338
:1029F00004EB8303EE005B685BB303682F484FF47E
:102A00000472C3F8042302B0F0BC7047DA69002AEC
:102A100047D101251961DD610368C3F81021D3F89E
:102A2000106103680196019EC3F84421D3F8442144
:102A300003680092009AC3F83415C3F83855026849
:102A4000D2F8003243F02003C2F80032CDE71C4830
:102A50007047036801E0C1B9E8B9D3F81021D3F891
:102A60004411D3F82401002AF5D0144B3544154EF7
:102A7000002204EB850490420CBF18463046083310
:102A8000A261914218BF1846BDE7354404EB8504A6
:102A90000D48A261B7E7354404EB85040948A161FC
:102AA000B1E735B1036809484FF40472C3F8042351
:102AB000A9E70648A7E700BFD44401200000AD0BFA
:102AC0000A00AD0B0100AD0B0800AD0B0B00AD0B08
:102AD00010B50378012B0C4602D0022B00D010BD9C
:102AE000D0E9011204F11000F8F760F8606804F111
:102AF0002001BDE81040FFF745BF00BF10B40368D8
:102B00000022C3F8402183B0D3F84021036801922A
:102B10004FF48032019CC3F804230368C3F84015C6
:102B200003B05DF8044B7047F0B42D4B2D4A1B6881
:102B3000156819682C4A01244C641B68D3F8446555
:102B400002F1200452F8043F13B11979814203D0F5
:102B5000A242F7D1F0BC7047DA793ABB5A6998695A
:102B6000D9891C8A9F89AA1AA4B2301AC2EB0242E0
:102B700014FA81F102444FF6FE744FF6FF70A24240
:102B800088BF0246B1FBF7F007FB1011986820F8E8
:102B900011201A8A998992B291421BD91A8A01325C
:102BA00092B21A825D619E61F0BC70471F2888BF97
:102BB0000E4A597994BF4FF0A04200F01F00D2F89E
:102BC000102522FA00F000F001008142EAD0002234
:102BD000DA71E7E7DA89013292B2DA81E2E700BF1F
:102BE0009C48012028480120D834012000030050CF
:102BF0002DE9F047002482B081468A46174600F549
:102C0000A075A0464FF480362B6806FA04F283B113
:102C1000D9F80413A00000F5A0730A4298B208D0B6
:102C2000C5F800802B6801933968DAF80030019A02
:102C300098470134042C05F10405E5D102B0BDE844
:102C4000F08700BF0349044801F110020C31FFF77F
:102C5000CFBF00BF5444012000A0004002490348F8
:102C60000A1DFFF7C5BF00BF54440120009000407B
:102C70002DE9F0430679594F06EBC60307EB8302B3
:102C80008646507F83B0002840F085809B000C462C
:102C9000FB584FEAC60C0BB1012353770CEB06052A
:102CA00007EB850594E80F0095F8209005F10C08D6
:102CB000B9F1FF0F88E80F0002D0AB7F002B3CD0AA
:102CC00022686AB102F06043B3F1005F08D0664445
:102CD00007EB8607002342487B7703B0BDE8F0830B
:102CE000A36823B103F06043B3F1005FEFD1DEF8D6
:102CF00000306168C3F84425C3F84815D4E90212CE
:102D0000C3F834150021C3F83825C3F81811D3F8D7
:102D10001821019201200CEB0602019CC3F850150A
:102D2000C3F84015186157F82220B2B12D4840224F
:102D3000C3F8042303B0BDE8F083EB7F7BB3B9F1A4
:102D40001F0F8ABF284A4FF0A04209F01F09012334
:102D500003FA09F3C2F80835B2E7D3F81821002ABC
:102D6000FBD0664407EB860797F82030FF2B24D072
:102D7000BA7F12BBFA7F12B31F2B88BF1A491948BA
:102D800094BF4FF0A04103F01F03012202FA03F3A6
:102D9000C1F80C35A1E7154803B0BDE8F083B9F1DF
:102DA0001F0F8ABF104A4FF0A04209F01F090123EC
:102DB00003FA09F3C2F80C3582E70A488DE71F2BA6
:102DC00088BF0949074894BF4FF0A04103F01F0393
:102DD000012202FA03F3C1F808357EE70C44012012
:102DE0000A00AD0B0000AD0B000300500B00AD0B53
:102DF0001AB32DE9F043DFF8489085B080460E46BF
:102E00001546002701E02D1B13D0D8F804000097C9
:102E1000C4680197AC4228BF2C466946CDE90264DC
:102E2000FFF726FF48452644EDD0002005B0BDE859
:102E3000F083012005B0BDE8F0830120704700BF9A
:102E40000000AD0B2DE9F04F0746406885B0D0F883
:102E5000008022B3DFF85CA0DFF85C900E461546D8
:102E60000FE032464FF0000B6946CDE90024CDE972
:102E700002BBFFF7FDFE4845264414D12D1B0ED0A2
:102E80007868C468AC4228BF2C46D045E9D12246B8
:102E90000748314644F0D2FD7868054AE2E7012050
:102EA00005B0BDE8F08F584605B0BDE8F08F00BF13
:102EB00000E0002000F002400000AD0B70B582B0D1
:102EC000FF2305460E46083001218DF80430FAF73D
:102ED00087FA002468680134012201A9FFF7B2FFD4
:102EE000A642F7D102B070BD40F20110814204D079
:102EF00016221A604FF0FF30704712F00100FBD02D
:102F0000034BD88980B2003818BF0120704700BF3A
:102F1000DC22012040F20110814204D016221A6006
:102F20004FF0FF30704712F00400FBD0044B58788C
:102F30000028F7D09B78002B0CBF0020042070479E
:102F4000DC22012008B5074BD3F80630B3F5966FA5
:102F500000D008BD4FF080434E22C3F81C25F8F77F
:102F600021FA00BFB006012030B483780579194CEE
:102F700003F07F01DB09580001EB41021844D20045
:102F800002EB800222441572ABB9134A01F10C0026
:102F9000012303FA00F0C2F80403D2F8140503FA7F
:102FA00001F10143C2F81415BFF36F8FBFF34F8FC8
:102FB000012030BC7047084A881C012303FA00F046
:102FC000C2F80403D2F8100503FA01F10143C2F874
:102FD0001015E9E7740F01200070024070B4846896
:102FE000944218D3446802EB420204EB820492003C
:102FF000657A85B94D7995B10E78A479C6F1080640
:1030000034411C6040680244107A10281CD80A79A8
:103010004AB3154600E00025284670BC70470D797C
:103020004DB9097AA28809B152BA92B2012528464F
:103030001A6070BC70470978A279C1F108010A4191
:1030400028461A6070BC7047D0798A78121A92B2FA
:1030500002F10A0080B2142803D912B212F1DB0F78
:1030600009DA0A7922B1002228461A6070BC70473A
:1030700001221A60D0E7DB2AC9DDF2E7F0B583B0A0
:10308000002305460C468DF80430EFF31083002B27
:1030900075D04FF080531A69B5FBF2F302FB13535E
:1030A0006BB94F4B0222C3F804251A46C3F80855E2
:1030B000D2F80034D907FBD50023C2F80435484BB9
:1030C0000122C3F8042515F0030339D14FF48056CB
:1030D0004FF4806204EB8202DFF804E1043A211F1E
:1030E000A5EB040C51F8047FDEF8000410F0010099
:1030F000FAD04CF80170BFF35F8F8A42F2D1CBB1A6
:10310000334405F003022344354434444FF0FF3187
:1031100001AE3244019114F8011B02F8011BA342D5
:10312000F9D101992E4AD2F80034DB07FBD529608A
:10313000BFF35F8F2A4B0022C3F8042503B0F0BD14
:103140004FF0FF32C3F10407019201AA21461A444D
:103150003C44EE1A11F8010B02F8010BA142F9D11F
:1031600001981F49D1F80024D207FBD53060BFF386
:103170005F8F40F6FC763D4440F2FF32AAE701A89B
:10318000F8F70EF99DF80430002B82D0154E012778
:10319000280B3770F8F70AFDF8B9F8F709FD02288F
:1031A0001BD04FF40072214628463770F8F7FCFC1C
:1031B00098B9F8F7FDFC02280FD004F5006105F579
:1031C00000604FF400723770F8F7EEFC28B9F8F79A
:1031D000EFFC023818BF0120B0E7002003B0F0BDBB
:1031E00000E001407C480120F0B5ADF5805D81B084
:1031F00016461F460C46054611B9B2F5805F13D03E
:10320000294668464FF4805244F018FC324639464D
:103210000DEB040044F012FC69462846FFF72EFF30
:103220000DF5805D01B0F0BD1946FFF727FF0DF5E4
:10323000805D01B0F0BD00BFF8B546680E44C6F32E
:103240000B01761AABB117461D4601E02D1B10D0BD
:10325000C1F58054AC4228BF2C463B46304622463E
:10326000FFF7C2FF274406F5805600210028EDD164
:10327000F8BD0120F8BD00BF044B054A5B8B054833
:103280009BB2002B18BF1046704700BFB00601204C
:10329000F8190800EC190800F0B54279012A83B04A
:1032A00004460D461AD0D0E9023101338360488CC0
:1032B0008342C8BF4B8405F11003C8BF6279002167
:1032C0003F2BA17115D8803D032AEDB20CD92046C1
:1032D0000121F5F747FA057003B0F0BD01F11003C5
:1032E0003F2B40D8803DEDB2A36A0133A362204654
:1032F000F1E7032A37D901212046F5F733FA1423E1
:103300000DF1050103700E4605F07F02E8B2ED11E4
:103310006B1C012B374606F8012DF5D801352BD053
:10332000430603D5002306F8013CBE1E6379032B38
:10333000A1EB06011CD8A36A1944A162204601AC86
:10334000A6420BD00146334613F8012B62F07F02F0
:10335000A34201F8012BF7D19E1B30449DF80430A5
:10336000037003B0F0BDA36A0133A3622046C6E731
:103370002046F5F7F7F9E2E74206D7D47F2306F8AF
:10338000013CBE1ED2E700BF30B4C468828EA58B5C
:10339000638B44792B44042C02F101051A4408BFC5
:1033A000C36B858608BF43F82210172130BCF5F7A0
:1033B000F5B900BF4379012B0ED0D0E9023210B429
:1033C00001338360548CA342C8BF538400235DF84B
:1033D000044B8371FFF7D8BFFFF7D6BF806A8968B7
:1033E000FFF7E8BF4379012B15D010B5D0E90232C1
:1033F00001338360548CA342C8BF53840023142933
:1034000083711AD0152921D013290DD0BDE81040A1
:103410002249FFF7B9BF142939D015292BD0132918
:103420002FD01E49FFF7B0BF4379032B17D90121D5
:10343000F5F798F91023037010BD4379032B12D9C7
:103440000121F5F78FF91123037010BD4379032B88
:103450000DD90121F5F786F91223037010BD836A97
:1034600001338362E6E7836A01338362EBE7836AB1
:1034700001338362F0E7836A0133836212230370AE
:103480007047836A01338362102303707047836A35
:103490000133836211230370704700BFC019080015
:1034A00010B5044600210068F5F754FD206814218A
:1034B000FFF798FF20680121BDE81040F6F720B81B
:1034C00010B504460022806AF5F752FB54F8280F25
:1034D00000231A461946F5F7BFFF2046BDE8104005
:1034E000FFF7DEBF0C4A00F07F0302EB430202EB62
:1034F000D01000F12003987810F0010008D19A78DC
:10350000520707D49A7842F004029A70012070475B
:1035100000207047704700BFFC3B01200C4A00F0C0
:103520007F0302EB430202EBD01000F120039A78F4
:1035300012F0010209D19978C1F38000490706D53C
:10354000997862F382019970704700207047704744
:10355000FC3B01204206064B0BBF012240F4807069
:103560005A65C3F81805BFF36F8FBFF34F8F7047CD
:1035700000700240084608B5FFF7ECFF094B01F068
:103580007F0003EB400303EBD11191F8223043F0AD
:10359000020381F8223091F8223043F0010381F8D0
:1035A000223008BDFC3B012001207047704700BF5E
:1035B00040F20110814217BF162202F004001A6087
:1035C0004FF0FF30704700BF00487047F419080003
:1035D000012070470120704700487047F419080027
:1035E00000487047F419080080687047007940006F
:1035F00040F00100704700BF02280BD193070BD1A8
:1036000010B50D4B0C461168994282B006D00B489C
:1036100002B010BD00207047084870479168A0684C
:103620000192F6F769FE019A0028F0D01279237909
:103630009A42ECD10248EBE7ACDD0700EC19080038
:10364000F8190800807D400040F00100704700BF7D
:10365000034A8079034B002814BF10461846704770
:10366000F8190800EC1908008088400040F00100BB
:10367000704700BF406820F0030040F00200A0F156
:10368000FF407047428D8AB32DE9F041184E194F23
:103690000546884600246B6853F83430990704D1F6
:1036A0001868B04206D0B8420CD001349442F2D32C
:1036B000BDE8F08193F8512068F3410283F851206E
:1036C0006A8DF2E793F82E008446C0F3C0004045AF
:1036D00068F3C30CE9D01CF0040F83F82EC003D1AB
:1036E00041461846FFF7CEFF6A8DDEE7704700BF00
:1036F0004CFF070028FB070090F8B7309FED040A45
:10370000F7EE007A002B08BFB0EE670A704700BFE3
:103710000000000004288A6809D0052805D108485F
:1037200000EA420040F00100704700207047054B5E
:10373000054990B2002814BF18460846704700BFDC
:10374000FEFF0100F8190800EC190800808840000D
:1037500040F00100704700BFC088400040F0010009
:10376000704700BF10B504460846F6F719FA2071F5
:10377000004810BDF419080008B5F9F7B3FE014878
:1037800008BD00BFF419080008B50868F9F7AAFEDB
:10379000004808BDF419080000234360C3600148D5
:1037A000704700BFF41908000B68024800225A60F5
:1037B000704700BFF4190800034A8068034B0028D3
:1037C00014BF104618467047F8190800EC19080095
:1037D00010B5044601211C30F9F702FE636800228F
:1037E0001A7210BD836803B970470430F9F77ABEC6
:1037F00008B5FFF7F7FF014808BD00BFF41908003E
:1038000008B50868FFF7EEFF004808BDF419080086
:10381000836803B9704710B504460430F9F762FEB7
:1038200094F820309A0702D4DB0708D410BD04F1C5
:103830000C00F9F757FE94F82030DB07F6D504F1B9
:103840001400BDE81040F9F74DBE00BF08B5086888
:10385000FFF7DEFF004808BDF419080008B5FFF7C0
:10386000D7FF014808BD00BFF419080090F82430C4
:1038700083B1002210B41346144600EB83030132D7
:10388000DB6A9C6090F82410D3B29942F5D85DF8B9
:10389000044B7047704700BF836803B9704710B589
:1038A00004460430F9F71EFE04F10C00BDE8104098
:1038B000F9F718BE08B50868FFF7EEFF004808BD25
:1038C000F419080008B5FFF7E7FF014808BD00BF7D
:1038D000F419080008B50868C36813B10430FFF78D
:1038E00081FF014808BD00BFF41908000B680248B9
:1038F0000022C3E901227047F419080041680A7ADE
:103900002AB901230B72416818460A7270470020D9
:10391000704700BF43681A7A12B9012018727047C5
:103920000020704741680A7A2AB901230B72416866
:1039300018460A7270470020704700BF037A1BB90F
:10394000012303720148704701487047F8190800C5
:10395000EC190800054B0649064810B403F144026F
:1039600001240C705A665DF8044B7047B84501207D
:103970005E480120F41908004279032A0346026ACE
:1039800002D8114419627047006B11441044196247
:10399000704700BF70B58AB06846F3F731FB0F4A35
:1039A0000F4C15680F4E241A05F580602044012144
:1039B000F8F7E2F9306030B10B4B1D6003680B4A39
:1039C0001A600AB070BD04F5C8400121F8F7D4F9B7
:1039D000054B30604FF4C0421A60EFE7440201200B
:1039E000000004208048012030400120EF297801A8
:1039F00010B50A4C206880B1094A0A4B12681B684E
:103A00009A4207D0F8F72AF900232360BDE8104056
:103A1000FFF7C0BF0368044A1A6010BD8048012048
:103A20004402012030400120EF297801037A012B64
:103A300005D0044A0448022B08BF104670470348CB
:103A4000704700BFACA40800F4190800A8A408003F
:103A50000E4B10B54FF4D8721846002144F034F8DC
:103A6000034600F12401002200F1A4045960084833
:103A7000DA8101211A825C615A829860DA83986146
:103A80001A84197319775A8410BD00BFDC220120F3
:103A90008000010038B5134B4FF40B62184600212B
:103AA00044F012F803464FF44242FF20012108255A
:103AB00003F130045871DA8003F586600022198121
:103AC0004FF482315A831D739A831C61DA83186222
:103AD0005A855A819A851A7683F828205961596245
:103AE000DA8538BDB00601202DE9F043C36885B002
:103AF0000646013B901C9842ADF8062002D905B05D
:103B0000BDE8F0830F46EFF3108172B6DFF8D08086
:103B1000D8F80830002B5BD12F4A304C0120C8F870
:103B20000800D2F880002040C8F80000C2F88040A9
:103B3000D2F88400C8F804004FF0FF309946C2F86C
:103B4000840001B962B606F108052846F7F724F8A3
:103B5000F368BDF80620013B02321B1A93424FF076
:103B6000020213D20DF10E012846F7F743F8BDF813
:103B70000E30002BE9D000242846F6F7E3FF01348D
:103B8000BDF80E20A3B29A42F6D8DEE70DF1060189
:103B90002846F7F70BF8BDF8062039462846F7F710
:103BA00005F8D8F80830002BA9D0B9F1000FA6D13C
:103BB000EFF3108272B6084BD8F800101960D8F8ED
:103BC00004105960C8F80890002A98D162B696E7A8
:103BD0004FF00109B5E700BF00E100E0FC06FFBDC2
:103BE0001048012038B50388A3F130021F2A0BD8F2
:103BF0004D8C8288ADB29542044605D1392B10D048
:103C00003C2B03D0382B01D0002038BD0B8C002278
:103C10009BB281F8272013B10846F9F767FA012013
:103C200038BD4B6842899B8A9A42F8D10846E2899E
:103C300004F11001FFF758FF237B022BEFD16189BC
:103C40002846F9F751FA012038BD00BF38B502887F
:103C5000502A034605D0572A19D0112A10D0002027
:103C600038BD4868DA88848A9D88944220D0408C88
:103C700090420AD15B8ADB0715D54D84012038BDFF
:103C80004A8C808893B298420DD0012038BD0B8CAD
:103C900000229BB281F82720002BF6D00846F9F7C6
:103CA00025FA0120F2E74FF6FF734B84012038BD5F
:103CB0004A8C4FF6FF7092B282420BD04A8C92B27D
:103CC0009542CCD108461A8A03F11201FFF70CFF86
:103CD000012038BD4D84F5E708B5074B1B78012B53
:103CE00002D9012800D0FEE7044B054A43EA002030
:103CF0009061F7F757FB00BF2E400120AF0000ADE9
:103D0000C8480120F8B5244ED6F8FC70002F40D0EA
:103D1000C01B48BF0F300711F908D6F8F80007F0AC
:103D20000704435C0122A24023EA020343544FEA02
:103D3000970ED6F8F04014F80E107546384607F086
:103D400003034FF0030C5B000CFA03F321EA0303B7
:103D500063550130D6F8F040850800F00303615D3B
:103D60005A0041FA02F202F00302022AEBD0C01B11
:103D7000082828BF0820833056F820307345D6F82D
:103D8000303288BF46F820E0734538BFC6F830E2CD
:103D9000F8BD0820FFF7A0FFB8450120034BB3F89A
:103DA0000C2212B908B1FFF7ADBF7047B84501202A
:103DB00010B504464068F8F7A3FD94F82100F9F720
:103DC00073FB94F82200F9F76FFBFF2384F821308E
:103DD00084F822302069FFF7E1FF0023C4E90533AE
:103DE000E36110BD08B5086890F82230FF2B01D0C0
:103DF000FFF7DEFF004808BDF419080008B50220EF
:103E0000FFF76AFF08B50120FFF766FF08B50A2033
:103E1000FFF762FF08B5124AD36913B90620FFF70E
:103E20005BFF996C586011611968D1611846C468CC
:103E3000056946698769D0F81C80D0F82090D0F8D1
:103E400024A0D0F828B0D0F82CD090ED0C8B90EDB9
:103E50000E9B90ED10ABD0F808E00120704700BF3A
:103E6000B845012008B5094AC31DD2E9031023F063
:103E7000070303448B4201D8136108BD40F21E3191
:103E80000348F5F7A5FFFFF7C5FF00BFB8450120C0
:103E90004C3C0800400040F0010108B50248F5F72D
:103EA00097FFFFF7B7FF00BF983B080010B501462A
:103EB00082B040F24530F6F765FCC4684CB1084664
:103EC00001AB00220121A047013005D0044802B017
:103ED00010BD1620FFF7DEFF0198FFF7DBFF00BFE4
:103EE000F419080010B5014682B040F24530F6F7EB
:103EF00049FC024601ABD468084600220421A047D1
:103F0000013002D0024802B010BD0198FFF7C2FF95
:103F1000F41908000868FFF7E5BF00BF0868FFF75D
:103F2000E1BF00BF38B501460446456851F8280B8B
:103F300004F108030122A847A36833B910B984F833
:103F4000280038BD94F8280038BD1846FFF7A2FFB6
:103F500008B5838803F03003302B00D008BD1E2045
:103F6000FFF798FF38B5094BD3F8DC405CB1054644
:103F700001E0E4683CB12168284643F0FBFD0028DD
:103F8000F7D1A06838BD1620FFF784FFB84501209F
:103F900000B585B00223009303ABF6F769FC039BE1
:103FA0002BB10B2B09D1064805B05DF804FB40008E
:103FB00040F0010005B05DF804FB1846FFF76AFF0A
:103FC000F4190800FFF7E4BF08B5044B5A6E02B9B4
:103FD00008BD586E00225A66FFF71CFFB845012045
:103FE000014608B50248F5F7F3FEFFF713FF00BFDF
:103FF000B839080008B50248F5F7E0FEFFF70AFFF8
:10400000C43C080008B520B90448F5F7D7FEFFF70F
:1040100001FF09680148F5F7DBFEF8E73C3D0800C1
:1040200070B543681E7A8EB901251D7290F8313043
:1040300090F83020C16A04464068F9F723F904F18A
:104040001C003146F9F7CCF9284670BD002070BD40
:1040500010B5084A084B1068084A01681268012424
:10406000CC601B889BB232F81310FEF747FD036843
:104070001C6010BDA04801203448012030480120B8
:10408000B0F5A07F00D0704710B4244B244A1B68C1
:1040900024481B68008801245C60138823449BB279
:1040A000138013889BB2984222D9138813F0010F12
:1040B0004B6815D05B684FF0FF32C3F860254B6842
:1040C0001A7A1F2A86BF184902F01F024FF0A0413A
:1040D00001239340C1F80C355DF8044BFFF7B8BFDE
:1040E0005A681B7AC2F860355DF8044BFFF7B0BF21
:1040F0004B685B684FF0FF32C3F860254B681A7A53
:104100001F2A86BF084902F01F024FF0A041012379
:104110009340C1F80C355DF8044B7047A04801206E
:1041200034480120364801200003005010B5037BBD
:10413000DB07044602D50023A36010BD8068FFF7AB
:104140002DFE0023A36010BD022970B5044615D0D2
:10415000042908D0012904D016221A604FF0FF303C
:1041600070BD002070BD45682DB12B7BDB0720D5CD
:104170002846FFF713FE0020606070BD50680128DC
:1041800015D002280CD161684D68106829182CBF21
:1041900001260026002813DB002EDDD10B4602E0AD
:1041A00011680B4648B9A1601360002070BDA56876
:1041B000EBE7A868FFF7F2FDDAE70029F3DA00255C
:1041C000A942EBD900210B46EDE700BF2DE9F043F2
:1041D00014468BB00A46A107129E074698461BD488
:1041E00014F0040F0CBF00232023009302A8139B9C
:1041F0002021F5F7C5F9E305054602D5431C1F2B21
:1042000018D914F0400909D09DF808302F2B1CD97B
:1042100002A94FF0000902E02B23E6E702A9CDE94D
:10422000008623462A463846F3F73AFE48440BB048
:10423000BDE8F0830AAA154425211A4405F8201C7C
:1042400000211D4602F8201CDBE70122002302A901
:10425000CDE900323846F3F723FE013E013D8146A9
:104260000DF10901DBE700BF2DE9F04F0B7889B0B4
:10427000824690464FF00009002B00F08E800C46DD
:1042800002E014F8013F0BB1252BFAD1A14280F0D6
:104290000781651ADAE900032A4698472378A9447A
:1042A000002B7AD063780134002B00F0FF804FF0B0
:1042B000200B00260DE02B2B15D0202B16D0212B08
:1042C00017D0302B18D146F040069B4614F8013F1A
:1042D0003BB12D2BEFD114F8013F46F00106002B26
:1042E000F7D100251EE046F00206EFE746F004068F
:1042F000ECE746F00806E9E72378A3F13002092A43
:104300004FF000050BD805EB850503EB450514F8C8
:10431000013FA3F13002092AA5F13005F3D92E2B74
:1043200000F0C98027784FF0FF326C2F04BF677808
:10433000013497B3A7F14503332B00F2A980DFE8DE
:1043400003F0919191A7A7A7A7A7A7A7A789A7A7B8
:10435000A7A7A7A7A77AA7A7A7A7A7A7A7A7A75E63
:10436000506C919191A7A7A7A7A7A7A7A7893DA739
:1043700030A71AA7A77A612358F8041B0022CDE9B9
:104380000036CDE902B50A235046F3F7E5FD814436
:104390006378611C002B7FF472AF484609B0BDE81A
:1043A000F08F531C58F8041B00F0AD80CDE900B528
:1043B00033465046F3F774FD8144E9E707A958F8FE
:1043C000040B0592F3F7DAFC059A0146501CEDD177
:1043D000CDE900B5079A33465046F3F761FD8144B5
:1043E000D6E73346012258F8046B8DF81C60CDE9FE
:1043F00000B507A95046F3F753FD8144C8E758F8C4
:10440000043BCDE900B5002B75D046493346042264
:104410005046F3F745FD8144BAE7612358F8041B81
:104420000122CDE90036CDE902B50A235046F3F763
:1044300093FD8144ACE7A7F11703DBB258F8041BE6
:1044400003958DE84808102300225046F3F784FDB9
:1044500081449DE7612358F8041BCDE902B5CDE9FD
:104460000036F0E708F1070828F00708F8E802012D
:104470000592F2F797FF059A00EE100ACDE9005277
:104480005B46324639465046FFF7A0FE81447FE73F
:10449000DAE9000301222146984709F1010977E78B
:1044A0000C4601342378002B7FF401AF1E464FF0F9
:1044B000200B002536E767782A2F06D158F8042B01
:1044C000A77822EAE27202342FE7A7F13003092B22
:1044D00004F101044FF000023FF627AF02EB820225
:1044E00007EB420214F8017FA7F13003092BA2F178
:1044F0003002F3D919E70C49334605225046F3F749
:10450000CFFC814444E70846059143F025FBCDE903
:1045100000B50246059933465046F3F7C1FC814485
:1045200036E700BF507C0700587C07000EB400B58A
:1045300082B003AA52F8041B0192FFF795FE02B065
:104540005DF804EB03B0704700B50B4683B001463D
:1045500018460193F6F770FA019B02460846034994
:1045600003B05DF804EBFFF7E1BF00BF847C0700F8
:1045700010B50B7A0446C8684BB9F6F75DFA0246E7
:104580000B4620460749BDE81040FFF7CFBFF6F7BE
:1045900053FA02460B4620460349BDE81040FFF798
:1045A000C5BF00BFBC7C07009C7C070038B50C462B
:1045B000D1E9012308490546FFF7B8FFE268012A5F
:1045C000284604D0BDE838400449FFF7AFBFBDE836
:1045D00038400349F3F754BCDC7C0700EC7C07004F
:1045E000107E07000B4602495A68FFF79FBF00BFC5
:1045F000F47C07002DE9F8430C4615462149254473
:104600000646F3F73DFCAC4221D21F4FDFF888800D
:10461000DFF88890013C013D0DE01F2A1DD80A2AD1
:1046200025D00D2A28D0092A1CD041463046FFF754
:104630007DFFAC420BD014F8012F222A01D05C2A56
:10464000EBD139463046FFF771FFAC42F3D130462B
:104650000C49BDE8F843F3F713BC0C493046FFF7AB
:1046600065FFE6E749463046F3F70AFCE1E708490B
:104670003046F3F705FCDCE706493046F3F700FC6B
:10468000D7E700BFF87C0700FC7C0700007D07002F
:10469000047D0700087D0700107D07000C7D0700E2
:1046A0002DE9F04782B00546084601A91646F5F700
:1046B000CDFE032E04467ED0C6B1019E0644B04214
:1046C00080F081800346002103E0222A17D09E4219
:1046D00007D913F8012B272AF7D19E424FF0010189
:1046E000F7D800290CBF2727222709E00346019AA3
:1046F00038492846FFF71AFF02B0BDE8F0872727A0
:104700003549DFF8EC90DFF8EC80DFF8ECA03A46B2
:104710002846FFF70BFF11E00A2A38D00D2A40D0B7
:10472000092A43D0FF2A37D9B2F5803F34BF41462A
:1047300049462846FFF7FAFEA64215D92046F3F768
:1047400071FC02462046F3F795FC9742044613D0CD
:104750005C2A17D0A2F120035E2BDDD81E49284623
:10476000FFF7E4FEA642E9D81B493A462846FFF780
:10477000DDFE02B0BDE8F08718493A462846FFF74B
:10478000D5FED9E716492846F3F77AFBD4E7154951
:104790002846F3F775FBCFE751462846FFF7C6FEDC
:1047A000CAE711492846F3F76BFBC5E70F492846CE
:1047B000F3F766FBC0E70146019A2846FFF71AFFA8
:1047C00002B0BDE8F087044927222846FFF7AEFE75
:1047D0002727C9E7187D0700007D0700FC7C07003C
:1047E000207D0700047D0700087D07000C7D070081
:1047F0002C7D0700107D0700247D070030B40A4699
:10480000054C15680549064B8D420CBF21461946DB
:1048100030BCFFF78BBE00BF347D0700F4480800B2
:10482000487D07000B460249DA88FFF77FBE00BFCC
:104830005C7D07000A460149FFF778BE6C7D0700E2
:104840000B4602495A68FFF771BE00BF747D07002E
:1048500000B583B0024608460191F5F76BF90146B1
:10486000019B1046CA88034903B05DF804EBFFF7CB
:104870005DBE00BF847D07000B4602495A68FFF702
:1048800055BE00BF907D070000B50A4B83B08B4238
:1048900014BFDA21A82140F22913CDE900314FF4E9
:1048A000DE72054940F25913FFF740FE03B05DF890
:1048B00004FB00BF14EB0700A07D070000B5084B08
:1048C00083B08B4214BFB821DE2100918B230549B0
:1048D00040F20E22FFF72AFE03B05DF804FB00BF92
:1048E000E8F40700AC7D070000B5094A83B040F248
:1048F00023138A4214BF1946DC2100918D230549F8
:1049000040F20E22FFF712FE03B05DF804FB00BF79
:1049100048F50700AC7D070000B5094A83B040F2B6
:104920005B138A4214BF1946872100914FF4987394
:10493000044940F20E22FFF7F9FD03B05DF804FBD5
:10494000CCF50700AC7D070010B586B004AA04467C
:1049500003AB084605A9F9F7FDF9059A42B1039B97
:1049600000930749049B2046FFF7E0FD06B010BD09
:10497000DDE9033203492046FFF7D8FD06B010BD3C
:10498000AC7D0700B87D070000B50B4B994283B0A2
:104990000FD00A4B994214BFD2217521009140F2E9
:1049A0003F1307494FF43A72FFF7C0FD03B05DF8BB
:1049B00004FB4FF4A171F1E77415080044150800D9
:1049C000AC7D070000B50C4B994283B010D00B4B67
:1049D000994214BFD7214FF49C7100914FF4B273E8
:1049E000074940F24442FFF7A1FD03B05DF804FB24
:1049F00040F23311F1E700BFA8A40800ACA40800FE
:104A0000AC7D07002DE9F0478D18A942074660D21A
:104A10000C460B46002203E022290ED09D4207D906
:104A200013F8011B2729F7D19D424FF00102F7D857
:104A3000002A0CBF2726222600E027262849DFF877
:104A4000B080DFF8B090DFF8B0A032463846FFF70C
:104A50006DFD013C013D07E07E2A20D82049384603
:104A6000FFF764FDA54213D014F8012FB2421BD00A
:104A70005C2A1FD01F2AEFD80A2A20D00D2A23D063
:104A8000092A0CD149463846F3F7FAF9A542EBD189
:104A9000324638461249BDE8F047FFF747BD414668
:104AA0003846FFF743FDDDE70E4932463846FFF74B
:104AB0003DFDD7E70C493846F3F7E2F9D2E70B4959
:104AC0003846F3F7DDF9CDE751463846F3F7D8F924
:104AD000C8E703492722FFF729FD2726D8E700BFAB
:104AE000007D0700FC7C0700207D0700047D070097
:104AF000247D07000C7D0700087D070070B5174B6B
:104B00000B40062B82B00446164619D0D1E9023577
:104B1000032E01931BD0042E0AD011492046F3F72F
:104B2000AFF9019A29462046FFF76CFF02B070BD2D
:104B3000019A0C492B462046FFF7F8FC02B070BDE5
:104B4000C80801A9F3F71AF9032E0546E3D1019A23
:104B500029462046FFF74EFD02B070BD070080FFDA
:104B60001CB60700187D070010B504468068FFF7E3
:104B700015F92046BDE81040FFF710B903789B07F0
:104B800000D570478068FFF709B900BF10B503680A
:104B9000044623B92046BDE81040FFF7FFB840683F
:104BA000FFF7FCF82046BDE81040FFF7F7B800BF5C
:104BB00080B310B50446006808B1FFF7EFF86068ED
:104BC0000023236008B1FFF7E9F8A06800236360C1
:104BD00008B1FFF7E3F8E0680023A36008B1FFF72E
:104BE000DDF820690023E36008B1FFF7D7F86069BA
:104BF0000023236108B1FFF7D1F8A06900236361A6
:104C000008B1FFF7CBF80023A3612046BDE81040B0
:104C1000FFF7C4B8704700BF08B1FFF7C9BF7047BE
:104C200010B50C686068FFF7F7FF0023C4E909338B
:104C30006360A361A363014810BD00BFF4190800BD
:104C400010B504460068FFF74DF92046BDE8104056
:104C5000FFF7A4B870B543681E7A7EB901251D72AE
:104C600041690446334632464068F8F70BFB04F1CD
:104C700008003146F8F7B4FB284670BD002070BD2F
:104C80002DE9F84383681E7A002E4AD10125044697
:104C90001D7232463346884604F11809016B80685C
:104CA000F8F7F0FA29464846F8F79AFB216A0B789C
:104CB0000F4683F0400307F8013B2A46A068FEF741
:104CC000C1F8A58DE18D0735ED100235B9B194F825
:104CD0003400C0074FEAE60306F0070206F10106BA
:104CE00004D418F803301341DB0705D53946A06812
:104CF0002A46FEF7A7F8E18D8E422F44E7DB01221A
:104D00003946A068FEF79EF848460021F8F768FB90
:104D1000A36800221A7294F8343062F3000384F816
:104D20003430BDE8F88300BFF0B50388112B83B0A1
:104D300004460E464BD0262B44D0102B02D0002028
:104D400003B0F0BD364F00233A464FF6FF7011888E
:104D5000814202F1880203D00133052BF7D10423ED
:104D600003EB0313DA002F4DA1882F48B95207EB4C
:104D7000C30302F16001D865D5F8D4001866394440
:104D80002A489866C5F8D410002004F108015B6633
:104D900083F85A00A3F87600B06151F8080F6C321E
:104DA0004968174403C76846F8F702F9BDF80030B0
:104DB000228A9A4202D8628A9A4203D2A08869461D
:104DC000F8F7F0F800230120F36003B0F0BD144FB2
:104DD00080883A4600231188814202F1880203D07C
:104DE0000133052BF7D1042303EB031307EBC301B6
:104DF0000E48DD00F6F788FC0B48CB6D4FF6FF72CE
:104E00007A5383424FF0000281F85A2002D05A6050
:104E1000227A1A7200230120B36103B0F0BD00BFF3
:104E2000703D0120B8450120F4190800519B030092
:104E3000044B0022DA811A601A825A82DA831A84B9
:104E40005A847047DC220120054B00225A831A60E5
:104E50009A831A71DA835A859A85DA85704700BF7A
:104E6000B0060120827940F20113012A14BF1846CE
:104E700021207047A1F10101B1FA81F1F8B549098A
:104E8000164605461430069F1C46F8F7A9FA012E6F
:104E900017D1AFB1274405F11C06012221466868ED
:104EA000FDF7D0FF01213046F8F79AFA01200444BB
:104EB000F8F700FC00213046F8F792FABC42ECD13A
:104EC000F8BD68683A462146BDE8F840FDF7BABF2C
:104ED00010B500F1240420460021F8F781FA4FF4C0
:104EE0007A70F8F7E7FB20460121F8F779FA4FF4DA
:104EF0007A70F8F7DFFB012010BD00BF034B426A58
:104F00009A4201D0FFF7E4BF00207047203B080021
:104F10002DE9F0410025D0F800808D7583690646A3
:104F20000C46002B55D0C36A01330AD001F1160795
:104F3000D8F8103033F8150000284CD12544002350
:104F4000AB750023A07D19462E27F5696A5C202ADF
:104F500001F1010121D0052A08BFE522092904D168
:104F6000E51800B9AF756F72013304EB030C8CF8D0
:104F7000092088B9A2F14105192D0BD8F569082936
:104F800095F80CE08CBF102508251EEA050F1CBF04
:104F90002032D2B28CF8162001330B29D5D130B98A
:104FA000E2189075F269127B002A08BF002323449F
:104FB00000225A72F369DB7A2372F0691C30F6F72B
:104FC000EDFB2060F0691630F6F7E8FBE080000C9E
:104FD000A080BDE8F0817F2802D9F6F735FC30B11A
:104FE0000135B5F5807F02D007F8010BA0E7002559
:104FF000A4E700000549064B064810B4002201242E
:105000000C701A705DF8044B704700BF683D0120BA
:105010005E480120F4190800084BD3F8182102B9A2
:105020007047002282B0C3F81821D3F818310193D9
:10503000019B034802B0F6F76DBF00BF003002408D
:105040000C4401202DE9F843914B1C682368D3F8E8
:10505000402112B10022C3F84021A36B226C1A60D8
:10506000D4E90B231360A26A1360236801225A60FB
:105070001A64D3F8403594F86830E26A216B116005
:10508000012BDFB200F0F68094F86330012B00F0C2
:10509000DE80002F40F0E98094F86120DFF8F48191
:1050A0004AB33E4648F0010901250FE002EB031325
:1050B00012589B6813604FF40070C84794F8612041
:1050C0000136F3B26D009A42EDB214D994F869300A
:1050D00094F86A104B401D42F2D094F86920F3B264
:1050E0002A424FEA0310A26CE0D102EB0312D2E98C
:1050F00001321A60DFE794F86920236DD2B248F0DC
:10510000010884F86A2094F8682094F8631001324A
:10511000D2B2914284F868200CD8002184F868103B
:1051200094F8692094F864000132D2B2904284F875
:1051300069207AD922680121BB4051604020D160AA
:10514000C2F840351160C047D4E90F321A60B4F894
:105150005C3094F8696094F8630094F8682094F8DF
:105160005E10073300FB0626DB1094F86500DD00B7
:1051700001FB06F205FB02F620B194F86720E06C13
:1051800000FB0266012900F0DA80022900F0848029
:10519000626AD9B24F1ED4E90130FFB2D4E90645A4
:1051A000324400293FD002EB471707F1400120327B
:1051B00052F8206C1E601C6000BF00BF056052F8F2
:1051C0001C6C1E601C6000BF00BF056052F8186CAC
:1051D0001E601C6000BF00BF056052F8146C1E60AA
:1051E0001C6000BF00BF056052F8106C1E601C60A0
:1051F00000BF00BF056052F80C6C1E601C6000BF51
:1052000000BF056052F8086C1E601C6000BF00BF44
:10521000056052F8046C1E601C6000BF00BF2032A5
:105220008A420560C4D1BDE8F88384F8691094F817
:105230006B2042B194F86720C2F10102D2B284F827
:10524000672084F86B10A26D0132A26572E7D4E981
:105250001432C3EBC3036433DB0893422365BFF40A
:1052600018AF2265002F3FF417AF0A4A236D42F0B2
:10527000010848E7D4E91432C3EBC3036433DB0805
:105280009A422365EDD8034A42F001083BE700BF8C
:10529000A406012010F20700626A606894F86210A8
:1052A000A568DBB203F1FF3CD4E906475FFA8CFC4A
:1052B000324400EB4101002BB5D002EB0C1C0CF189
:1052C0002003103232F8106C0E80046000BF00BF63
:1052D0002F6032F80E6C0E80046000BF00BF2F609C
:1052E00032F80C6C0E80046000BF00BF2F6032F8F3
:1052F0000A6C0E80046000BF00BF2F6032F8086C9B
:105300000E80046000BF00BF2F6032F8066C0E8074
:10531000046000BF00BF2F6032F8046C0E80046090
:1053200000BF00BF2F6032F8026C0E80046000BF27
:1053300000BF10329A422F60C4D1BDE8F883626A80
:10534000606894F86210A568DBB203F1FF3CD4E911
:1053500006475FFA8CFC32440144002B3FF463AFF4
:1053600002EBCC0C0CF11003083212F8086C0E7032
:10537000046000BF00BF2F6012F8076C0E7004605D
:1053800000BF00BF2F6012F8066C0E70046000BFF3
:1053900000BF2F6012F8056C0E70046000BF00BFE4
:1053A0002F6012F8046C0E70046000BF00BF2F6005
:1053B00012F8036C0E70046000BF00BF2F6012F87B
:1053C000026C0E70046000BF00BF2F6012F8016C09
:1053D0000E70046000BF00BF083293422F60C4D13A
:1053E000BDE8F883438C4FF6FF729BB2934227D0FF
:1053F00030B4154A448C1146A4B200230D88A5424E
:1054000001F1880106D00133052BF7D14FF0FF30B1
:1054100030BC704703EB031302EBC303B3F87630E1
:105420003BB14268108A033B9842A8BF184630BC83
:1054300070474368188A1428A8BF142030BC7047EE
:105440004FF0FF30704700BF703D012043685BB1F3
:105450005A680AB192790AB1188A70479A7D12F097
:10546000060FF9D0FFF7BEBF4FF0FF30704700BF07
:1054700010B50446C068FEF791FC0023C4E901336F
:10548000E360014810BD00BFF419080008B5436887
:1054900013211888F7F7FAFD004808BDF419080031
:1054A00070B5104E82B04FF42A240125200B3570C0
:1054B00004F58054F6F77AFB08B9F6F779FBB4F5F2
:1054C000322FF3D1084B019301A901224FF42A2076
:1054D000F6F792FB01A901220448F6F78DFB02B012
:1054E00070BD00BF7C48012031304442FC1F0B00DE
:1054F00010B54FF6FF720446FF210120F6F720F9A0
:1055000038B1E31C23F00303044A083303449342F5
:1055100002D9FFF7C5FF024810BD00BFFB1F0B00FB
:1055200004A00A0008B5FFF7BBFF014808BD00BF93
:10553000F419080010B504464068FFF76DFB00231E
:10554000C4E909336360A361A363014810BD00BFD0
:10555000F419080010B50446406818B1F7F7C2FF07
:1055600000236360004810BDF419080008B5044B1F
:1055700002689A4201D1F9F79DFF024808BD00BFB9
:1055800018650800F419080008B590F82230FF2BC0
:1055900001D0FEF70DFC014808BD00BFF41908005A
:1055A0002DE9F04FB1B014911290002800F06B85F6
:1055B00003680093002B00F066854368002B00F021
:1055C000628581681191002900F05D85C1680291B2
:1055D000002900F0588501691091002900F05385D9
:1055E000D0F8BC27002A40F34E811499DDF840B072
:1055F000C1EB4112900001EBC10203EB0213002248
:105600000C92119A159003F1500A411E029B0493CB
:105610000A44089203F5905253460192DA469B469B
:105620005BF8143C022B00F0798116234FF00D0932
:105630000693DBF81830009AB74F126ACDF82CA009
:1056400001335B0007935BF8203C0593520804BFCD
:1056500002330593059A089B03974FF00008002139
:10566000C2F1D202CDE909291991454644469A462C
:1056700028E0009BDBF814705A6B1AF8013F32F9EE
:10568000156002EB450205F10109B2F90220961BF3
:1056900032461FB1039F97F800C06344079FBC4682
:1056A000099F03FB0C73FBF739FF039B0133039343
:1056B000344448EA000800B11995019B1B689C42DC
:1056C00007DA4D46049B03EB8401069B9D42084686
:1056D000CFD1DDE90A9A199B0022B9F10B0FCAE973
:1056E000C822CAE9CA23CAF81823CAF81C2300F33F
:1056F0000781159B0C9ACDF834B0C2EB42121733D8
:1057000003EB420309EB49021344059ADDF840B06C
:10571000CDF81880C2F1D2020E92119ACDF86C9099
:10572000D318CDE91999039319AB0F93C846CDF857
:105730004CA0009B049A5B6B0F9EDDF80C90CDF89B
:10574000248003EB480302EB8405B3F93010B3F96E
:105750002E200D9B05938A1A08F101084FEA820A50
:105760002F465946059819F801CB50F8043B05908F
:105770000E9800EBC303079800FB0C333846CDE9C5
:105780000A12FBF7CBFE069B0A990B9A0343574478
:105790005144069308B1099B336004361CAB9E420A
:1057A000E0D102EB4203002A1C444FEA42031ADD17
:1057B00002F1804103F18043013BABF10400013968
:1057C0000BEB830300EBC2020BEB810150F8046F7B
:1057D0002E6051F8046F6E6053F8046FAE60914212
:1057E00005F10C05F2D1019B1B689C4206DA039B74
:1057F000B8F10D0F03F1030303939AD1019BDDF878
:1058000034B01C605BF8102CDDF84CA0DDF818807B
:10581000DDE91931002A18BF02201B9ACAF81C338F
:1058200008BF01208B42B8BF0B469342B8BF134656
:10583000B8F1000FCAE9C923CAF81803CAF820133F
:1058400000F0BA80C0F2FE8200235FEA48081A46E0
:1058500003F10103F9D50199129B8A60043101918A
:1058600004990C9AD3F8BC3701F51061049108999A
:1058700001323E3193420C920AF1180A0BF1480BA7
:1058800008913FF7CDAE009B1C6A2046002C34D017
:10589000029A41F20823D358002B50DD029A41F2BC
:1058A0000C23D358002B4ADD5FEA640C00F0EE8332
:1058B00014F0010100F08280109AD2F83033002BEE
:1058C00040F0B482D2F84433009A0133526B32F97B
:1058D00013507DE04FF0FF33029A02F59055029C81
:1058E00041F20C2141F204226350A35829688B42F3
:1058F000B8BF0B462B60A350002031B0BDE8F08F3D
:10590000904559D0C0F29E8213465FEA48081A4675
:1059100003F10103F9D59EE7045408005BF8103C3D
:1059200006934BB1009B1B78002B0CBF082306236A
:1059300006934FF003097CE6DDF8189079E6029BA8
:1059400003F590552968002915DD029B974C043B0F
:1059500003EB81016FF0404002E08B421C600AD0F3
:1059600053F8042FB2F1404FF7DDB2F1804FA8BFDA
:1059700018608B42F4D1029A41F20423D1580029D5
:1059800016DD029B894C03F6FC0303EB81016FF0EB
:10599000404002E08B421C600AD053F8042FB2F161
:1059A000404FF7DDB2F1804FA8BF18608B42F4D1B1
:1059B000009B1C6A204677E71F224CE7029A41F2BF
:1059C000042302F59055D2582D689542B8BF15466C
:1059D0004FF0000A002DD44624DD029B5646574660
:1059E000191F03F6FC0451F8043F54F8042F9818CB
:1059F0009B1A0860236008683A4680EAE072A2EBCE
:105A0000E0724CEA020C3A4683EAE372A2EBE372DC
:105A10000136B5424AEA020AE5D1009B1C6A2046DB
:105A200004F00101002900F09F80029B009903F51A
:105A300090550A782B68002A40F0BE801098D0F864
:105A400030C366100E96BCF1000F40F0E181D0F833
:105A500044934A6BD0F82C83554809F10107C6EBF3
:105A6000C60A32F9171000EB8A00C14501904FEACF
:105A7000C60BA3EB01000B4680F2CE81002840F359
:105A8000CB81149CC4EB441E09EB8E0E119C0EF1CD
:105A90003E0E7444A64608F101040394454C5C4450
:105AA00004941EF8014F072CE246E34641D001372B
:105AB000019D32F9172055F82460AD69511A00296B
:105AC000A5EB060541DD029A02EB8304411A043C72
:105AD00000EB030801E0002844D054F8043F1A46C4
:105AE00085FB02929200C4F80029D94682EAE27945
:105AF000A9EBE2794AEA090A86FB03239B002360AB
:105B00005A4683EAE372A2EBE372013881424CEA1F
:105B1000020CA8EB0003DED1039ABA4222D009B3EB
:105B2000009A1EF8014F526B072C084632F91710E5
:105B3000BDD101371F4C0E9D32F9172054F8356046
:105B4000049C511A00296568BDDC039ABA4209D049
:105B50000146E5E7069B019A01330132032B0693C8
:105B6000019277D1009B186A00283FF4C6AEBCF1C1
:105B7000000F00F07E82C0F2838200235FEA4C0CAB
:105B80001A4603F10103F9D5029941F20823BAF14B
:105B9000000FCA5000F06F82FFF69CAE00225FEA51
:105BA0004A0A134602F10102F9D595E6010000C048
:105BB00074A7080064A708001198AF49D0F8F8202E
:105BC0004FEA420B0BEB640B6210059201EB8B1B4F
:105BD00000F1FC0400F586770022012654F8041B2E
:105BE000E06806FA01F1002801F1FF310ADD1044F6
:105BF00019AD05EB820205EB800542F8041BAA42B1
:105C0000FBD10246BC42E9D1109AD2F830C311460A
:105C1000BCF1000F00F08580149B109A0599029F3B
:105C2000C3EB431E02F54772119B0892934A03EBA4
:105C30008E0901234FF0000A09F1550902EBC10258
:105C4000259307F510630792D446CDF818A0049366
:105C5000CDF80490089B009A9869D2F8349053F8D4
:105C6000042B089309EB400303210C46B3F93030B1
:105C700006990130904213FB04113FF76BAF0132DC
:105C800003920DF1640E4A46019E5EF8204000EB3F
:105C90004005755DA54200F0D8806C1CED074FEA09
:105CA000640440F1D9805BF824805C4625680130AB
:105CB00000F1140402EB4402B2F90620D21A002AC1
:105CC00024DD02EB42020A4457F8213085FB03939E
:105CD000049E9B0046F821304FF0000983EAE379E7
:105CE000A9EBE37957F821304AEA090A88FB0393C4
:105CF0009B0047F821304FF0000983EAE379A9EBD4
:105D0000E379033191424CEA090CDDD1039B9842BF
:105D10003FF420AF009B5A6B02EB4404B4F9063009
:105D2000B2E7D2F84443009AD1F82C13526B039196
:105D3000601C149932F91020059DCDF810B0A3EB2A
:105D4000020819ABC1EB411E03EB800304EB8E0983
:105D50000121119C0193494B09F13E09CDE92E1116
:105D60004C4403EBC5030693E2466646A146039BFB
:105D70008342FFF6F7AE019C19F8011F54F8043B6B
:105D8000019499426DD04B1C11F0010F4FEA63034F
:105D900004996DD051F823400B461D68009B5B6B46
:105DA00003EB400133F91030B1F90210C91A414533
:105DB000A8BF4146002900F1010025DD029B01EB4F
:105DC000020E03EB8E0703EB820252F8043B85FBC5
:105DD00003B39B00C2F8FC38B34683EAE37BABEB2A
:105DE000E37B52F8043C4AEA0B0A84FB03B39B00B2
:105DF00042F8043CB34683EAE37BABEBE37B974298
:105E00004CEA0B0CE1D17246B8EB0108AFD1A9E620
:105E10000CF1FF31012933D92046002C3FF46DAD40
:105E2000029941F208221F238B5058E5009B109ADB
:105E30005B6BD2F8402303EB4203B3F9305005EB20
:105E40004505C5E54FF0FF3205E50C4C059D54F8BE
:105E50003580079C65682AE7DBF800800BEB84043B
:105E600024E7064B059953F83140069B5D6895E79A
:105E70000C6801EB830390E7ACA7080064A7080057
:105E80001099009ED1F84003766BD1F82813109139
:105E900006EB40010E9FB1F93010DFF8FC8101EBF9
:105EA0004101A3EB010E431CC7EBC7070493109BF2
:105EB00008EB87080E9F98424FEAC70BACDABEF199
:105EC000020FA9DD149B049CC3EB43139B005533C5
:105ED00004EB44001844119B034401936D4B5B4455
:105EE0000F9319AB9246944691466400059305982A
:105EF000019FDDF83CB016AB17F8012B072A00F024
:105F0000A58058F82250D8F818201D60521B026056
:105F1000059A04339A4200F10400EDD1049B344405
:105F20000133B4F930000D93B4F92E30C01A0028B3
:105F300040F39580199B0693169B07931A9B089331
:105F4000179B09931B9B0A93189B0B9300EB400034
:105F5000029BAEEB00000EEB010203EB81030C92FF
:105F6000039003E0BEF1020F7FF7FCAD1A68069CB8
:105F70001146204680FB01418900C3F800194C46B8
:105F800081EAE174A4EBE1740799084680FB0212F0
:105F900092001A60494682EAE271A1EBE2715A6806
:105FA000089E1546304680FB0565AD00C3F80459D0
:105FB0004F4685EAE577A7EBE577099D284680FB04
:105FC000025292005A604E4682EAE276A6EBE276F0
:105FD0009A680A98154680FB05B5AD00C3F80859C4
:105FE000CB4685EAE57BABEBE57B3C4344EA0B041F
:105FF0000B984AEA040A80FB024292009A604C46DF
:1060000082EAE274A4EBE2740C9A31432143AEF1CC
:10601000030E4CEA010CA2EB0E01039A964503F124
:106020000C039FD1DDE90303109A93423FF49AAD2C
:10603000019B022803F1030301937FF793AD009BBB
:106040005E6B0D9B049386465C0050E7114A0E9DE3
:1060500052F83550DBF804201D60026058E7049BBD
:10606000109A93423FF47EAD019B03330193704637
:10607000E7E71F2288E5029A1F2302F590552EE4D8
:106080004FF0FF3280E54FF0FF3036E42146E24624
:10609000C8E400BF64A7080074A7080010B501F1A8
:1060A000FF4186B021F00302002300EE102A0446CF
:1060B000009367220623102102A8F3F761FA02A9D0
:1060C0002046F1F7DDFE02A82E2141F099FD08B12E
:1060D00006B010BD652102A841F092FD0028F7D15D
:1060E00002A86E2141F08CFD0028F1D10249204622
:1060F000F1F7C6FEECE700BFC07D07002DE9F041D7
:10610000D0F88020054672B13F48002350F8331084
:106110008A4276D00133042BF8D10020F6F75AF8E2
:106120000023C5F88030394B95F8B3601A6805F143
:106130001407974204BF00221A6076B105F1870464
:1061400026444FF0FF0814F8010FFF2801D0F7F79D
:10615000ABF9A64284F80080F5D195F8B46076B129
:1061600005F1A50426444FF0FF0814F8010FFF289D
:1061700001D0F7F799F9B44284F80080F5D195F889
:10618000B000FF2801D0F7F78FF995F8B100FF2391
:10619000984285F8B03001D0F7F786F995F8B2004B
:1061A000FF23984285F8B13001D0F7F77DF96B6A8B
:1061B000FF2285F8B2206BB96C220021384641F0ED
:1061C00083FCA868F9F74EF90023C5E90033AB60FA
:1061D000BDE8F081AB6B43B13846FBF717FCA86B09
:1061E00018B1F9F73FF90023AB63E86D18B1F9F77F
:1061F00039F90023EB65686A0028DDD0F9F732F938
:10620000DAE700EBC30089E74C020120A406012075
:10621000FFF774BF08B5FFF771FF014808BD00BF65
:10622000F419080008B5C36813B10430FDF7DAFAB1
:10623000004808BDF41908002DE9F04F89B09DF819
:106240004850002B65D016464268DFF8F0A01C4687
:10625000137912688146342000FB03A3002D4FF010
:1062600006004FF0020583F82D505FFA81F8C2F85E
:10627000000514BF002320234FF6FF7B0027CDE944
:1062800005765C45D9F804200797254628BF5D466A
:10629000049510798DF80C7000EB40018DF80D809D
:1062A00000EB81000AEB80001168019303AAF5F767
:1062B000F5FF1D4B98422E440AD1641B019BDED191
:1062C000D9F80400F6F74EFA204609B0BDE8F08F81
:1062D0000190D9F80400F6F745FA144B019A9A4256
:1062E0001FD006D9124B9A420BD1132009B0BDE83A
:1062F000F08F104882420CBF0520002009B0BDE895
:10630000F08F0D4882420CBF0520002009B0BDE887
:10631000F08FC9B2F6F764FF002814BF00201320E5
:10632000E4E71020E2E700BF0000AD0B0B00AD0B6F
:106330000100AE0B0A00AD0B0200AE0B6C44012055
:106340002DE9F04385B002AF8146BE6A31BB4FEA0A
:10635000460C0CF1070222F00702E846ADEB020DF5
:1063600002AA6EB11E44013E591E0DF1090480209F
:1063700011F8015F04F8010CB14204F8025BF7D197
:106380000124B9F81C10D9F8040000946346FFF703
:1063900053FF0C37C546BD46BDE8F08306F1080241
:1063A00022F007026C46ADEB020D402219468DF833
:1063B0000820731C32460DF1090001257B6041F075
:1063C0003DFB7B68B9F81C10D9F80400009502AABF
:1063D000FFF732FF0C37A546BD46BDE8F08300BF8E
:1063E00000B543F20402124B12689A4283B00DD0FA
:1063F0004FF08043D3F80C0400F00110A0F101101D
:10640000B0FA80F0400903B05DF804FB002301A856
:106410008DF80430F4F7C4FF9DF80430002BE7D06A
:1064200001A8F5F7FFFC0198003818BF0120EAE742
:10643000DBE5B1510A4B82699A420FD010B500F1E9
:10644000180420460021F6F7CBFF0420F7F732F9B5
:1064500020460121F6F7C4FF012010BD002070473F
:10646000203B08000A4B42699A420FD010B500F158
:10647000140420460021F6F7B3FF0420F7F71AF9B9
:1064800020460121F6F7ACFF012010BD0020704727
:10649000203B080030B591ED010A87B0B5EE400A07
:1064A0000023F1EE10FA0C460546009302A84FF0C7
:1064B00006034FF067024FF010010AD194ED020A73
:1064C000F3F75EF8174902AA2846FEF72FF807B03F
:1064D00030BDF3F755F8144902AA2846FEF726F80E
:1064E00094ED020AB5EEC00AF1EE10FA13DAB4EE3A
:1064F000400AF1EE10FA0ED600230093672206231D
:10650000102102A8F3F73CF8084902AA2846FEF732
:106510000DF807B030BD06492846F1F7B1FC94EDFF
:10652000020AE9E7C47D0700C87D0700D07D0700A7
:10653000CC7D070038B5084B1B6800250446C3F81E
:1065400000550079F6F7B0FF60792571F6F7ACFFDA
:106550006571024838BD00BF48020120F4190800E7
:1065600090F8B72002B1704700B5034683B01430ED
:10657000B3F8862099680190FBF708FC019803B0F6
:106580005DF804EBFBF742BB837AFF2B11D010B50B
:1065900004464068F6F780F8A07AF6F785FF607A3F
:1065A000F6F782FF6268FF230021A3726372117203
:1065B00010BD704708B50868FFF7E6FF004808BD42
:1065C000F419080008B5FFF7DFFF014808BD00BF58
:1065D000F4190800428D002A36D02DE9F0411B4EF7
:1065E0001B4FDFF87080054600246B6853F83400B9
:1065F000830706D10368B34208D0BB420DD04345A0
:106600001CD001349442F0D3BDE8F08105F10803B9
:106610008361F9F779F86A8DF3E790F8503023F049
:10662000140305F1080243F01403826280F850302D
:10663000F8F73AFBF8F77EFB6A8DE2E705F108010F
:1066400000F00AF86A8DDCE7704700BFD0A20800AE
:106650004CFF070028FB07000A1E90F82E3018BFD9
:10666000012262F3410380F82E309B072CD570B4D1
:106670008C7BB0F92420B0F9263014B114461A46A8
:10668000234691F904600D8890F8284006FB0252D9
:10669000028191F905504A8805FB032343810B7958
:1066A00013FB04F303734B7913FB04F343738B7BEA
:1066B00083750B7B03754B7B43758B7913FB04F35D
:1066C000837370BCFFF786BF01B97047FFF782BFC5
:1066D00038B505460C46F9B16B689C422FD094F84A
:1066E0002E2012F002022CD12BB193F82E1062F35F
:1066F000410183F82E1005F124012046FFF7ACFF7D
:1067000094F82E3043F0020384F82E3001236C609D
:1067100085F85830184638BD0C4B93F82E20C2F33C
:10672000400092070FD56A689A42F4D0002AF2D04E
:1067300092F82E3061F3410382F82E30E6E7012013
:1067400038BD002038BD1C46C6E700BF7C010120D3
:106750002DE9F84F90F82E20438D6FF3000280F85A
:106760002E20C3B15D1E6A4FDFF8B481DFF8B4910B
:106770000646ED0073685C5914F0030207D12368E4
:10678000BB420AD0434561D04B4500F08880083DAC
:1067900015F1080FEED1BDE8F88F237F002BF6D05E
:1067A000D4E90103227704F120019847A3699A7B79
:1067B000002A78D1B4F914A0B4F9202093F9040088
:1067C0001988B4F922B0B4F916E0524410FB02F073
:1067D000084400B2208493F90520B3F802C0B4F94C
:1067E0002410F34412FB0BF2624412B2628493F958
:1067F00004C0B4F926B05144B3F800A01CFB01FC5E
:10680000D4440FFA8CFCA4F824C093F90510B3F813
:1068100002A00BEB0E0311FB03F353441BB28445A0
:10682000BCBFA4F820C0A0849342E384B8BF6384B3
:106830002369B8BFE2840022A26213F00302A6D14A
:10684000344819688142A2D11A73A0E7B4F93830EC
:10685000B4F93C209A4256D094F8512092074ED079
:10686000A38794F85030A26823F0070312F00301C5
:1068700084F8503004D127481368834208BF11734D
:10688000636813F0030182D11A682348824203D05F
:10689000224882427FF47BAF9982198377E72046B2
:1068A000FFF756FF73E7B4F916A0B4F9222093F965
:1068B00004001988B4F920B0B4F914E0524410FB74
:1068C00002F0084400B2208493F90520B3F802C016
:1068D000B4F92610F34412FB0BF2624412B2628444
:1068E00093F904C0B4F924B05144B3F800A01CFBE0
:1068F00001FCD4440FFA8CFCA4F824C085E794F87A
:1069000050305B07ADD5D4E91123C4E90E23A8E7C5
:10691000D0A2080034FD070094F6070008FE070027
:106920004CFF070028FB070070B50A4E3368054688
:106930002BB1094A1478013CE4B2147014B100235D
:106940002B7270BD1846F5F745FC00232B7234609E
:1069500070BD00BFA4480120A848012070B4158D67
:1069600005B3D46A002204E00132AA4204F108040B
:1069700018D06668B342F7D1227852B1012A08D004
:10698000022A0D686288194608D0AC46012370BC03
:1069900060474C681946234670BC1847AC46002334
:1069A00070BC604700231B78FFDE00BF38B504468B
:1069B000F6F706FB236906480122002583F8252007
:1069C0005D602169F4F7A0FE2561024838BD00BF73
:1069D000499A0300F41908002DE9F043438D85B06E
:1069E00005460F46002B46D0DFF8B480DFF8B490A0
:1069F000002401266A6852F83400820704D1026834
:106A000042452AD04A4521D0B6B1DDE90123C7E984
:106A100000236B8D00260134A342EBD895F82E306D
:106A2000DB070ED566BB384605F11801F8F7C8F943
:106A3000012005B0BDE8F08301A93846F8F7C0F998
:106A4000E7E786F0010005B0BDE8F08301A9FFF794
:106A5000C3FF0028D8D16B8DDDE7B0F93C20B0F939
:106A600038109142D7D0816BC38FADF808200191C7
:106A7000ADF80A30C8E790F82E0010F00100E2D01F
:106A8000B5F918303B80B5F91A307B80B5F91C3068
:106A9000BB80B5F91E30FB80012005B0BDE8F08356
:106AA0004CFF070028FB0700F0B5436853F831504E
:106AB00015F0030685B00AD12B682A4A9342044692
:106AC00022D0294A93422FD0284A934201D005B0C0
:106AD000F0BD01A92846FFF77FFF3146074628464B
:106AE000FFF7BAFD002FF2D094F82E30DB0715D453
:106AF000DDE90123C4E9062394F82E3043F00103B5
:106B000084F82E3005B0F0BD194BAB61D5E90823F0
:106B1000284601920293F8F7F7FDE5E701A904F191
:106B20001800F8F74DF9E7E7B5F93C30B5F938202A
:106B30009A420ED095F85020A96BADF8083066F354
:106B40000412EB8FAE6285F850200191ADF80A3047
:106B5000CAE795F85030AE6266F3041385F85030FA
:106B6000B5E700BFD0A208004CFF070028FB0700D4
:106B70007C02012070B5428D4368054603EBC103DA
:106B8000013A42855E680C46FFF78EFF6B8D9C4292
:106B90000DD2E20008326B68134493E8030003E966
:106BA00003006B8D01349C4202F10802F3D3696843
:106BB000002241F83320698D6B6803EBC103304636
:106BC0005A6070BD0F4B1A785107C2F3800000D491
:106BD00070471A78C2F3C000120710D40A4A5278DC
:106BE000002AF5D002F07F0103EB410303EBD2133F
:106BF00093F8220000F0010080F0010070470020AF
:106C0000704700BFFC3B0120382001202DE9F04FE8
:106C100090F82E30DC07438D48BF016283B00646F2
:106C200048BF00F118015C1EA3B1B34FDFF8D0825A
:106C3000DFF8D092E40073681D59A80706D12B68CD
:106C4000BB420BD043451ED04B452AD0083C14F123
:106C5000080FF0D1084603B0BDE8F08F2B7F4BB989
:106C60002B699A07F2D1A54A18689042EED11B7B96
:106C7000002BEBD028460191F8F746FD0199A96257
:106C800005F12001E2E795F85130B5F93800B5F982
:106C90003C209B070AD09042D8D0296405F13801E6
:106CA000D4E72846FFF7B2FF0146CFE795F850300A
:106CB00013F0040F02D0904240F09780D5F804A062
:106CC0001AF0030F2AD1DAF800C0DFF83CE2F445ED
:106CD00000F0C180DFF834E2F4451FD1BAF914C0E6
:106CE000BAF918E0E64519D00AF114039942CAF836
:106CF0001C1000F0FE80A5F82CC0BAF91630EB8508
:106D0000BAF918C095F85030A5F830C0BAF91AC0D1
:106D1000A5F832C043F0010385F8503013F00203A8
:106D20005DD1D5F808C01CF0030E00F08C8095F8FA
:106D300050C063F3410C1CF0020F85F850C05FFA9D
:106D40008CF34ED190424CD0DB077FF57FAFAB6A1E
:106D50009A7B002A00F09E80B5F90EA0B5F92EB0FE
:106D600093F904201888B5F92CC0B5F90CE0D34488
:106D700012FB0BF2024412B2AA8593F905000192AC
:106D8000F4445A88B5F932B010FB0CF0104400B24C
:106D9000E88593F904C0D344B3F800A01CFB0BFCB6
:106DA000D4440FFA8CFCB5F930B0A5F830C093F993
:106DB00005A05B886963DE441AFB0EFA53441BB2DC
:106DC00098426B86C8BFEB85019BC8BF68869C450F
:106DD000BCBF2B86A5F82CC005F12C0136E701239A
:106DE000A5E7E96405F1440130E7B5F944B0B5F928
:106DF00048A0B5F93AC0B5F946E0B5F93E30019181
:106E00005845A8BF58465245B8BF5246F445A8BF9A
:106E1000F446B5F94AE0A8857345B8BF734605F155
:106E20002C0A2A866B86A5F82EC05046F8F718F86B
:106E30002A8A6B8A019903FB02F3B0EB430F22D835
:106E40006963514602E7DFF8B4A0DCF8003053452F
:106E50004CD073466BE7BAF914C0BAF918E0E645AE
:106E60003FF45CAF0AF114039942CAF81C1040D0F9
:106E7000EB8A012B3FF43FAF95F8503043F002030B
:106E800085F850304AE705F138032964EB6405F1D1
:106E90004401DBE6B5F90CA0B5F92CB093F9042058
:106EA0001888B5F92EC0B5F90EE0D34412FB0BF2E9
:106EB000024412B2AA8593F905000192F4445A885B
:106EC000B5F930B010FB0CF0104400B2E88593F92E
:106ED00004C0D344B3F800A01CFB0BFCD4440FFA4D
:106EE0008CFCB5F932B0A5F830C060E79CF80C30E6
:106EF0001DE795F8503011E7D0A2080034FD0700D7
:106F00004CFF070028FB070094F6070008FE070067
:106F1000084B187910F0010000D17047064A137829
:106F2000C3F380005B07F8D51078C0F3C00080F091
:106F300001007047B0060120FC3B012008B5FFF7B7
:106F4000E7FF034A034B00280CBF1046184608BD54
:106F5000EC190800F81908002DE9F843DDE9087874
:106F60002AB30C461E4615464FF0000913E0E1789F
:106F700001F00301B14212D1FBF7F6FFD0B1A378C3
:106F8000DA0914BF88F800303B70237809F1010951
:106F90004D451C440BD06378052B2046E7D0094BA8
:106FA0001B68DA0700D500BE0020BDE8F883012089
:106FB000BDE8F883034B1B68DB07F5D500BEBDE8D1
:106FC000F88300BFF0ED00E008B5104A8B88107818
:106FD000DBB2984212D10B7803F06003202B01D072
:106FE000012008BD4B78092BFAD14888CB8818328C
:106FF000010AC0B2F4F758FB012008BD044B186821
:1070000010F00100EDD000BE002008BD38200120A6
:10701000F0ED00E02DE9F0414589ADB245B30B46F6
:107020004189878889B28A428CBF45891546C289C1
:1070300088BFADB215FA82F2BA4204461BDCC189A0
:10704000C288066889B2184602FB016102FB05F29C
:1070500040F0F4FCE389A28815FA83F39BB29342D3
:1070600024BF9B1A9BB2E38163895B1B9BB2638144
:107070002846BDE8F081C689C089E188B6B21FFA0A
:1070800080FCA7EB060820681FFA88F808FB01F2CD
:1070900001FB0C01184640F0D1FCE289A18818FAE6
:1070A00082F292B28A4224BF521A92B2E28161897C
:1070B000E288F61BB6B216FA81F189B26181E189E4
:1070C00027682E44B6B289B208FB020002FB0171A8
:1070D00002FB06F240F0B2FCE389A28816FA83F3C1
:1070E0009BB2934224BF9B1A9BB2E38163899E1B90
:1070F000B6B266812846BDE8F08100BFF8B512B986
:1071000000242046F8BD224D95F82E310E46144637
:1071100005F59577E3B904223946A818FFF77AFFF9
:107120000028EDD095F82A2102F00F03052B0BD093
:107130000F2B09D002F00B02022A24D00C3B012BAA
:1071400023D903231A4601E001231A4685F82E218C
:1071500095F82F219B1A9C4228BF1C460132B91872
:107160003046224640F06AFC95F82F3195F82E21E2
:107170002344DBB29A4285F82F3104BF0023A5F8DF
:107180002E312046F8BD1346E0E702231A46DDE71C
:10719000DC2201202DE9F04F2DED028BD5B02B9391
:1071A0000890002802F061820F4609689046044664
:1071B000F9F782FD031E1A460393C2F22C823B6844
:1071C00013443B602668002E02F04882089AD2F8E9
:1071D00004A0BAF1000F02F041823278002A00F0D8
:1071E0001483327F4293032A14BF11220922029290
:1071F000049242AA0821029B45931446104608EEC9
:10720000102A0022CDE94322F9F7F6FCCAF8000063
:10721000337F032B0CBF012102212046F9F7ECFC40
:10722000CAF804000899D1F8C427002A40F38180E5
:10723000D1F8BC3718EE105ACDE905A7D3464FF068
:1072400000090F46002B6CDD5C464FF0000A0C2154
:107250002846F9F7D1FC0921A0622846F9F7CCFCB1
:107260000821E0622846F9F7C7FC20633378002B39
:107270000CBF042109212846F9F7BEFC01216063F7
:107280002846F9F7B9FCA063002801F042860221E4
:107290002846F9F7B1FC0121E0632846F9F7ACFC78
:1072A000052120642846F9F7A7FC052160642846DB
:1072B000F9F7A2FC0023C4E9120303212846F9F7D9
:1072C0009BFC032120652846F9F796FC03216065A5
:1072D0002846F9F791FCE36BA065002B41F0BA87D3
:1072E000E26D6363C4E90A33C2F1140222663378A3
:1072F000002B01F02D860020606601212846F9F759
:107300007BFC0121A0662846F9F776FCE066D7F8F9
:10731000BC370AF1010A9A4504F1480497DBD7F813
:10732000C42709F1010991450BF1900B8ADBDDE9D6
:1073300005A70899DAF80030C1F8D8373B68049AF5
:107340001344DDE902023B60D8F8003002449B1A86
:10735000C8F80030D1F8B827002A02F02D80D1F803
:10736000B027002A42F0C180D1F8CC679E4202F3D8
:107370008681089CD4F8DC17D4F8D827914223469C
:10738000C2F24C811C33891A194418461D461093C9
:1073900040F082FBD4F8D807D4F8CC2739682844C9
:1073A00040F04CFBD4F8CC17D4F8D8270A44C4F8E2
:1073B000DC273B680B443B60D4F8CC27D8F800307E
:1073C0009B1AC8F80030D4F8DC27D4F8C437D200B0
:1073D000002B119241F3AB83002320932993069352
:1073E0000393089B03F5FC632A93089BD3F8BC37EF
:1073F000002B40F3C583299B44331293209B0993B0
:107400002A9B199300239B46089B1D68002D01F0C1
:10741000BC875A680292002A01F0B7879C68002C4A
:1074200001F0B3870699119A0A4410990023CDE917
:107430002C132E93D31D48BF02F10E03DB102F93A4
:10744000069B002B41F033852B78002B41F03284D2
:10745000039D05EBC5030BEBCB021B0103EBC20342
:10746000029A1344BC4A586BD96B12F8109002EB85
:107470004002022956784FEACB004FEAC502059038
:10748000079201F0D385039B002B01F04B864FEA56
:107490000B13029A083302EB0308D358002B01F0B8
:1074A0007686CBEB4B11099A4800611D431E013AC9
:1074B00001444FEA4B1023442244049013F8010F77
:1074C00002F8010F9942F9D1D8F80430002B01F0ED
:1074D00075860398049AC0EB4013A2EB0B029B0045
:1074E00003EB420304EB4202234491799971D17971
:1074F000D971117A1972517A5972927A9A72D8F8AE
:1075000008304FEA4019002B01F07086049B099A5D
:10751000A3EB0B00410001F10B0304F110000B324F
:1075200023440844224413F8011B02F8011B98422B
:10753000F9D1D8F80C30002B01F01786049B099A7A
:10754000A3EB0B00410001F1100304F11500103210
:1075500023440844224413F8011B02F8011B9842FB
:10756000F9D1039BA9EB0309049B4FEA8909A3EB1B
:107570000B0309EB43094C4400236375A375079B78
:10758000039A109C02992C98199D9A18059B120138
:107590005B4402EBC3022E9B001B1144C3EBC003F0
:1075A0000698896A45F8041B181A04EBE3040C9446
:1075B0000C1A0294119C1995201A1A90002B03F0B2
:1075C00007001090C1F2E186A14201F3DE86089B1C
:1075D0001968002900F004815C680D941846002C9D
:1075E00000F0FE809B68002B00F0FA80C3681793C0
:1075F000002B00F0F580029B002BC0F2F1802244AA
:10760000936B1BB1D36B022B01F06A85039A079B26
:10761000496B1344059A1B015A4403EBC2030D9AAC
:107620001344D3E91702431C1A44013231F91330D1
:1076300031F91220079903980D9C179DCDF870B071
:1076400008180599000101EB0B0600EBC600204469
:1076500005EB8B01C06A4000B0F5107FA8BF4FF466
:1076600010708242A8BF02468342A8BF0346CDE9FC
:10767000433205EB0623189343AB0B93129B1E90EA
:10768000E31801F590570A93109B069301460C9B53
:107690004591002032021B970F901D923960049390
:1076A0000B9A0F9852F8043B0F93A3EB000ABAF120
:1076B000000F0B9240F37A81029B002BC0F2908066
:1076C0000A9B264E1D68069B04995B4206EBC50289
:1076D00013F0070318BF11F8017B14791CBFC3F125
:1076E000200207FA02F2189F08BF1A4607EB80092A
:1076F000002C01F0D2821A48DFF868E050F825C06B
:1077000002980EEB4C07012CA0EB03000E9701F042
:107710005D83A71E012F63D856F835C00E9F0CF16C
:1077200001051395CDE9154ACCF1200514950025E6
:1077300011950F2840F3AB804D7811F8024BC3F13F
:10774000100EC3F1180605FA0EF5B44025431038A3
:107750002A43103308E000BFE0BC0700BCA90800C2
:10776000BCAA08003CAB08000A2BE2DD3D8805F00E
:107770000F05C5F1200422FA04F4013437F814404F
:107780005FEA143E7ED0C4F30326C4F303140F2C27
:10779000A3EB0E0302FA0EF235462CD07CBB0F2E63
:1077A00011D0A5B9119EB3421ADB169F4E46023F77
:1077B000002F46F8084B1697C9F8045041F3F0859E
:1077C0000E9FB146D0E7159D032D7FD0354602F0C0
:1077D00000463543119E013BB3424FEA4202E4DAD0
:1077E00008982B99FAF7F0F86FF0080055B0BDEC47
:1077F000028BBDE8F08F159F032F00F09A8002F0F6
:107800000047013B3C435200C9E7327F4293032AC1
:1078100014BF202211220292049242AA0921029B43
:10782000459310460025144608EE102A9146CDE9EE
:107830004355F9F7E1F9CAF80000337F032B0CBF79
:10784000052103212046F9F7D7F9089BCAF804005F
:10785000D3F8BC37AB427FF7E5AC0AF11804A4F1CA
:10786000100B01214846F9F7C7F94BF8040BA34563
:10787000F7D1089BD3F8BC3701359D4204F11004C1
:10788000EDDBCFE45B1BAA4007EB44076CE7C418B1
:10789000002CA5DD002805DD11F8015BC3F11806F9
:1078A000B5402A43082805DDC3F1100011F8013B5B
:1078B00083401A434FF00040631E40FA03F30B204D
:1078C0001A40119004F10B0300204DE7139E1D1880
:1078D000AE4285DC9E4241F32284ACEB0305ED0809
:1078E0006E1C0E44C3F1180711F801EB0EFA07FEE7
:1078F0008E4242EA0E02A7F10807F5D10838C5EB1F
:107900004571083310EBC10003EBC50307D50344F1
:10791000591E4FF0004040FA01F10A40002014992E
:1079200022FA01F5A3EB0C0331460F3502FA0CF2F3
:1079300037E7139C002E18BF0134A2461C18A2453D
:107940003FF74EAF534528DADC4304EB0A0701EB5F
:10795000D7070137C3F118088E461EF801BB0BFA92
:1079600008FB774542EA0B02A8F10808F5D1544418
:10797000E4080838C4EB4477083304F1010E10EB37
:10798000C70003EBC403714407D50344581E4FF0EE
:10799000004444FA00F002400020149C22FA04F44F
:1079A000A3EB0C030F3402FA0CF2F7E60020029A64
:1079B00090423FF715AF069B121A0344029203F060
:1079C00007020692049A02EBE30304930A9B043332
:1079D0000A930B9B46AA9A427FF462AE029BDDF8A3
:1079E00070B0002B41F37982039A079B25490498D4
:1079F000029E1344059A1B015A4403EBC2030D9ADD
:107A00001A44D36E204A51F8231052F82340069BA3
:107A10005B4213F007031EBF10F8015BC3F12002A5
:107A200005FA02F21E9DC5F50F7808F1010808BF9E
:107A30001A46B8F1000FA6EB030E41F34E82C4F1D3
:107A4000200A124C189E4FF00009611806EB8506BB
:107A500007914D46BEF10F0F41F3F98090F801C038
:107A600010F8021BC3F11004C3F118070CFA04F458
:107A7000B9402143AEF1100E0A43103306F1100451
:107A80000AE000BFC8D20800C0D20800D0D2080067
:107A9000092B04F11004DDDD079E22FA0AF1715C66
:107AA0000E0911F0080CA3EB111302FA06F205D02F
:107AB00002F0004C013B4CF0010C520011F00407A5
:107AC00005D002F00047013B47F00107520011F0DA
:107AD000020605D002F00046013B46F001065200C6
:107AE00011F0010105D002F00041013B41F001011C
:107AF00052004B4507DB0435454544E9026144E942
:107B000004C72646C4DB1B9A13681D44B5F5107FD5
:107B100015600FDA059B5B4405EB8315179B03F596
:107B2000106203EB85051D9B1A44002345F8043BB6
:107B3000AA42FBD1069B029A1344049A02EBE3018A
:107B400003F0070306930C9BC91A3FF549AE109B3F
:107B50000698089AC3EBC10303441A98D2F8BC27CD
:107B6000C31A11930C9B0B441093129B483312932E
:107B7000099B0BF1010B3E3393450993FFF644AC8F
:107B800003990898FDF70CFD0028C1F27185089B48
:107B9000D3F8BC37002B40F3F685299B2833259377
:107BA00000232193089B1B68002B01F0E384089AB3
:107BB000546823941146002C01F0DC84D2F80CB0F8
:107BC000BBF1000F01F0D68452690492002A01F043
:107BD000D1841A78219E5B6BC34F002A039A0CBF95
:107BE0000821062102EBC20233F91130120106EB23
:107BF000C60002EBC00287FB03152244DB17C3EB70
:107C0000A5031CB2D16B039B1994DB00F40002297D
:107C10002494269301F0788306F5906340F226229F
:107C20005BF82330934241F38A83030205930BEB05
:107C300000231C9340F23623079320230C93F8274C
:107C40001F231F441C9BDFF8B8A2A84EA84D03EBCE
:107C5000C7070297D3E91112A64F084687FB00C059
:107C600094468AFB0CECA0EB0C004000586487FBA8
:107C700002028AFB0101186C114407F146774900A2
:107C800007F525379964DA6C014607F57D7787FBA0
:107C900001C1994C944684FB0CECA1EB0C0149000A
:107CA000196487FB021284FB0010D96B104440005A
:107CB000D8641A6D084686FB00C0944685FB0CEC20
:107CC000A0EB0C004000D86386FB020285FB01019B
:107CD000986B1144A4F18B444900A4F58204196502
:107CE0005A6D0146A4F6A20484FB01C1834F944659
:107CF00087FB0CECA1EB0C014900996384FB021299
:107D000087FB0010596B104404F1C774400004F560
:107D1000F03458659A6D0846103484FB00C0DFF8D3
:107D2000E4C196468CFB0E8EA0EB0E00400058631B
:107D300084FB02028CFB0101186BDFF8CCC11144FB
:107D400049009965DA6D01468CFB01E1DFF8BCE181
:107D500090468EFB0898A1EB0801490019638CFB43
:107D600002128EFB0010D96ADFF8A4C11044400053
:107D7000D8651A6E08468CFB00E0DFF898E1904663
:107D80008EFB0898A0EB08004000D8628CFB020232
:107D90008EFB0101986A114449000CF5453C1966B7
:107DA0005A6E0CF1310C01468CFB01E1DFF868E101
:107DB00090468EFB0898A1EB0801490099628CFB64
:107DC00002128EFB0010024452005A66029A483397
:107DD0009A427FF43FAF219D269B039A079E249CE5
:107DE000049F41490BEB850B0BF590509A180368E3
:107DF0009E42B8BF1E462C4433461201239E0360A8
:107E000002EBC40232441133126C239E07EB85054A
:107E1000002A07EBC41281FB0341059C279505F559
:107E2000D85C41F208203C444FEAE373C3EBA10362
:107E3000CDF8A0C027461A945BF80040DCF800009B
:107E4000229341F6083C259B189055F80C000E90A3
:107E5000334441F610301D930C9B28580D9002F5C9
:107E600090521998159408BF0020002B19901B926E
:107E700041F35783C4F107010020062C1F91C8BFAE
:107E8000014607EE901A1C99049007EB83030A90B1
:107E9000A1F10C061E93059209971D9A93695269E8
:107EA00007922BB1199B0A998B42C8BF00220792F7
:107EB0000D9B0A9A934200F3C4860E9B0799129376
:107EC0001A460A430292159B062B00F3A286059BD5
:107ED000DDF87CE0243306F14800002413939C462F
:107EE0001490234639AF19E0398EE338736E8D79DB
:107EF0004A3FE3D7F053C26D49499EC37611B7E8B4
:107F0000AA0025BE2FFEE4F3407EE47FC7A3C1FA9A
:107F100063B2FC7FC6BD2EFE5DC286FFD0E90115AF
:107F20005CF8042D45FA0EF5EB1A41FA0EF108380B
:107F30001C1B42FA0EF2CB1A86423C62CCF800209F
:107F400047F8043DEAD1DDE93814329DDDF8D0E090
:107F5000309F359A3798319E64100F94369CA5EB6C
:107F60000E09A9EB0103C4EB6708141A16934FEA34
:107F7000670C0B94339F824C05EB0E0384FB07A721
:107F8000A6EB020AAAEB000A1797D14684FB09A9BF
:107F90007C4C9A4684FB0ABA7B4F0D4487FB05B59F
:107FA000A1EB0E0184FB01E187FB03E307F17057AE
:107FB00007F54C27A2EB000E07F2CB2787FB0EBE7E
:107FC000724C304484FB00B01644324687FB026298
:107FD0000B9E274687FB06465B00C3EB41037600FA
:107FE00036993D9CC6EB4206179A0CEB610C6D006E
:107FF000400000EB4E0005EB4A050CEB420EACEBEB
:10800000420C05EB030B0EEB050A65442D1A0B958C
:10801000169D3B99409A8244CDF8C0A008EB650AB2
:10802000A8EB0508CDF8D0800AEB4908301A454680
:108030000CEB03087344ACEB0B0CAEEB0B0EACEB90
:10804000000C9B1B7044CDE935030B9B4198389382
:10805000B0440F9B3F9E3195A1EB040EAEEB000E9A
:108060003E98474DAAEB490A9E1BCDF8DCA0169618
:10807000CDE9328CDDF8F0903A9E01EB040A801ACB
:1080800085FB09393E9BA6EB030CACEB020CE046EA
:1080900085FB08383B4DD34685FB0B3B419F39445C
:1080A000394F87FB0131419F3B1B1F4685FB07373B
:1080B000354C84FB0A3A04F1705404F54C24844690
:1080C00004F2CB2484FB0C3C304D324485FB02325D
:1080D0003E9B1E4484FB063685FB00304FEA4A0374
:1080E000C3EB47030F9C3F9F169D490001EB4B01DB
:1080F00004EB67074000C0EB4600A7EB490407EB21
:108100004906CF180F970F9F520002EB4C0206EB67
:10811000010A04EB03093344F61BE71B0C4405EB8F
:108120006E0CA0EB020B0AEB0201A41A029A399121
:108130000CEB480AA5EB0E0EACEB480C8144A7EB08
:108140000B075E441B1ACDE93B97CDE93E63CDF8A2
:10815000F4E0CDF8E8A0CDF800C14194002A40F049
:10816000E9840B49DDF824E0DFF82C800598094B01
:108170000B9D01F1480938AF76469446934612E0CC
:10818000A1EBD96E8BBE0D627E1A3A16322E0E7E90
:10819000D40308005CEB270B64EC07003C6A58F83A
:1081A000043D57F8045D83FB042404EBA503D0F8D9
:1081B00000A040F8043B51F8082CA4EBA505CAF137
:1081C000000314465A1B82FB043451F8043C05EBAF
:1081D000840482FB0353CAEB83034EF8804B624650
:1081E000C6F8803884EAE472A2EBE472644683EA5B
:1081F000E374A4EBE3740831224389454BEA020B94
:10820000A6F18006CAD1CDF808B00A9D099C05994F
:1082100017EE903A2A462046F9F7FEFA2A460299C6
:10822000149E01320A92049A0843024323460492A0
:108230001E9A1399059104339A4209937FF42DAE47
:108240000C9B1C9A229903EBC30302EBC3021C9202
:108250001B9A02EB83031B930C9B8B4281F2698177
:10826000159A1C981793062AC2F107021692C8BFE6
:10827000002206EE902A1B9A02F1240B1A9A02EBB6
:108280008303059302EB810300F104081493DDE9F5
:108290000D230C9CA242C8BF002307EE103A159B89
:1082A000ABF12401062B07EE901AA8F1040013DCB1
:1082B000169C002250F82230234140F8223058F812
:1082C0002230234148F8223051F8043B0232234146
:1082D000122A41F8043CEDD1D8F83870D8F82C5067
:1082E000D8F82010D8F81400D8F8082058F8044C12
:1082F000B84EED1B491B401A131AC91BE41A5B1A2E
:1083000064105B1086FB002004EB650909EB400A52
:10831000651BA9EB400986FB012103EB670E0EEB01
:108320004106AD48490080FB0626AC4CDB1BB6007D
:1083300084FB03239B00AEEB010E0293A84981FB53
:108340000E2ED8F83C20D8F83070D8F82400D8F891
:108350001840D8F80C10D8F80030BF1AC01BA4EB96
:10836000000CA1EB0C010AEB0604AAEB0606A3EB3A
:10837000010A029B3094801AEC18091AEB1A09EBD7
:108380008E05A9EB8E0ECDE9325E3596319434938D
:108390004FEA6A0A49108F4D85FB0C3C0AEB6704D3
:1083A00004EB4C09AAEB0707A4EB4C0C85FB00304F
:1083B00001EB620404EB4006874D400085FB063666
:1083C0008A1AB60011460296844A82FB0131241AA9
:1083D0008A00834880FB0434D8F83450D8F840E051
:1083E000D8F82810D8F81C00D8F81030ACEB840668
:1083F000A5EB0E0A3996029ED8F80450A1EB0A01AB
:108400000CEB840C401ABC1A1744A9EB06024E442C
:108410001B1AA1EB0E010796079E3A94ED1A5B1A00
:10842000CDF824C00A97CDF8E0C037973B92369636
:108430006D105B10674C84FB002005EB6A0202EBB9
:108440004006A5EB0A05A2EB400084FB012103EBEB
:108450006E0202EB41044FEA410C5F4981FB047458
:108460005E49A3EB0E03A40081FB03735C4FA2EBF8
:108470000C019B0087FB0121A0EB810CEF18ED1A8A
:1084800000EB8103CDE93E3CA6EB040E331917EE59
:10849000102A18EE101A17EE900A4095CDF804E154
:1084A0000B933D97F9F72CF9059B4E491A46CDE9F8
:1084B000128B03F5C0730F9318EE10CA00230DF151
:1084C000C00E32AD02935CF8043B4FF000089B00F5
:1084D00083EAE378A8EBE3781360DCF808304FF028
:1084E000000A9B0083EAE37AAAEBE37ADEF80C0049
:1084F000C2F8803151F8043B044683FB0464DCF885
:108500001430002604EB830383EAE376A6EBE376DC
:10851000C2F80033EF688B6883FB0747DCF8203034
:10852000002407EB830383EAE374A4EBE374C2F84B
:1085300080342F684B69043D83FB079751F8043C56
:10854000DEF824909B468BFB0939DCF82C304F4435
:1085500007EB8303002783EAE377A7EBE377C2F80F
:108560000036DEF800000B6A0EF1040E83FB00906B
:108570008B68D5F828909B468BFB0939DCF838309E
:10858000484400EB8303002083EAE370A0EBE37030
:1085900048EA0A0949EA06063443C2F88037274305
:1085A000029B3843034302930F9B803293428AD14C
:1085B000079B9E100A9BDDE9128B9A10099B9C1069
:1085C0004BE909624BF81C4C0B9AABF118043CAB1D
:1085D0000CE000BFA1EBD96E1D75A37B9A79825A7E
:1085E00083FB202180CD080053F8042F921044F81B
:1085F000042B5C45F8D10C9E059D17EE901A16EEE3
:10860000903A32462846F9F707F932460132029984
:108610000C92049A01430A432B460492149A0433A1
:108620009A42059304F1240B08F148087FF42FAE19
:10863000179A229B9B1A1B9A03EBC30302EB83033B
:108640001B93189B1946229B994240F37A8754AAA0
:10865000DDF86C80059218EE109A1E4600241F4625
:10866000DDE90D13B942C8BF00231A46404649460A
:10867000F9F746F807F0010302931A9BDDF810B0F2
:1086800007EE909A47F3000A4A4603EB870CA8F1DD
:10869000040E002013684FEA8309CCF800902146AD
:1086A00089EAE971A1EBE9715368029D8AEA8303C3
:1086B0002B4449EA030940EA0900CCF88030A1467E
:1086C00083EAE379A9EBE379059B4EF8044F08327E
:1086D00041EA090193424BEA010B0CF5807CD9D1A8
:1086E000189BCDF810B0002818BF3E460137BB429A
:1086F00017EE909A08F12408B2D1189B1F2B10DCBA
:108700001A9B1899002003EB81031A4603F51064A5
:1087100042F8800B9442FBD10131202903F104037C
:10872000F3D1049B002B00F04186C0F21F8704990F
:10873000002349001A4603F10103FAD50399269B49
:10874000219D2798199C0B4424991B01294403EB74
:10875000C103239919440B4628990E6041F6083647
:10876000DB6B835141F6183141F61036089B84517A
:1087700042502599D3F8BC376A1C48319A4221925D
:108780002591FFF60FAA0898039CD0F8C827C16866
:1087900002FB04F42B9A03FB04F402EB44040029CB
:1087A00000F0748742690B92002A00F06F8782699B
:1087B0000C92002A00F06A87022B00F0E6860C9BE0
:1087C00003F5085309931A680B9B03F5D85300214E
:1087D00004F1400018330791059088460D934FF03F
:1087E000007A4FF00C0907980D9B0C9D0B9C1B68A1
:1087F000009300F001010E460A910B4604EBC010F5
:108800002946F8F741FB099B32011B68324403EB10
:10881000821305EB830455F82300E16D534642466D
:10882000C0FB08326FF07300C1FB00324FF4557C7F
:108830006068A16DC0FB0C32CE48C1FB003241F62E
:10884000D477A068616DC0FB0732CB48C1FB003212
:1088500046F2B865E068216DC0FB0532C748C1FB30
:108860000032C74E2069E16CC0FB0632C548C1FB2F
:1088700000326069A16CC0FB053245F28400C1FB87
:108880000032A069616CC0FB073240F22C70C1FB62
:108890000032E069216CC0FB0C327420C1FB003255
:1088A000142002FA09F142FA00F223FA00F343EA33
:1088B00001035915B1EBE37F4FEAE37218BF82F46D
:1088C000FF4305990CBF9B1183F07F0304F5805291
:1088D00021F8403C11684FF4D07052464346C1FB2A
:1088E000002341F2040141F67C006158C1FB0023E2
:1088F00041F2080149F2FC706158C1FB002341F2CA
:108900000C01A1486158C1FB002341F210019F48AE
:108910006158C1FB002341F214016FF0B3006158AC
:10892000C1FB002341F218014FF412706158C1FBE2
:10893000002341F21C016FF013006158C1FB0023BA
:10894000142003FA09F143FA00F322FA00F242EA92
:1089500001025115D317B1EBE27F18BF83F4FF4238
:10896000059B8B4D02930CBF921182F07F0223F87E
:10897000202CA3F14002049268266FF0030747F60B
:10898000FF7E01E055E91076D4F800B1D4F85CC15F
:1089900052464046CBFB072053464146CBFB0631AF
:1089A0007642CCFB0620CCFB073155E90E7CD4F88F
:1089B00004B1D4F85861CBFB0720CBFB0C31CCF1D0
:1089C000000CC6FB0C20C6FB073155E90C7CD4F823
:1089D00008B1D4F85461CBFB0720CBFB0C31CCF1B0
:1089E000000CC6FB0C20C6FB073155E90A7CD4F805
:1089F0000CB1D4F85061CBFB0720CBFB0C31CCF190
:108A0000000CC6FB0C20C6FB073155E908CBD4F897
:108A10001061D4F84C71C6FB0C20C6FB0B31CBF1B6
:108A20000006C7FB0620C7FB0C3155E906C6D4F883
:108A300014B1D4F84871CBFB0C20CBFB0631764245
:108A4000C7FB0620C7FB0C3155E904C6D4F818B1A2
:108A5000D4F84471CBFB0C20CBFB06317642C7FB2C
:108A60000620C7FB0C3155E902C6D4F81CB1D4F876
:108A70004071CBFB0C20CBFB06317642C7FB0620B6
:108A8000C7FB0C31142700FA09F640FA07F022FA66
:108A900007F242EA06025615D017B6EBE27F18BF7E
:108AA00080EA0E02049808BF921120F8022F049069
:108AB000142001FA09F241FA00F123FA00F343EA23
:108AC00002035915DA17B1EBE37F18BF82EA0E03F0
:108AD000029A08BF9B1122F8023D2E4B02924035AC
:108AE0009D4204F580747FF44DAF09990A9B0A6892
:108AF0000598D21A079B013302F007024030122B6F
:108B0000079305900A607FF46EAE2999089B039A3B
